:1000000000800020BD01000031D20000E9D10000D5
:10001000E9D10000E9D10000E9D10000E9D10000F8
:10002000E9D10000E9D10000E9D1000031D200009F
:1000300031D20000E9D10000B9F40000BDF50000A4
:1000400031D2000031D2000031D2000031D20000A4
:1000500031D2000031D2000031D2000031D2000094
:1000600031D2000031D2000031D2000031D2000084
:1000700031D2000031D2000031D2000031D2000074
:1000800031D2000031D2000031D2000031D2000064
:1000900031D2000031D2000031D2000031D2000054
:1000A00005B3000011B3000031D2000031D20000CE
:1000B00031D2000031D2000031D2000031D2000034
:1000C00031D2000031D2000031D2000031D2000024
:1000D00031D2000031D2000031D2000031D2000014
:1000E00031D2000031D2000031D2000031D2000004
:1000F00031D2000099F7000031D20000C5F80000AD
:1001000031D2000079DF000031D2000031D200008E
:1001100031D2000031D2000031D2000031D20000D3
:1001200031D2000031D2000031D2000031D20000C3
:1001300031D2000031D2000031D2000031D20000B3
:1001400031D2000031D2000031D2000031D20000A3
:1001500031D2000031D2000031D2000031D2000093
:1001600031D2000051E2000031D2000031D2000053
:1001700031D2000031D2000031D2000031D2000073
:1001800031D2000031D2000031D2000031D2000063
:1001900031D2000031D2000031D2000031D2000053
:1001A00031D2000031D2000031D2000031D2000043
:1001B00031D2000031D2000031D20000564B4CF257
:1001C000205210B51A804DF628121A8000BF00BFC9
:1001D0000DF032F8514B4FF010621A60504A9A609D
:1001E000504ADA60504A136813F4807304D14F49BF
:1001F0000B604FF4A85313604D4B1A78110703D5C9
:100200001A7842F008021A704A4B4B492A221A7097
:100210004A4A4B4B8B4204D252F8040F43F8040B6A
:10022000F8E7484B484900228B4202D243F8042B9E
:10023000FAE74649464A002352F8230041F82300D2
:1002400001336F2BF8D1434B434A802103F8011B44
:100250009342FBD1414B3D4A1A60414B8A221A70AE
:10026000A3F5805324225A70A0221A709A7992071B
:10027000FCD59A79D406FCD43A4A937903F00C035E
:10028000082B384BF9D103221A7140225A719A79FE
:100290009006FCD5334A9179324B4906FBD5324A58
:1002A000324911600221516020221A709A7902F0BD
:1002B0000C020C2AFAD12E4B2E4A1A602E4B2F4AD2
:1002C0001A6000225A60072243F8042C2C4AC3F813
:1002D0000C2D62B60DF018FD144B1B68DA0705D51E
:1002E00028480DF0E5FA284B284A1A60284B1B785D
:1002F0005B0609D5244C254B22689A4204D121483B
:100300000DF0D6FA0023236010F0E4FD0CF09AFF04
:100310000FF0C8F9FEE700BF0E2005403080044012
:10032000823F04000100002B10D0034014D0034092
:1003300002D0074000E007403C9DFF1FC045010080
:100340004088FF1F3C9DFF1FB4A3FF1F0082FF1FBB
:100350000000000000E400E05FE400E008ED00E0E1
:100360000050064000400640448004400000030165
:1003700004800440C010050014E000E0FF76010096
:10038000000020207814E95C1CE00340A5C3945AC7
:1003900000F00740FFFFFFFFFFFFFFFFFFFFFFFF32
:1003A000FFFFFFFFFFFFFFFFFFFFFFFFFFFFFFFF5D
:1003B000FFFFFFFFFFFFFFFFFFFFFFFFFFFFFFFF4D
:1003C000FFFFFFFFFFFFFFFFFFFFFFFFFFFFFFFF3D
:1003D000FFFFFFFFFFFFFFFFFFFFFFFFFFFFFFFF2D
:1003E000FFFFFFFFFFFFFFFFFFFFFFFFFFFFFFFF1D
:1003F000FFFFFFFFFFFFFFFFFFFFFFFFFFFFFFFF0D
:10040000FFFFFFFFFFFFFFFFFFFFFFFFDEF9FFFF23
:1004100010B5054C237833B9044B13B10448AFF33E
:1004200000800123237010BD3C9DFF1F00000000D1
:10043000C4450100084B10B51BB108490848AFF38B
:1004400000800848036803B910BD074B002BFBD0A0
:10045000BDE81040184700BF00000000409DFF1F8E
:10046000C44501003C9DFF1F0000000070B44C68B3
:10047000A04220D901230133DBB21CB2A60051F8FF
:10048000244084421D46F6D3A04211D005F1804598
:10049000013D965951F8251052F82530401AF21AAC
:1004A00000FB02F0641AB0FBF4F4E01870BC704773
:1004B000905970BC704704260125E5E700280CDA46
:1004C000064A434282FB0320DA17C2EB600000EBCE
:1004D0004000A3EB8000C0F10C007047ABAAAA2A31
:1004E000684B1B880C2B12D8DFE803F01E29333D24
:1004F0001148525C66707A12070063490B68984293
:1005000078D90B6C9842C0F0A580604B186C70478E
:100510005D490B68984240F28E800B6C9842C0F0A7
:1005200096805B4B186C704757490B6898427FD98F
:100530000B6C9842C0F08880564B186C704752493B
:100540000B68984271D90B6C98427AD3524B186C55
:1005500070474D490B68984264D90B6C98426DD333
:100560004E4B186C704748490B68984257D90B6C32
:100570009842C0F084804A4B186C704742490B681F
:10058000984249D90B6C984276D3464B186C704709
:100590003D490B6898423CD90B6C984269D3424B59
:1005A000186C704738490B6898422FD90B6C9842E9
:1005B0005CD33E4B186C704733490B68984222D984
:1005C0000B6C98424FD33A4B186C70472E490B680E
:1005D000984215D90B6C984242D3364B186C704731
:1005E00029490B68984208D90B6C984235D3324B95
:1005F000186C7047254B186870472F4B1868704768
:100600002C4B186870472A4B18687047274B18689E
:100610007047254B18687047224B18687047204B6D
:10062000186870471D4B186870471B4B1868704757
:10063000184B18687047164B18687047174AFFF731
:1006400015BF154AFFF712BF124AFFF70FBF104A36
:10065000FFF70CBF0D4AFFF709BF174AFFF706BFA8
:10066000144AFFF703BF124AFFF700BF0F4AFFF714
:10067000FDBE0D4AFFF7FABE0A4AFFF7F7BE084A69
:10068000FFF7F4BE989EFF1F988AFF1F848BFF1F01
:10069000408BFF1F488DFF1F3889FF1F048DFF1FF0
:1006A000C08CFF1FA08DFF1F7C89FF1FC089FF1F0B
:1006B000048AFF1F648CFF1FFC8BFF1F38B5284A7C
:1006C000284B14881D68AC4247DA274A274B10682C
:1006D0001B88421F191BAB42A8BF2B469142A3EBBC
:1006E0000403C3BF043843430131534393FBF1F187
:1006F00005310A200DF0EEF81D4A1E4B14881B68C8
:10070000A34205DC00210920BDE838400DF0E2B825
:1007100019491A4A0D881068AB42A5EB0401A0F1F3
:100720000502A8BF2B4691420CDD1B1B043800FBC1
:1007300003F30131092093FBF1F1BDE838400531A5
:100740000DF0C8B81B1B02FB03F3092093FBF1F16A
:10075000BDE8384005310DF0BDB80021C9E700BF44
:10076000169EFF1FD49EFF1FF88DFF1FE89EFF1FE0
:10077000E49DFF1F689DFF1FC89EFF1F8C8DFF1FFC
:100780002DE9F04F8FB002AD0024E1B26E480AF0BF
:100790002DFE01340C2C45F8040BF6D16B4B6C4C40
:1007A000B3F800E00A9B00227345227014DB089B1B
:1007B0009E4500F3B480069B664A9E4503DD137890
:1007C000002B40F0BC80049B9E4540F3AE804FF070
:1007D000020C84F800C009E0069B5E4A9E45CCBF2F
:1007E0004FF0060C4FF0050C84F800C00C9F039EE0
:1007F0000598079982F800C0BE45D4BF002701279D
:10080000B645D4BF002601268645099ADFF87081D7
:100810000B9B0D9DDFF86CA1DFF86C918AF80060EE
:10082000D4BF002001208E45D4BF0021012188F8CB
:10083000001096454849DFF854B1484E89F8000049
:10084000D4BF002201229E45D4BF002301230A7099
:10085000AE45434A8BF80070D4BF00250125012026
:10086000137035700DF0F4FB3E4B3F4A1D68118844
:100870003E4BA842D4BF002201220B291A7001D995
:100880000C2901D0A84246DC00230193384B9AF88A
:1008900000E01F7899F800C098F800209BF800301D
:1008A0002D49DFF8ECA091F800902D49367891F8A9
:1008B00000802478A7EB4E07CCEB070CA2EB82025A
:1008C000C3EB83776244C3EB8703134403EB490311
:1008D000BAF80020274FDFF8BCE0B7F800C0264F79
:1008E000434403EB8606033A0C2313FB046602EB36
:1008F000420206EB8202019BCEF800606244A842ED
:10090000A2F10C021A44C8BF1C4B3A60C8BF1E704B
:100910000FB0BDE8F08FA1F10C030193B6E74FF0E3
:10092000040C84F800C00B4A60E7029B9E45C6BFDA
:100930004FF0010C84F800C04FF0000C56E74FF068
:10094000030C84F800C051E7109EFF1FF09EFF1FAC
:100950003C9EFF1F489EFF1FD19EFF1F2D9FFF1F24
:100960002C9FFF1F548CFF1FCA9EFF1F949DFF1FCB
:10097000BC8CFF1FA49DFF1FF49EFF1FF29EFF1F54
:10098000299FFF1FC09EFF1F289FFF1F2A9FFF1F39
:10099000B29EFF1FF09DFF1F30B50E4C85B00123A6
:1009A00020463C2202210BF04FFF20460BF0DCFEDC
:1009B00001250022402180232046019100930295C9
:1009C0001146054B0BF0DCF9204605B0BDE8304080
:1009D0000CF06CB8009FFF1FC037010010B500EB92
:1009E000C000821DD2B293B284B09C1E981C3D23DD
:1009F00003918DE81900392102480BF025F904B064
:100A000010BD00BF009FFF1F70B50E4C84B01225B3
:100A10000422012306460390029320468DE8240019
:100A2000142310210BF010F90622092302930396D8
:100A3000019520460092142310210BF005F904B013
:100A400070BD00BF009FFF1F10B50C4C81B2204647
:100A50000BF0DCFB204602210BF0D2FB20462122CA
:100A60005A210BF0C9FB064B204619880EF012FEE6
:100A70002046BDE810400EF0BDBD00BF009FFF1F27
:100A8000B88CFF1F10B50C4C81B220460BF0BEFB9A
:100A9000204602210BF0B4FB204621225A210BF004
:100AA000ABFB064B204619880EF0F4FD2046BDE84E
:100AB00010400EF09FBD00BF009FFF1F948AFF1FD4
:100AC00010B50C4C81B220460BF0A0FB2046022151
:100AD0000BF096FB2046212253210BF08DFB064B99
:100AE000204619880EF0D6FD2046BDE810400EF0D5
:100AF00081BD00BF009FFF1FBA8CFF1F38B50C4699
:100B00000546C9B20CF048FB210A681CBDE8384014
:100B10000CF042BB38B505460CF024FB4FF0000446
:100B200060F30704681C0CF01DFB60F30F24A0B2F7
:100B300038BD00BF38B50F4D2B78013B01381B0283
:100B4000C4B203F47063200443F4404343F00C0345
:100B500000F4FE0018430EF04DF82868013860F0EC
:100B60003F00C0B20DF0E2F92046BDE838400DF07C
:100B7000DDB900BFFC9DFF1F38B5104D2B78013B40
:100B80001B0203F47063044643F41043000443F073
:100B9000090300F4FE0018430EF02CF82868013811
:100BA00060F06F00C0B20DF0C1F920460DF0BEF943
:100BB0000020BDE838400DF0B9B900BFFC9DFF1F13
:100BC00038B50E4D2B78013B1B0203F470630446CD
:100BD00043F45043000443F00D0300F4FE001843B7
:100BE0000EF008F82868013860F02F00C0B20DF050
:100BF0009DF92046BDE838400DF098B9FC9DFF1FD7
:100C000010B504464FF440600DF040F90DF098F92E
:100C10002CB1102C044BA8BF10241C6010BD024B3B
:100C200001241C6010BD00BFFC9DFF1F10B50446D1
:100C300041F0E0000DF07AF904F07F000DF076F954
:100C4000C4F3C610BDE810400DF070B938B5114DB1
:100C50002B78A0F50052013B1B0202F30D0202F5B6
:100C6000005203F47063044643F46043100443F0FD
:100C70000E0300F4FE005204184302F0FE4210433B
:100C80000DF0B8FF296801392046C9B2BDE83840E7
:100C9000FFF7CCBFFC9DFF1F2DE9F04F172087B059
:100CA0000DF0D6F9DFF86093C9F8000016200DF0BA
:100CB000CFF9B84BB84A1B8810600C2B00F04F825C
:100CC0000023B64C0F2023700DF0C2F9B44A2378EC
:100CD000128801921146B34A054652F821404BB1A1
:100CE00020460FF03BFE4FF07C510FF08BFE10F0D2
:100CF00065F80446AC4BDFF814831B88D8F800A0D5
:100D0000AA4A013B554552F823B050DAA84BA94EE8
:100D10001B88012B00F0D581A74BA84A30680093AF
:100D20001F4604920FF01AFE4FF07C510FF06AFE3E
:100D3000A34902900988039120460FF00FFE049A00
:100D400003993F6852F821100FF05CFE0146002025
:100D50000FF04EFD10F032F8CBEB070BAB45CAEBB2
:100D60000B015A46B8BF2A46CAEB02028842BABFF4
:100D700000FB02220131424392FBF1F0DFF890A226
:100D80000FF0ECFD4FF07C510FF03CFE02990FF09C
:100D900031FD10F013F830608A4A1288013A032AB4
:100DA0006AD8DFE812F0EB00D3005300DF00DFF871
:100DB00060A2DAF80020954238DD7D4B05921B8851
:100DC0007C4E012B00F0AC817B4B00931F463068BA
:100DD0007A4B04930FF0C2FD4FF07C510FF012FEDE
:100DE000774902900988039120460FF0B7FD0399D7
:100DF000049B3F6853F821100FF004FE0FF0DEFF54
:100E0000059ABB44C2EB0B01AB45A8BFAB46884279
:100E1000C2EB0B0B80F2AD8100FB0BBB01319BFBE6
:100E2000F1F00FF09BFD4FF07C51ADE7614E624B4E
:100E3000306800931F460FF091FD4FF07C510FF08A
:100E4000E1FD0FF0BBFF3F683060A5E738460FF0CB
:100E500085FD5D490FF0D6FD834628460FF07EFDE7
:100E60005A490FF0CFFD014658460FF0C3FC0FF072
:100E7000A5FF009B074618605549564A0888128806
:100E8000D9F80010544DC0EB070EC3199142C8F8B1
:100E900000E0CAF80030B5F800E080F2DC80002500
:100EA000C2EB0E0C3C4B64451F6880F2C880631C8B
:100EB000974205FB03F50CF1010C95FBFCF5C0F224
:100EC0006681BE45A8BFBE46C2EB0E0E03FB0EF404
:100ED00094FBFCF4914200F39D80BA42C0F29A80E8
:100EE0003E4C20680FF03AFD3D490FF08BFD3D4927
:100EF0000FF080FC0FF062FFA0F5FF531C3B082BA6
:100F000098BF4FF400503368184400282060C0F2A6
:100F10009480B0F5804F80F2A580334B1B781BB1D5
:100F2000B0F5005F40F0A680304D2B78002B40F0EC
:100F3000A9802F4D20682B68284C984203D0FFF7DA
:100F400085FE23682B6007B0BDE8F08F38460FF0B0
:100F500005FD28490FF056FD834628460FF0FEFC9C
:100F600025497EE738460FF0F9FC1D490FF04AFD90
:100F7000834628460FF0F2FC204972E738460FF00E
:100F8000EDFC1F490FF03EFD834628460FF0E6FCBE
:100F90001C4966E7CA9EFF1FFC9EFF1F659DFF1F41
:100FA000CC9DFF1F088BFF1FB88CFF1FC88BFF1F36
:100FB000F69DFF1F849DFF1FBC9EFF1F6C8AFF1FB5
:100FC000B89DFF1F948AFF1FCDCC4C3FCDCC4C3E2B
:100FD000BA8CFF1F2C9EFF1FB49DFF1F988DFF1F13
:100FE0009A99193FCDCC4C45DC9EFF1F119EFF1FE7
:100FF0003489FF1F6666663FCDCCCC3DCDCCCC3E60
:101000003333733FCDCC4C3DC89DFF1FE09DFF1F88
:10101000349EFF1F019B002B3FF462AF2B1B002B64
:10102000B8BF5B42092B34DC33685A4C4FF4005094
:10103000184400282060BFF66CAF002214E09742ED
:1010400005FB04F5B8BF002395FBFCF580F2968004
:1010500093FBFCF43EE77145D4BFC2EB0105C2EB44
:101060000E051DE743F6FF724B4B22601B78002BE9
:101070003FF45AAF00210D200CF0BCFD474B01227C
:101080001A7056E701210D200CF0B4FD00232B70DF
:101090004FE705F500500130001B0FF05FFC4049A1
:1010A0003C4C0FF0AFFC054620680FF057FC3D4963
:1010B0000FF0A8FC014628460FF09CFB0FF07EFEC7
:1010C00021E7394B00931F463068384B04930FF0EB
:1010D00045FC4FF07C510FF095FC354A0290128888
:1010E000039220460FF03AFC039A049B3F6853F8A2
:1010F00022100FF087FC0FF061FECBEB070BAB4526
:10110000CAEB0B02B8BFAB46CAEB0B0B8242C6BFA1
:1011100000FB0BBB013200FB0BFB9BFBF2F02DE64F
:10112000224B0493204B306800931F460FF016FCAF
:101130004FF07C510FF066FC1D4902900988039125
:1011400020460FF00BFC049B03993F6853F82110D5
:101150000FF058FC014600200FF04AFB4EE601203C
:101160000CF076FF134B1B689842D4BF0023012379
:10117000A7E500FB0BFB9BFBF1F052E67745D4BFE4
:10118000C2EB0703C2EB0E0304FB03F360E79646D2
:101190009AE600BF988DFF1FDC9EFF1F119EFF1F68
:1011A000CDCCCC3E9A99193FBC9EFF1F6C8AFF1F85
:1011B000B89DFF1F548CFF1F38B5054642F0B000A4
:1011C0000C460CF0B3FE28460CF0B0FEE0B2BDE8D1
:1011D00038400CF0ABBE00BF70B50F4D2B78013B13
:1011E0001B0203F47063044643F4304308062204F0
:1011F00000F0FE4043F00B03034302F4FE001843EB
:101200000E460DF0F7FC2A68013A3146E0B2D2B240
:10121000BDE87040FFF7D0BFFC9DFF1F10B50C4C20
:10122000236843B90B4B1B88022B0CD00A4A0023BE
:101230001370236010BD00210520FFF7CDFF054B83
:101240001B88022BF2D100214120FFF7C5FFEDE7FB
:10125000E49EFF1F209EFF1FE69DFF1F08B564212F
:101260000720FFF7B9FF7F210B20BDE80840FFF7FB
:10127000B3BF00BF10B500217B20FFF7ADFF0024F6
:10128000E0B2FFF779FC013402200CF0EFFC802C77
:10129000F6D110BD30B58DB06D460024E1B23448B2
:1012A0000AF0A4F801340C2C45F8040BF6D1314BAC
:1012B0000A9A1B889A4216DA009A934213DD029A20
:1012C000934210DD049A93420DDD2B4A2B4B11887B
:1012D0001B882B4A0B4412685B10934238DB294A67
:1012E0001268934201DB0DB030BD274B00241C7007
:1012F000FFF7C0FF21460D200CF07CFC32200CF0E3
:10130000B5FC01210D200CF075FC32200CF0AEFC78
:1013100021460D200CF06EFC32200CF0A7FC0121C0
:101320000D200CF067FC32200CF0A0FC21460D20B3
:101330000CF060FC32200CF099FC0D2001210CF027
:1013400059FC4FF42F700DB0BDE830400CF08EBC4E
:101350000D4B002101240D201C700CF04BFC3220A1
:101360000CF084FC0D2021460CF044FC3220EAE70E
:10137000109EFF1FF09EFF1FB49DFF1F2C9EFF1F9E
:10138000C89DFF1FFC9EFF1FA09DFF1F294A2A4BDF
:1013900010881B68294A2A491288834270B52DDBC0
:1013A0009342A8BF134698420B60C8BF002327DDB5
:1013B000101AB0F5804FAABF9B03C3EB83330130F3
:1013C00093FBF0F0FFF78CF81E4E3368C0F3C615A0
:1013D0009D42044606D01C4B1B882BBB1B4B1B8815
:1013E000F3B935601A4D2B689C4206D0164B1B880A
:1013F0005A1F032A0BD92C6070BD70BD03460860CC
:101400009A42D4BFC0EB0203C0EB0303D0E7114AFA
:10141000D05C04F07F012030FFF7DEFE2C6070BD51
:101420002846FFF7CDFBDCE70A4A2946D05CFFF7E8
:10143000D3FED3E7169EFF1FAC9EFF1FE89EFF1F43
:10144000D49EFF1FD49DFF1F909EFF1F129EFF1F63
:101450009C9DFF1FA88CFF1F2DE9F0417B4C7C4D0C
:1014600020680FF07BFA7B490FF0CCFA064610207B
:101470000CF0EEFD0FF072FA77490FF0C3FA314627
:101480000FF0B8F90FF09AFC2B882060002B3FD0AA
:10149000724F3A8890423BDB01467148067836B974
:1014A0004FF0010E042B80F800E000F0B380012B18
:1014B0006AD0022B00F0BC80032B36D1694B1B880D
:1014C000092B32D023683C88674AA342128853DB39
:1014D0009342D4BFC4EB0303C4EB0203141B7E2C62
:1014E000DFF88881D5BFC3EB8313C3EBC3135B0065
:1014F000013493FBF4F4D8F800300134A34203D054
:1015000021464A20FFF768FEC8F80040BDE8F08198
:10151000534A117849B10024012B147016D0022BC4
:101520001FD0032B03D0042B28D0BDE8F0814D4BF6
:101530001B88092BF9D04D4D2B68002BF5D0214687
:101540004A20FFF749FE2C60BDE8F081474D2A682C
:10155000002AEAD018462146FFF73EFE2C60BDE87F
:10156000F081424D2B68002BDFD021460420FFF78D
:1015700033FE2C60BDE8F0810023AFE72146402018
:10158000BDE8F041FFF728BE374B1B888B42D4BF24
:10159000C2EB0306C2EB01069A1ADFF8D0807E2A5E
:1015A000D8BFC6EB8616D8F80030C6BFC6EBC61645
:1015B0000132760096FBF2F60136B34203D0314693
:1015C0000120FFF709FE2B88C8F80060022B7FF48A
:1015D00073AF23683E88244AB34212882CDA002372
:1015E000961B7E2EDFF88480D5BFC3EB8313C3EB3D
:1015F000C3135B00013693FBF6F6D8F800300136D2
:10160000B34220D031460420FFF7E6FD2B88C8F80E
:10161000006051E77F214020FFF7DEFD2B88012B82
:10162000D4D121683A88104B91421B88B4DBADE7D6
:101630000D4A236812883E889A42D4BFC6EB020343
:10164000C6EB0303CCE70223E1E700BFBC9DFF1F0D
:10165000C49DFF1F9A99193FCDCCCC3E8E9DFF1F94
:10166000D89EFF1F909EFF1F469EFF1F289EFF1FB4
:1016700038B5114A114B14881B68114AA3421288CD
:1016800013DA0023141B0F4D7F2CCABFDB01C3EB01
:10169000C313013493FBF4F42B68A34203D0214617
:1016A0000520FFF799FD2C6038BD9342D4BFC4EBF1
:1016B0000303C4EB0203E5E7E49DFF1F689DFF1FE2
:1016C000C89EFF1FE49EFF1F10B5174B1B78DBB1B0
:1016D00015200BF063FC154B1860154A12887AB17F
:1016E00014491B68098899420ADC134C23781BB9FA
:1016F000022A13D001232370BDE81040FFF7B8BFC2
:101700000D4B1B7833B910BD11200CF0A1FC074B19
:101710001860E2E7BDE81040FFF780BD7F2141205F
:10172000FFF75AFDE6E700BF189EFF1F689DFF1FE9
:10173000209EFF1FE49DFF1FE69DFF1F38B5054655
:1017400042F090000C460CF0F1FB28460CF0EEFB4A
:10175000E0B2BDE838400CF0E9BB00BF70B50F4DFA
:101760002B78013B1B0203F47063044643F41043DF
:1017700000040A0600F4FE0043F00903034302F0EC
:10178000FE4018430E460DF035FA2A68013A3146FC
:101790002046D2B2BDE87040FFF7D0BFFC9DFF1FCE
:1017A00008B50BF097FC084809F0B8FD00230121AB
:1017B0004FF07E52054809F0A9FF04210448BDE816
:1017C00008400AF0B9BF00BF109EFF1F689EFF1FB0
:1017D000009FFF1F00B5244B1A7883B00121052319
:1017E00002B3002201910093114620480AF040F90B
:1017F0001F4B1A7802B305230122019200930022A5
:101800000A211A480AF034F91A4B1A7802BB052348
:10181000012101910093142114480AF0ABF903B09F
:101820005DF804FB01910093114610480AF0A2F9FB
:101830000F4B1A78002ADED1052301210191009374
:101840000A210A480AF096F90A4B1A78002ADED0D3
:1018500005230122019200930022142103480AF07B
:1018600007F903B05DF804FBD19EFF1F009FFF1F27
:101870002C9FFF1F2D9FFF1F2DE9F04FC54D2B788B
:10188000A3F10A02022A83B040F22281C24EA3F1E0
:101890001402022A3CD8DFF83083C04AD8F800E0AE
:1018A0001268BF499645D1F8009080F20E82C2EBD3
:1018B000090CBCF15A0F4FF00004BA4F40F31282EA
:1018C000D7F800A05B2052450CF1010100FB04F4A5
:1018D00094FBF1F404F11C0440F3E882002292FB33
:1018E000F1F11C31A14200F0158209B20023262239
:1018F000AD480AF0B3FE21B201232622AA480AF01D
:10190000ADFEA9480BF0D2F8D8F800202B783A6049
:10191000A3F11E02022A00F28B80A44FDFF8ACA2D2
:101920003968DAF80030DFF8A8929942D9F8002037
:1019300080F25A81D01A5A284FF00004DFF89482BE
:1019400040F35E81D8F800104FF05B0E8B420EFB27
:1019500004F400F1010E94FBFEF404F11C0400F306
:10196000B9829142A8BF1146C3EB010C5B2101FB78
:101970000CF191FBFEF11C31A14200F0548109B23F
:101980000023262288480AF069FE21B2012326227C
:1019900085480AF063FEDAF80030DFF83CA2D9F897
:1019A0000020DAF8001099424FF0010CA2EB03007E
:1019B000C0F244819142D4BFC3EB0104C3EB0204E3
:1019C0005A28DFF8189240F34081D9F800B000F1AE
:1019D000010E5B454FF05B0000FB04F494FBFEF44A
:1019E00004F11C0400F378825A45A8BF5A46D21A63
:1019F0005B2000FB02F090FBFEF01C30A04200F0E8
:101A0000398101B20023262267480AF027FE21B25D
:101A10000123262264480AF021FE63480BF046F8B1
:101A2000DAF800103A682B78C8F80020C9F80010DE
:101A3000A3F12802022A42D8DFF8A4815C4AD8F830
:101A400000E012685B499645D1F800C080F21A8127
:101A5000C2EB0C015A294FF00004574F40F31E818E
:101A600038684FF05B09824201F1010109FB04F47F
:101A700094FBF1F404F11C0400F316828445A8BF22
:101A80008446C2EB0C0C5B2000FB0CF090FBF1F1E8
:101A90001C31A14200F0158109B2002326224248E0
:101AA0000AF0DCFD21B2012326223F480AF0D6FDD0
:101AB0003D480AF0FBFFD8F800202B783A603C3B09
:101AC000012B40F23A810023337003B0BDE8F08F60
:101AD0003A4ADFF810811668D8F800E0384AB6456F
:101AE000126834DA911B5A294FF00004354F38DD63
:101AF00038684FF05B0C864201F101010CFB04F4E5
:101B000094FBF1F404F11C0400F3E8819042A8BFB7
:101B10001046861B5B2000FB06F090FBF1F11C31A8
:101B2000A14230D009B2002326221F481A4E0AF0E3
:101B300095FD21B2012326221B480AF08FFD1A4889
:101B40000AF0B4FFD8F800202B783A609FE6911B8A
:101B50009645D4BFC6EB0E04C6EB02045A29194FB2
:101B6000C6DCD7F800C05A20664500FB04F494FB9D
:101B7000F1F404F11C0440F3BC81002292FBF1F16A
:101B80001C31A142CED1044E3278002A40F0D380DD
:101B90007246DAE70C9EFF1F679DFF1F688AFF1FD2
:101BA000E48DFF1F549EFF1F009FFF1FC89DFF1F56
:101BB000FC8DFF1F5C8AFF1F809DFF1F309EFF1F53
:101BC000588AFF1FCC9EFF1F689DFF1FE88DFF1FD7
:101BD0003C8BFF1FD09DFF1FFC9EFF1F309FFF1FF0
:101BE000BC9DFF1FAC9EFF1FD01A9142D4BFC3EB18
:101BF0000104C3EB02045A28DFF824833FF7A2AEA6
:101C0000D8F800E05A21734501FB04F494FBF0F48A
:101C100004F11C0440F36481002191FBF0F11C31BC
:101C2000A1427FF4ACAE3478002C77D1DFF8F4A277
:101C3000DAF800109942A446BFF6BCAE5A284FF01D
:101C40000004DFF8E4923FF7C0AED9F800E04FF0AF
:101C50005A0B73450BFB04F494FBF0F404F11C04E1
:101C600040F319814FF0000B9BFBF0F01C30A042B9
:101C70007FF4C7AE3378002B56D1BCF1000F3FF490
:101C8000D1AECAE6C2EB0C01E645D4BFC2EB0E04EE
:101C9000C2EB0C045A299B4F3FF7E2AED7F80090F5
:101CA0005A204A4500FB04F494FBF1F404F11C04AF
:101CB00040F30781002292FBF1F11C31A1427FF435
:101CC000EBAE327872BB7246F8E6C2EB090CCE4539
:101CD000D4BFC2EB0E04C2EB0904BCF15A0F8A4F09
:101CE0003FF7EEAD39685A208A4200FB04F494FBBA
:101CF000FCF404F11C0400F3E2804945A8BF494606
:101D0000891A5A2000FB01F090FBFCF11C31A14222
:101D10007FF4EBAD32781AB97246F8E509B235E6D0
:101D200009B2E9E509B2BEE601B2012326227748ED
:101D30000AF094FC71E609B2FCE6262200248DE844
:101D4000140076231C217148714D724F09F0C2FEB8
:101D50001DE08242D4BFC3EB0201C3EB0001D31AE2
:101D60004FF05A0E73454FF05B00CABF41430EFB64
:101D700001F1013391FBF3F303F11C0101231C4436
:101D8000262209B261480AF069FC0C2C09D0E1B2A4
:101D9000614809F02BFB2B683A688342D9DD0021AA
:101DA000DDE7DFF888815D4C01200CF051F9D8F8AF
:101DB00000C023683A682968CCEB030E8B1A9E4555
:101DC000CCEB00005BDD03FB00000EF1010390FB98
:101DD000F3F3134499424EDC9A42D4BFC1EB0203A1
:101DE000C1EB0303521A5A2ACABF5B215A2101329E
:101DF00001FB03F393FBF2F202F11C0109B2012390
:101E0000262242480AF02AFC00200CF021F9D8F8DA
:101E100000E03A68296824688B1ACEEB04049C42DF
:101E2000CEEB000031DD03FB0000631C90FBF3F3FD
:101E30001344994221DC9A42D4BFC1EB0203C1EBA7
:101E40000303521A5A2ACABF5B215A21013201FBED
:101E500003F393FBF2F202F11C0109B201232622E3
:101E60002A480AF0FBFB29480AF020FE00233370C1
:101E700003B0BDE8F08F0023B4E70023E1E703FBE4
:101E800000F393FBFEF31344A4E703FB00F393FB7F
:101E9000F4F31344CDE77245D4BFC3EB0203C3EBA5
:101EA0000E030BFB03FBDFE69446EAE5D145D4BF06
:101EB000C2EB0902C2EB0A0200FB02F20FE5114677
:101EC0001EE7CC45D4BFC2EB0C02C2EB090200FBFB
:101ED00002F2F0E6194647E51A4688E5304618E66C
:101EE0007245D4BFC3EB020EC3EB0E0E01FB0EF125
:101EF00093E66245D4BFC6EB0202C6EB0C0200FBC0
:101F000002F23BE6809DFF1F549EFF1F009FFF1FB4
:101F1000F48DFF1F408CFF1F109EFF1F5C8CFF1F66
:101F2000D09DFF1FFC9EFF1F309FFF1F608AFF1F79
:101F300008B581B217480AF069F9022115480AF07C
:101F40005FF921225A2113480AF056F9124B114821
:101F500019880DF09FFB0F480DF04CFB0F4B1978C3
:101F600091B90C480AF052F901210A480AF048F9DF
:101F70003322742107480AF03FF901220849054835
:101F8000BDE808400DF022BB012102480AF03EF9ED
:101F9000EAE700BF009FFF1F589EFF1FDE9EFF1F46
:101FA0001435010010B5104C012120460AF02EF91D
:101FB000204601210AF024F92046342255210AF056
:101FC0001BF92046022209490DF000FB204605229C
:101FD00007490DF0FBFA20460DF00CFB2046BDE84A
:101FE00010400AF063BD00BF009FFF1F00350100D5
:101FF000043501002DE9F84F0C200AF09BFF0C205E
:102000000BF066FDDD4914200BF072FD0221032068
:102010000BF004FE022104200BF000FE022105203B
:102020000BF0FCFD022106200BF0F8FD01210A2037
:102030000BF0F4FD012109200BF0F0FD01210D2032
:102040000BF0ECFD012128200BF0E8FD012114200C
:102050000BF0E4FD02210B200BF0E0FD01210C2030
:102060000BF0DCFD00210C200BF0C4FD0020FEF77E
:1020700051FD172840F25C8204200BF0C1FD0028BE
:1020800000F050820020FEF745FD1F2800F08C82F2
:102090001F210020FEF732FD0C210E20FEF72EFD41
:1020A00001211020FEF72AFD02211220FEF726FD55
:1020B00000211420FEF722FD00211620FEF71EFD50
:1020C00002211820FEF71AFD01211A20FEF716FD45
:1020D00002211C20FEF712FD04211E20FEF70EFD3A
:1020E00014212020FEF70AFD01212620FEF706FD1F
:1020F00003212820FEF702FD04212C20FEF7FEFC20
:102100000F212E20FEF7FAFC00213020FEF7F6FC0E
:102110000C213220FEF7F2FC00213420FEF7EEFC09
:1021200000213620FEF7EAFC00213820FEF7E6FC0D
:1021300000213A20FEF7E2FC00213C20FEF7DEFC05
:1021400000213E20FEF7DAFC00214020FEF7D6FCFD
:1021500000214220FEF7D2FC1F214420FEF7CEFCD6
:1021600013214620FEF7CAFC0E214820FEF7C6FCCC
:1021700011214A20FEF7C2FC0A214C20FEF7BEFCCA
:1021800000214E20FEF7BAFC06215020FEF7B6FCD7
:1021900002215220FEF7B2FC0F215420FEF7AEFCC4
:1021A00000215620FEF7AAFC0220FEF7B3FC744B78
:1021B000744C18800420FEF7ADFC734BDFF84082AE
:1021C00018800620FEF7A6FC704BDFF838A21880B6
:1021D0000820FEF79FFC6E4B6E4E18800A20FEF71B
:1021E00099FC6D4B6D4D18800C20FEF793FC6C4BE9
:1021F00018800E20FEF78EFC6A4B18801020FEF728
:1022000089FC20801220FEF785FC674B1880142083
:10221000FEF780FC654B18801620FEF77BFC644BB4
:1022200018801820FEF776FC624B18801A20FEF703
:1022300071FC614B18801C20FEF76CFC5F4B188012
:102240001E20FEF767FC5E4B18802020FEF762FC24
:102250005C4B18802220FEF75DFC5B4B188024202D
:10226000FEF758FC594B18802620FEF753FC584BBC
:1022700081462820A3F80090FEF74CFC554B1880AF
:102280002A20FEF747FC544B07462C201F80FEF700
:1022900041FC524B18802E20FEF73CFC504B18801E
:1022A0003020FEF737FC4F4B18803220FEF732FC0F
:1022B0004D4B18803420FEF72DFCA8F80000362086
:1022C000FEF728FCA8F802003820FEF723FCA8F847
:1022D00004003A20FEF71EFCA8F806003C20FEF79A
:1022E00019FCA8F808003E20FEF714FCA8F80A0024
:1022F0004020FEF70FFCA8F80C004220FEF70AFC75
:102300003A4B80464420A3F80080FEF703FC384B8C
:10231000A0F1180246201A60FEF7FCFBA0F118039A
:102320004820CAF80030FEF7F5FBA0F118034A2058
:10233000CAF80430FEF7EEFBA0F118034C20CAF8EF
:102340000830FEF7E7FBA0F118034E20CAF80C3066
:10235000FEF7E0FB274B18805020FEF7DBFB264BF7
:1023600018805220FEF7D6FB244B18805420FEF72D
:10237000D1FB30805620FEF7CDFB45E0001B3746F1
:10238000169EFF1F589EFF1FE89EFF1FE49DFF1F24
:10239000C89EFF1FBA8CFF1F2C9EFF1FEE9DFF1FC4
:1023A000B49DFF1FA49DFF1F909EFF1F129EFF1F45
:1023B0005C9DFF1F209EFF1FCC9DFF1FC49DFF1F24
:1023C000B89DFF1FDA9EFF1F8E9DFF1F469EFF1FB9
:1023D000649EFF1FB29EFF1FF09EFF1F989EFF1F6F
:1023E000B89EFF1FA29DFF1FCA9EFF1FEA9EFF1FF0
:1023F000048BFF1FC29DFF1FB88CFF1F948AFF1F15
:10240000709DFF1F448CFF1FB34ADFF838E3B349C8
:10241000D2F800A0B24BB34ADEF800B0D1F800C049
:10242000D3F800E01168B04AB04B85F80090CCEBCF
:102430000B0CCEEB0A0E82FB0CBAD3F80090AC4B1F
:10244000E2444FEAEC7CCCEBAA1CDFF8FCA218803B
:10245000A84BCAF800C082FB0EAC1868A64BF44427
:102460004FEAEE7ECEEBAC1EDFF8E0C21B68CCF884
:1024700000E0C1EB090982FB09CEC01ACE44DFF8A7
:10248000D0C29E4B9E491B6809684FEAE979C9EBA7
:10249000AE1ECCF800E082FB00EC8444C017C1EB18
:1024A000030EC0EBAC10DFF8ACC282FB0E92CCF88E
:1024B000000072449348DFF8A0C24FEAEE7E5FFA54
:1024C00088F8CEEBA212026008F002098E4A8CF85E
:1024D000009008F0040C82F800C0DFF880E28B481E
:1024E0008B4A08F008088EF8008000681268C91A44
:1024F000121A9142A7EB03030EDD02FB03330131F5
:1025000093FBF1F30344834A834813605A2108F094
:10251000A9FF002855D1FEE702FB03F292FBF1F37D
:102520000344F0E706200BF06BFB00287FF4AAAD14
:102530001F210020FEF7E2FA4FF4AF610220FEF700
:10254000DDFA04204FF47A61FEF7D8FA0B200BF085
:1025500057FB002800F0B58040F628210620FEF742
:10256000CDFA40F6E4410820FEF7C8FA4FF4AF6117
:102570000A20FEF7C3FA40F6FC010C20FEF7BEFA73
:102580004FF496612220FEF7B9FA4FF41661242029
:10259000FEF7B4FA7D212A20FEF7B0FA0020FEF7FC
:1025A000B9FA1F287FF474AD04200BF029FB002832
:1025B0007FF4FAAD06200BF023FB00283FF468AD52
:1025C000F2E5564A564812680023012109F0BCF88A
:1025D000FEF7E2F90B200BF013FB524B011E0CBF70
:1025E000012200221A7002D111200BF017FBDFF834
:1025F0003C814D4F0023C8F800303B604FF001098B
:102600000F200BF025FD3B68DFF81CA103440E20D2
:102610003B600AF0C3FCD8F8003009F00101034424
:102620000D20C8F8003009F101090BF0E3FAFA2097
:102630000BF01CFBB9F1050FE2D1DAF80030D8F845
:102640000020318839483A4E002BB8BF0333002AA6
:10265000B8BF03329B103B609210364F02605A1A8B
:102660000D200B44002133603A600BF0C3FAFA20CE
:102670000BF0FCFA01210D200BF0BCFAFA200BF054
:10268000F5FA00210D200BF0B5FAFFF78BFC40F2B4
:10269000DC500BF0EBFA284B012604201E600BF0F7
:1026A000AFFA10B9254B28701E702378244A1846BB
:1026B0001370FEF7A5FA01210D20BDE8F84F0BF0CD
:1026C00099BA4FF496610620FEF718FA4FF4FA61B2
:1026D0000820FEF713FA49E7E48DFF1F309EFF1F25
:1026E000688AFF1FE88DFF1FC94216B23C8BFF1F8F
:1026F000F69DFF1F5C8AFF1FFC8DFF1F408CFF1F94
:10270000F48DFF1FD89DFF1F149EFF1F608AFF1FBF
:102710005C8CFF1F548CFF1F109EFF1F4C8AFF1FF5
:10272000689EFF1F189EFF1FBC9EFF1F6C9DFF1F12
:10273000349EFF1FE09DFF1FC49EFF1F959DFF1F3E
:102740002F9EFF1F588AFF1F9C9EFF1FB49EFF1FD6
:10275000A09EFF1F4C9EFF1FBA9DFF1FDE9EFF1F06
:1027600070B5194C82B03426002301252046019310
:10277000009640230B223F2109F07AF940230B22D7
:102780002046009601953F2109F0F4F9294620469C
:1027900009F03CFD2946204609F032FD20460F2273
:1027A000442109F029FD0922084920460CF00EFFBA
:1027B00020460CF01FFF064B20461D7002B0BDE8FE
:1027C00070400AF073B900BF009FFF1F0C35010075
:1027D000F89EFF1F70B5194C82B0342600230125E6
:1027E00020460193009640230B223F2109F040F937
:1027F00040230B222046009601953F2109F0BAF9AB
:102800002946204609F002FD2946204609F0F8FC39
:1028100020460F22512109F0EFFC052208492046ED
:102820000CF0D4FE20460CF0E5FE2846FEF70CF92D
:10283000204602B0BDE870400AF038B9009FFF1F83
:102840001835010070B5194C82B0342600230125DB
:1028500020460193009640230B223F2109F008F9FE
:1028600040230B222046009601953F2109F082F972
:102870002946204609F0CAFC2946204609F0C0FC3A
:1028800020460F22512109F0B7FC052208492046B5
:102890000CF09CFE20460CF0ADFE2846FEF710F929
:1028A000204602B0BDE870400AF000B9009FFF1F4B
:1028B0001835010070B5194C82B03426002301256B
:1028C00020460193009640230B223F2109F0D0F8C7
:1028D00040230B222046009601953F2109F04AF93A
:1028E0002946204609F092FC2946204609F088FC3A
:1028F00020460F22512109F07FFC0522084920467D
:102900000CF064FE20460CF075FE2846FEF7BAF87F
:10291000204602B0BDE870400AF0C8B8009FFF1F13
:102920001835010070B5194C82B0342600230125FA
:1029300020460193009640230B223F2109F098F88E
:1029400040230B222046009601953F2109F012F901
:102950002946204609F05AFC2946204609F050FC39
:1029600020460F22442109F047FC0922084920464D
:102970000CF02CFE20460CF03DFE2846FFF7D8FA5E
:10298000204602B0BDE870400AF090B8009FFF1FDB
:102990002035010008B581B2104809F037FC02214A
:1029A0000E4809F02DFC4F2121220C4809F024FC8F
:1029B0000B4B198849B903220A4908480CF006FE56
:1029C0000648BDE808400CF015BE04480CF062FE55
:1029D0000248BDE808400CF00DBE00BF009FFF1F7D
:1029E0005C9DFF1F2C35010070B5194C82B0342658
:1029F0000023012520460193009640230B223F210E
:102A000009F036F840230B222046009601953F211D
:102A100009F0B0F82946204609F0F8FB294620467F
:102A200009F0EEFB20460F22472109F0E5FB0822C2
:102A3000084920460CF0CAFD20460CF0DBFD284674
:102A4000FFF7A8FF204602B0BDE870400AF02EB89C
:102A5000009FFF1F3035010010B581B2124C1348A2
:102A600009F0D4FB0221114809F0CAFB2388212276
:102A70006BB94F210D4809F0BFFB03220C490B48ED
:102A80000CF0A4FD0948BDE810400CF0B3BD5A217C
:102A9000064809F0B1FB218804480CF0FBFD03480F
:102AA000BDE810400CF0A6BDB89DFF1F009FFF1FA2
:102AB0003C35010070B5194C82B034260023012545
:102AC00020460193009640230B223F2108F0D0FFBF
:102AD00040230B222046009601953F2109F04AF839
:102AE0002946204609F092FB2946204609F088FB3A
:102AF00020460F22512109F07FFB0522084920467C
:102B00000CF064FD20460CF075FD2846FFF7A4FF8D
:102B1000204602B0BDE8704009F0C8BF009FFF1F0B
:102B20001835010010B581B21748184C09F06EFB3A
:102B30000221154809F064FB21224C21124809F0BA
:102B40005BFB23884BB9032211490F480CF03EFD73
:102B50000D48BDE810400CF04DBD02220D490A4859
:102B60000CF034FD08480CF045FD21226521064893
:102B700009F042FB218804480CF08CFD0248BDE8B6
:102B800010400CF037BD00BF009FFF1FCC9DFF1F02
:102B90003C3501004035010070B5194C82B0342637
:102BA0000023012520460193009640230B223F215C
:102BB00008F05EFF40230B222046009601953F213E
:102BC00008F0D8FF2946204609F020FB2946204678
:102BD00009F016FB20460F22442109F00DFB0922C3
:102BE000084920460CF0F2FC20460CF003FD284674
:102BF000FFF798FF204602B0BDE8704009F056BFCD
:102C0000009FFF1F4435010010B581B2124C1348DC
:102C100009F0FCFA0221114809F0F2FA2388212276
:102C20006BB94F210D4809F0E7FA03220C490B4814
:102C30000CF0CCFC0948BDE810400CF0DBBC5A217C
:102C4000064809F0D9FA218804480CF023FD03480E
:102C5000BDE810400CF0CEBCA29DFF1F009FFF1FDF
:102C60003C35010070B5194C82B034260023012593
:102C700020460193009640230B223F2108F0F8FEE6
:102C800040230B222046009601953F2108F072FF59
:102C90002946204609F0BAFA2946204609F0B0FA3A
:102CA00020460F22482109F0A7FA082208492046A9
:102CB0000CF08CFC20460CF09DFC2846FFF7A4FF8E
:102CC000204602B0BDE8704009F0F0BE009FFF1F33
:102CD0005035010010B50C4681B2194809F096FA3A
:102CE0000221174809F08CFA21225021144809F0DA
:102CF00083FA002C4FF0010214DB124910480CF04B
:102D000065FC0F480CF076FC5D2121220C4809F08F
:102D100073FA21460A480CF0BDFC0948BDE8104092
:102D20000CF068BC084906480CF050FC04480CF054
:102D300061FC5D212122024809F05EFA6142E9E767
:102D4000009FFF1F5C350100603501000CB42DE9C8
:102D5000F04184B00AAC0646294814F8045B884662
:102D600009F002FD0121264809F04AFA0121244810
:102D700009F04CFA00221146214809F03DFA30468C
:102D80000EF05EFE314602461D480CF01FFC1C484A
:102D90000CF030FC092201238DE80C0000217F2378
:102DA000174808F097FE0394EDB16F1EFFB201378C
:102DB00004EB87070C25043454F8046C1048039482
:102DC0002AB2002109F018FA30460EF039FE3146D9
:102DD00002460B480CF0FAFB09480CF00BFC0935D5
:102DE000BC42ADB2E7D140460121FDF7F7FD0448F2
:102DF00009F05CFE04B0BDE8F04102B0704700BFCE
:102E0000009FFF1F30B52B4D0FCD8DB006AC0FC40A
:102E100095E8030044F8040B232021800AF0BEF853
:102E200040F6B833984212DC234B40F6F50219887D
:102E30009B78ADF8251090428DF827300EDC1F4BA3
:102E40001A889B78ADF829208DF82B301EE01C4B9A
:102E50001A889B78ADF825208DF82730194A00EBA9
:102E6000400000EB001382FB0320DB17C3EB602064
:102E70000DF074FD14490DF0C5FD0DF1290301227B
:102E800003210AF03DFA56238DF82C300F4B1048E1
:102E90001978104D104C114A114B04900192009377
:102EA00006A8039502940F4B0622FFF74FFF0DB0C3
:102EB00030BD00BFB0350100643501006835010048
:102EC000AC350100976A3E2BCDCCCC3D3289FF1F3B
:102ED0007C35010088350100943501009C350100E6
:102EE000A43501007035010030B50A4B0A4D197840
:102EF0000A4C0B480B4A0C4B87B00290019200938E
:102F000004950394094B0A480622FFF71FFF07B0F8
:102F100030BD00BF948DFF1FE4350100F035010086
:102F2000FC3501000836010014360100C8350100E7
:102F3000D435010010B586B0084C094809490A4A41
:102F40000A4B03900291019200930494084B0948A4
:102F50000622FF21FFF7FAFE06B010BD5035010032
:102F60003C36010048360100303501005036010082
:102F7000203601002C36010010B586B0084C0948F7
:102F800009490A4A0A4B0390029101920093049462
:102F9000084B09480622FF21FFF7D8FE06B010BDF6
:102FA00074360100803601008C3601009436010031
:102FB000443501005C3601006836010000B585B07B
:102FC00008480949094A0A4B03900291019200936B
:102FD0000848094B0522FF21FFF7B8FE05B05DF850
:102FE00004FB00BFA8360100B4360100BC36010066
:102FF000C43601008C360100A036010010B581B244
:103000002048214C09F002F902211E4809F0F8F885
:10301000212250211B4809F0EFF823880B2B4FF099
:10302000010218DC194917480CF0D0FA15480CF0C9
:10303000E1FA21225D21134809F0DEF821881148C8
:103040000C390029B8BF49420CF024FB0D48BDE8FB
:1030500010400CF0CFBA0E490A480CF0B7FA0948F4
:103060000CF0C8FA21225D21064809F0C5F8218834
:1030700004480C390CF00EFB0248BDE810400CF07F
:10308000B9BA00BF009FFF1FA49DFF1F603501005C
:103090005C35010070B5194C82B03426002301253F
:1030A00020460193009640230B223F2108F0E0FCCC
:1030B00040230B222046009601953F2108F05AFD3F
:1030C0002946204609F0A2F82946204609F098F83A
:1030D00020460F22442109F08FF809220849204692
:1030E0000CF074FA20460CF085FA2846FFF786FFAC
:1030F000204602B0BDE8704009F0D8BC009FFF1F19
:103100007035010010B581B22048214C09F07EF8DD
:1031100002211E4809F074F8212250211B4809F0B1
:103120006BF82388022B4FF0010218DC194917486D
:103130000CF04CFA15480CF05DFA21225D21134881
:1031400009F05AF82188114803390029B8BF4942CB
:103150000CF0A0FA0D48BDE810400CF04BBA0E4937
:103160000A480CF033FA09480CF044FA21225D2198
:10317000064809F041F82188044803390CF08AFA1E
:103180000248BDE810400CF035BA00BF009FFF1F99
:10319000B29EFF1F603501005C35010070B5194C0F
:1031A00082B0342600230125204601930096402357
:1031B0000B223F2108F05CFC40230B2220460096A6
:1031C00001953F2108F0D6FC2946204609F01EF85B
:1031D0002946204609F014F820460F224D2109F017
:1031E0000BF80622084920460CF0F0F920460CF0B6
:1031F00001FA2846FFF786FF204602B0BDE870407E
:1032000009F054BC009FFF1FA435010000B5324BEC
:103210001B78013B85B0052B0AD8DFE803F00C21B1
:10322000364B54032D492E4B5A20012208701A7038
:1032300005B05DF804FB01232A4A194618461370AD
:10324000FDF7CCFB284809F031FC284A284B1268CE
:103250000192019A1A60FFF71DFF05B05DF804FBAB
:103260000123244A194602201370FDF7B7FB1E48BC
:1032700009F01CFC1D4A1E4B12680292029A1A6049
:10328000FFF78CFF05B05DF804FB01231A4A1946CD
:1032900003201370FDF7A2FB134809F007FC134A43
:1032A000134B12680392039A1A60FFF73BFB05B0B9
:1032B0005DF804FB09490A4B0A20012208701A70C4
:1032C00005B05DF804FB0549054B5020012208704C
:1032D0001A7005B05DF804FB3289FF1F0C9EFF1FBA
:1032E000588CFF1FA69EFF1F009FFF1F3C9FFF1FC4
:1032F000389EFF1FAC9DFF1FED9DFF1F08B581B2DB
:103300000D4808F083FF02210B4808F079FF2122C5
:103310004F21094808F070FF084B1B884BB908493A
:10332000032205480CF052F90348BDE808400CF0B0
:1033300061B902220349F4E7009FFF1F129EFF1F9D
:103340003C350100CC36010070B5194C82B03426F2
:103350000023012520460193009640230B223F21A4
:1033600008F086FB40230B222046009601953F2162
:1033700008F000FC2946204608F048FF2946204670
:1033800008F03EFF20460F22442108F035FF0922B5
:10339000084920460CF01AF920460CF02BF9284673
:1033A000FFF7ACFF204602B0BDE8704009F07EBBDD
:1033B000009FFF1F5036010008B581B20D4808F08C
:1033C00025FF02210B4808F01BFF21224F2109484D
:1033D00008F012FF084B1B88032243B10749054838
:1033E0000CF0F4F80348BDE808400CF003B90449B8
:1033F000F5E700BF009FFF1FF69DFF1FD4360100B9
:10340000D036010070B5194C82B034260023012556
:1034100020460193009640230B223F2108F028FB11
:1034200040230B222046009601953F2108F0A2FB85
:103430002946204608F0EAFE2946204608F0E0FE2C
:1034400020460F22442108F0D7FE092208492046D1
:103450000CF0BCF820460CF0CDF82846FFF7ACFF86
:10346000204602B0BDE8704009F020BB009FFF1F5E
:10347000A836010000B53A4B1B78013B87B0042BFE
:1034800016D8DFE803F0182D425703000123354A10
:10349000194605201370FDF7A1FA334809F006FB21
:1034A000324A334B12680592059A1A60FFF7AAFF59
:1034B00007B05DF804FB01232E4A19461846137025
:1034C000FDF78CFA284809F0F1FA284A284B1268CF
:1034D0000192019A1A60FFF7EDFA07B05DF804FB5C
:1034E0000123254A194602201370FDF777FA1E487A
:1034F00009F0DCFA1D4A1E4B12680292029A1A6009
:10350000FFF768F907B05DF804FB01231B4A194671
:1035100003201370FDF762FA134809F0C7FA134A43
:10352000134B12680392039A1A60FFF7C3F907B0AE
:103530005DF804FB0123124A194604201370FDF7BD
:103540004DFA094809F0B2FA084A094B1268049288
:10355000049A1A60FFF776F907B05DF804FB00BF24
:10356000488AFF1FDD9EFF1F009FFF1F3C9FFF1F1C
:10357000389EFF1F2E9EFF1F009EFF1FDC9DFF1F1A
:10358000DC9EFF1F08B581B20D4808F03FFE022106
:103590000B4808F035FE21224F21094808F02CFE87
:1035A000084B1B88032243B9074905480CF00EF865
:1035B0000348BDE808400CF01DB80449F5E700BF1A
:1035C000009FFF1FC29DFF1FDC360100D83601009F
:1035D00070B5194C82B03426002301252046019392
:1035E000009640230B223F2108F042FA40230B2291
:1035F0002046009601953F2108F0BCFA2946204656
:1036000008F004FE2946204608F0FAFD20460F2265
:10361000442108F0F1FD0922084920460BF0D6FFAD
:1036200020460BF0E7FF2846FFF7ACFF204602B02C
:10363000BDE8704009F03ABA009FFF1FE036010074
:1036400000B5444B1B78013B87B0052B16D8DFE84B
:1036500003F0182D42576C0301233F4A19460620F8
:103660001370FDF7BBF93D4809F020FA3C4A3D4B89
:1036700012680592059A1A60FFF7AAFF07B05DF875
:1036800004FB0123384A194618461370FDF7A6F9C2
:10369000324809F00BFA324A324B12680092009A13
:1036A0001A60FFF75DF807B05DF804FB01232F4AAD
:1036B000194602201370FDF791F9284809F0F6F930
:1036C000274A284B12680192019A1A60FFF748F8BE
:1036D00007B05DF804FB254B0222012103201A707C
:1036E000FDF77CF91D4809F0E1F91D4A1D4B1268F0
:1036F0000292029A1A60FFF733F807B05DF804FBF4
:103700001A4B0322012104201A70FDF767F91348B0
:1037100009F0CCF9124A134B12680392039A1A600B
:10372000FFF71EF807B05DF804FB104B04220121DF
:1037300005201A70FDF752F9084809F0B7F9084A50
:10374000084B12680492049A1A60FFF709F807B050
:103750005DF804FB948DFF1F509EFF1F009FFF1F0D
:103760003C9FFF1F389EFF1F3D9EFF1FE09EFF1FD7
:1037700008B581B2154808F049FD0221134808F048
:103780003FFD4F212122114808F036FD104B1988CA
:1037900049B9104903220D480BF018FF0B48BDE84A
:1037A00008400BF027BF09480BF074FF07480BF0E7
:1037B00021FF28226921054808F01EFD0121034848
:1037C00008F01EFD02220449E5E700BF009FFF1F2D
:1037D000B89EFF1F3C350100EC36010070B5194C56
:1037E00082B0342600230125204601930096402311
:1037F0000B223F2108F03CF940230B222046009683
:1038000001953F2108F0B6F92946204608F0FEFC54
:103810002946204608F0F4FC20460F22452108F0F6
:10382000EBFC0922084920460BF0D0FE20460BF0A5
:10383000E1FE2846FFF79CFF204602B0BDE870403D
:1038400009F034B9009FFF1F3C36010008B581B272
:10385000154808F0DBFC0221134808F0D1FC4F2189
:103860002122114808F0C8FC104B198849B91049A9
:1038700003220D480BF0AAFE0B48BDE808400BF0F0
:10388000B9BE09480BF006FF07480BF0B3FE28222B
:103890006921054808F0B0FC0121034808F0B0FC9C
:1038A00002220449E5E700BF009FFF1FDA9EFF1FC9
:1038B0003C350100EC36010070B5194C82B034265D
:1038C0000023012520460193009640230B223F212F
:1038D00008F0CEF840230B222046009601953F21A8
:1038E00008F048F92946204608F090FC2946204671
:1038F00008F086FC20460F22472108F07DFC0822B4
:10390000084920460BF062FE20460BF073FE284665
:10391000FFF79CFF204602B0BDE8704009F0C6B832
:10392000009FFF1F8036010030B5544883B008F077
:103930001BFF0121514808F063FC01214F4808F0AA
:1039400065FC022219214D4808F056FC0B224C4917
:103950004A480BF03BFE49480BF04CFE1422002174
:10396000464808F049FC0322464944480BF02EFE25
:10397000424801240BF03EFE11228DE8140078230A
:1039800019213E4808F0A6F8132519231946009579
:1039900012223A48019408F09DF8782319460095C0
:1039A00012223648019408F095F81D228DE8140083
:1039B00078231921314808F08DF81C251923194660
:1039C00000951B222D48019408F084F878231946AD
:1039D00000951B222948019408F07CF8232200213D
:1039E000264808F009FC0322274924480BF0EEFD85
:1039F00022480BF0FFFD28251923194624221F48D1
:103A00000194009508F066F8782319462422019461
:103A100000951A4808F05EF81C4A1D4B11681B6897
:103A20001C4A5B1A5C2B12881DDC511A5C2202FBBB
:103A300001F292FBF3F31B33174A10481360012481
:103A40001BB21A2219468DE81400142208F042F81D
:103A5000124B20461C70FCF7D7FF084803B0BDE8A6
:103A6000304009F023B8521A02EB4202C2EB421274
:103A7000234492FBF3F31B33DEE700BF009FFF1FDD
:103A8000F0360100FC36010000370100F48DFF1F05
:103A9000408CFF1FF09EFF1F609DFF1F889EFF1F31
:103AA000F0B58548854E864D83B008F05DFE012156
:103AB000814808F0A5FB01217F4808F0A7FB0222FE
:103AC00019217D4808F098FB0A227E497A480BF0BC
:103AD0007DFD79480BF08EFD14220021764808F018
:103AE0008BFB0322784974480BF070FD7248012467
:103AF0000BF080FD11228DE81400782319216E4807
:103B000007F0E8FF132719231946009712226A4885
:103B1000019407F0DFFF78231946009712226648C8
:103B2000019407F0D7FF1D228DE814007823192196
:103B3000614807F0CFFF1C271923194600971B2265
:103B40005D48019407F0C6FF7823194600971B22B1
:103B50005948019407F0BEFF23220021564808F07F
:103B60004BFB0322594954480BF030FD52480BF0EF
:103B700041FD282719231946009724224E48019415
:103B800007F0A8FF78231946009724224A48019499
:103B900007F0A0FF32220021474808F02DFB032246
:103BA0004B4945480BF012FD43480BF023FD2F22F3
:103BB0008DE81400782319213F4807F08BFF312747
:103BC00019231946009730223B48019407F082FFE1
:103BD00078231946009730223748019407F07AFF7E
:103BE0003C228DE8140078231921334807F072FF36
:103BF0003B27192319463A222F480194009707F0D2
:103C000069FF782319463A22019400972A4807F061
:103C100061FF31682B682F4A5B1A5C2B128839DDF3
:103C2000521A02EB4202C2EB4212234492FBF3F31C
:103C30001B33294A2048136001241BB21A2219465B
:103C40008DE81400142207F045FF31682B682348E3
:103C5000234A04705B1A5C2B128823DC511A5C2205
:103C600002FB01F292FBF3F31B331E4A124813606E
:103C700001241BB2392219468DE81400322207F0C4
:103C800029FF2046FCF7C0FE0B4803B0BDE8F0401A
:103C900008F00CBF511A5C2202FB01F292FBF3F315
:103CA0001B33C6E7521A02EB4202C2EB4212234414
:103CB00092FBF3F31B33D8E7009FFF1FE88DFF1F34
:103CC0003C8BFF1F04370100FC3601000037010068
:103CD000103701002C9EFF1F609DFF1F889EFF1F55
:103CE000B49DFF1FA89EFF1FF0B58548854E864DE9
:103CF00083B008F039FD0121814808F081FA0121E3
:103D00007F4808F083FA022219217D4808F074FAEE
:103D10000A227E497A480BF059FC79480BF06AFC7C
:103D200014220021764808F067FA03227849744883
:103D30000BF04CFC724801240BF05CFC11228DE866
:103D40001400782319216E4807F0C4FE13271923A5
:103D50001946009712226A48019407F0BBFE7823A7
:103D60001946009712226648019407F0B3FE1D22FF
:103D70008DE8140078231921614807F0ABFE1C2759
:103D80001923194600971B225D48019407F0A2FEF3
:103D90007823194600971B225948019407F09AFE90
:103DA00023220021564808F027FA03225949544893
:103DB0000BF00CFC52480BF01DFC28271923194668
:103DC000009724224E48019407F084FE7823194678
:103DD000009724224A48019407F07CFE32220021F9
:103DE000474808F009FA03224B4945480BF0EEFB1F
:103DF00043480BF0FFFB2F228DE814007823192194
:103E00003F4807F067FE31271923194600973022F3
:103E10003B48019407F05EFE782319460097302254
:103E20003748019407F056FE3C228DE814007823B1
:103E30001921334807F04EFE3B27192319463A2231
:103E40002F480194009707F045FE782319463A223F
:103E5000019400972A4807F03DFE31682B682F4AED
:103E60005B1A5C2B128839DD521A02EB4202C2EB5C
:103E70004212234492FBF3F31B33294A2048136078
:103E800001241BB21A2219468DE81400142207F0EF
:103E900021FE31682B682348234A04705B1A5C2B8F
:103EA000128823DC511A5C2202FB01F292FBF3F32D
:103EB0001B331E4A1248136001241BB239221946D3
:103EC0008DE81400322207F005FE2046FCF79CFD29
:103ED0000B4803B0BDE8F04008F0E8BD511A5C2281
:103EE00002FB01F292FBF3F31B33C6E7521A02EB1B
:103EF0004202C2EB4212234492FBF3F31B33D8E796
:103F0000009FFF1F688AFF1FE48DFF1F1437010009
:103F1000FC3601000037010010370100E49DFF1F4F
:103F2000609DFF1F889EFF1FC89EFF1FA89EFF1F4A
:103F3000F0B58548854E864D83B008F015FC01210B
:103F4000814808F05DF901217F4808F05FF90222FD
:103F500019217D4808F050F910227E497A480BF06B
:103F600035FB79480BF046FB14220021764808F017
:103F700043F90322784974480BF028FB7248012466
:103F80000BF038FB11228DE81400782319216E48BC
:103F900007F0A0FD132719231946009712226A483B
:103FA000019407F097FD782319460097122266487E
:103FB000019407F08FFD1D228DE81400782319214C
:103FC000614807F087FD1C271923194600971B221B
:103FD0005D48019407F07EFD7823194600971B2267
:103FE0005948019407F076FD23220021564808F035
:103FF00003F90322594954480BF0E8FA52480BF0F0
:10400000F9FA282719231946009724224E480194CB
:1040100007F060FD78231946009724224A4801944E
:1040200007F058FD32220021474808F0E5F8032246
:104030004B4945480BF0CAFA43480BF0DBFA2F22F4
:104040008DE81400782319213F4807F043FD3127FC
:1040500019231946009730223B48019407F03AFD96
:1040600078231946009730223748019407F032FD33
:104070003C228DE8140078231921334807F02AFDEB
:104080003B27192319463A222F480194009707F03D
:1040900021FD782319463A22019400972A4807F017
:1040A00019FD31682B682F4A5B1A5C2B128839DDA9
:1040B000521A02EB4202C2EB4212234492FBF3F388
:1040C0001B33294A2048136001241BB21A221946C7
:1040D0008DE81400142207F0FDFC31682B6823489A
:1040E000234A04705B1A5C2B128823DC511A5C2271
:1040F00002FB01F292FBF3F31B331E4A12481360DA
:1041000001241BB2392219468DE81400322207F02F
:10411000E1FC2046FCF778FC0B4803B0BDE8F0401A
:1041200008F0C4BC511A5C2202FB01F292FBF3F3CB
:104130001B33C6E7521A02EB4202C2EB421223447F
:1041400092FBF3F31B33D8E7009FFF1FFC8DFF1F8B
:104150005C8AFF1F20370100FC3601000037010098
:10416000103701008E9DFF1F609DFF1F889EFF1F5F
:10417000469EFF1FA89EFF1FF0B58548854E864DC1
:1041800083B008F0F1FA0121814808F039F80121E3
:104190007F4808F03BF8022219217D4808F02CF8EE
:1041A00006227E497A480BF011FA79480BF022FA80
:1041B00014220021764808F01FF803227849744839
:1041C0000BF004FA724801240BF014FA11228DE866
:1041D0001400782319216E4807F07CFC132719235B
:1041E0001946009712226A48019407F073FC78235D
:1041F0001946009712226648019407F06BFC1D22B5
:104200008DE8140078231921614807F063FC1C270E
:104210001923194600971B225D48019407F05AFCA8
:104220007823194600971B225948019407F052FC45
:1042300023220021564807F0DFFF03225949544842
:104240000BF0C4F952480BF0D5F928271923194669
:10425000009724224E48019407F03CFC782319462D
:10426000009724224A48019407F034FC32220021AE
:10427000474807F0C1FF03224B4945480BF0A6F918
:1042800043480BF0B7F92F228DE814007823192149
:104290003F4807F01FFC31271923194600973022A9
:1042A0003B48019407F016FC78231946009730220A
:1042B0003748019407F00EFC3C228DE81400782367
:1042C0001921334807F006FC3B27192319463A22E7
:1042D0002F480194009707F0FDFB782319463A22F6
:1042E000019400972A4807F0F5FB31682B682F4AA4
:1042F0005B1A5C2B128839DD521A02EB4202C2EBC8
:104300004212234492FBF3F31B33294A20481360E3
:1043100001241BB21A2219468DE81400142207F05A
:10432000D9FB31682B682348234A04705B1A5C2B45
:10433000128823DC511A5C2202FB01F292FBF3F398
:104340001B331E4A1248136001241BB2392219463E
:104350008DE81400322207F0BDFB2046FCF754FB29
:104360000B4803B0BDE8F04008F0A0BB511A5C2236
:1043700002FB01F292FBF3F31B33C6E7521A02EB86
:104380004202C2EB4212234492FBF3F31B33D8E701
:10439000009FFF1F309EFF1F588AFF1F3437010008
:1043A000FC3601000037010010370100169EFF1F88
:1043B000609DFF1F889EFF1FE89EFF1FA89EFF1F96
:1043C00010B581B219481A4C07F020FF0221174896
:1043D00007F016FF4F212122144807F00DFF218816
:1043E0000B2910D90C2917D0012212490F480BF0C4
:1043F000EDF821880D480C390BF04CF90B48BDE85D
:1044000010400BF0F7B80C3908480BF043F9074897
:10441000BDE810400BF0EEB80322074903480BF04B
:10442000D5F80248BDE810400BF0E4B8009FFF1F2C
:10443000CA9EFF1F5C3501003C37010070B5194C66
:1044400082B03426002301252046019300964023A4
:104450000B223F2107F00CFB40230B222046009645
:1044600001953F2107F086FB2946204607F0CEFE46
:104470002946204607F0C4FE20460F22442107F0BB
:10448000BBFE0922084920460BF0A0F820460BF09D
:10449000B1F82846FFF794FF204602B0BDE870400F
:1044A00008F004BB009FFF1F7436010008B581B2FD
:1044B0000F4807F0ABFE02210D4807F0A1FE2122B4
:1044C0004F210B4807F098FE0A4B1A88012A0CD09E
:1044D000022A0EBF08490949032205480BF076F865
:1044E0000348BDE808400BF085B802220449F4E710
:1044F000009FFF1F209EFF1F403701003C35010039
:10450000CC36010070B5194C82B034260023012549
:1045100020460193009640230B223F2107F0A8FA82
:1045200040230B222046009601953F2107F022FBF5
:104530002946204607F06AFE2946204607F060FE1D
:1045400020460F22472107F057FE0822084920463F
:104550000BF03CF820460BF04DF82846FFF7A6FF7D
:10456000204602B0BDE8704008F0A0BA009FFF1FCF
:104570005C36010008B581B2224807F047FE0221EF
:10458000204807F03DFE21224F211E4807F034FE4F
:104590001D4B1B88042B33D8DFE803F0121A222AA4
:1045A000030021225321174807F026FE1749022253
:1045B00014480BF00BF81348BDE808400BF01AB88C
:1045C00021224F210F4807F017FE03221049EFE781
:1045D000212253210B4807F00FFE02220D49E7E785
:1045E00021225321074807F007FE02220A49DFE78C
:1045F00021225321034807F0FFFD02220749D7E794
:1046000008BD00BF009FFF1FC49DFF1F5037010062
:104610003C35010044370100483701004C370100A8
:1046200070B5194C82B03426002301252046019331
:10463000009640230B223F2107F01AFA40230B2259
:104640002046009601953F2107F094FA294620461E
:1046500007F0DCFD2946204607F0D2FD20460F2258
:10466000442107F0C9FD0922084920460AF0AEFF9F
:1046700020460AF0BFFF2846FFF77CFF204602B025
:10468000BDE8704008F012BA009FFF1F9436010089
:1046900000B53E4B1B78013B87B0052B16D8DFE8F1
:1046A00003F0182D425760030123394A19460620AA
:1046B0001370FCF793F9374808F0F8F9364A374B8E
:1046C00012680592059A1A60FFF7B8FE07B05DF808
:1046D00004FB0123324A194618461370FCF77EF991
:1046E0002C4808F0E3F92C4A2C4B12680192019AED
:1046F0001A60FFF707FF07B05DF804FB0123294AA2
:10470000194602201370FCF769F9224808F0CEF927
:10471000214A224B12680292029A1A60FEF73CFA72
:1047200007B05DF804FB01231F4A194603201370EC
:10473000FCF754F9174808F0B9F9174A174B1268F3
:104740000392039A1A60FFF76BFF07B05DF804FB52
:104750001649174B6E20012208701A7007B05DF8D9
:1047600004FB0123134A194605201370FCF736F9A0
:10477000084808F09BF9084A084B12680492049A0A
:104780001A60FFF799F807B05DF804FB548AFF1F21
:10479000969DFF1F009FFF1F3C9FFF1F389EFF1F1E
:1047A000449EFF1F589DFF1F649DFF1F0C9EFF1F0F
:1047B000588CFF1FC19DFF1F10B5334C334807F0C5
:1047C000D3FF237803BB01213048314C07F01EFD95
:1047D00006212E4807F014FD2388092B4ED9632BA0
:1047E0004FF00A0294BF1F211146284807F004FD2C
:1047F000218826480AF04EFF24480AF0FBFE234891
:10480000BDE8104008F052B9FCF7E4FF2378012B13
:10481000D9D9022B4FF001011C4817D007F0F6FC44
:1048200006211A4807F0ECFC0A221146174807F047
:10483000E3FC0322174915480AF0C8FE13480AF0A2
:10484000D9FE1248BDE8104008F030B907F0DEFC90
:1048500006210E4807F0D4FC0A2211460B4807F047
:10486000CBFC03220C4909480AF0B0FE07480AF0C5
:10487000C1FE0648BDE8104008F018B90A223021F0
:10488000024807F0B9FCB3E7669DFF1F009FFF1FBA
:10489000649EFF1F583701005437010008B581B2EC
:1048A000394807F0B3FC0221374807F0A9FC374B21
:1048B0001B884BB1013B092B65D8DFE803F01C24B2
:1048C0002C343C444C545C1421224F212E4807F0D8
:1048D00093FC2F4903222C480AF078FE2A48BDE8B1
:1048E00008400AF087BE21225321274807F084FCA4
:1048F00002222849EFE721225321234807F07CFCBC
:1049000002222549E7E7212253211F4807F074FCC2
:1049100002222249DFE7212253211B4807F06CFCC9
:1049200002221F49D7E721225321174807F064FCD0
:1049300002221C49CFE721224F21134807F05CFCDB
:1049400003221949C7E721224F210F4807F054FCE1
:1049500003221649BFE721224F210B4807F04CFCE8
:1049600003221349B7E721224F21074807F044FCEF
:1049700003221049AFE721225321034807F03CFCF2
:1049800002220D49A7E708BD009FFF1F909EFF1F51
:104990003C35010078370100443701005C370100E5
:1049A0006037010064370100683701006C3701008F
:1049B00070370100743701004C37010070B5194C95
:1049C00082B034260023012520460193009640231F
:1049D0000B223F2107F04CF840230B222046009683
:1049E00001953F2107F0C6F82946204607F00EFC46
:1049F0002946204607F004FC20460F22442107F0F8
:104A0000FBFB0922084920460AF0E0FD20460AF097
:104A1000F1FD2846FFF742FF204602B0BDE8704096
:104A200008F044B8009FFF1F2036010008B581B28E
:104A3000414807F0EBFB02213F4807F0E1FB3F4B09
:104A40001B880C2B77D8DFE803F0161E262E363E87
:104A5000464E565E666E070021225321364807F007
:104A6000CBFB3749022234480AF0B0FD3248BDE89A
:104A700008400AF0BFBD212253212F4807F0BCFB9C
:104A800002223049EFE7212253212B4807F0B4FBE3
:104A900002222D49E7E721225321274807F0ACFBEA
:104AA00002222A49DFE721225321234807F0A4FBF1
:104AB00002222749D7E721224F211F4807F09CFBFC
:104AC00003222449CFE7212253211B4807F094FBFE
:104AD00002222149C7E721225321174807F08CFB06
:104AE00002221E49BFE721225321134807F084FB0D
:104AF00002221B49B7E7212253210F4807F07CFB14
:104B000002221849AFE7212253210B4807F074FB1A
:104B100002221549A7E721225321074807F06CFB21
:104B2000022212499FE721225321034807F064FB28
:104B300002220F4997E708BD009FFF1F989EFF1FA5
:104B4000AC3701007C370100803701008437010059
:104B5000883701008C37010090370100943701003D
:104B6000983701009C370100A0370100A4370100ED
:104B7000A837010070B5194C82B0342600230125F6
:104B800020460193009640230B223F2106F070FF40
:104B900040230B222046009601953F2106F0EAFFB4
:104BA0002946204607F032FB2946204607F028FB1D
:104BB00020460F22502107F01FFB052208492046FE
:104BC0000AF004FD20460AF015FD2846FFF72EFFE7
:104BD000204602B0BDE8704007F068BF009FFF1F8D
:104BE0004836010000B5444B1B78013B87B0052BCC
:104BF00016D8DFE803F0182D42576C0301233F4A13
:104C0000194606201370FBF7E9FE3D4807F04EFFFA
:104C10003C4A3D4B12680592059A1A60FEF722F84D
:104C200007B05DF804FB0123384A19461846137093
:104C3000FBF7D4FE324807F039FF324A324B126894
:104C40000092009A1A60FFF7B9FE07B05DF804FB06
:104C500001232F4A194602201370FBF7BFFE284894
:104C600007F024FF274A284B12680192019A1A6024
:104C7000FEF76AFB07B05DF804FB0123254A1946DD
:104C800003201370FBF7AAFE1D4807F00FFF1D4A13
:104C90001D4B12680292029A1A60FDF7A5FE07B03A
:104CA0005DF804FB01231C4A194604201370FBF72E
:104CB00095FE134807F0FAFE124A134B126803924E
:104CC000039A1A60FFF756FF07B05DF804FB012353
:104CD000124A194605201370FBF780FE084807F0BA
:104CE000E5FE084A084B12680492049A1A60FEF71F
:104CF00075FD07B05DF804FB648AFF1FEC9DFF1F84
:104D0000009FFF1F3C9FFF1F389EFF1F5A9DFF1FE4
:104D1000D09EFF1F8C9DFF1F2B9FFF1FB69DFF1F67
:104D20002DE9F0430320ADF5257D08F069FFB0FAC9
:104D300080F4042008F064FF002814BF0021022141
:104D4000640905200C4408F05BFF002814BF002113
:104D5000042106200C4408F053FF9E4D9E4E2B6804
:104D6000002814BF0021082121449942316000F03D
:104D70002D819A4C9A4B22680492049A1A602368F7
:104D800005939848059B0068944F9B1A834220D94D
:104D9000954B1A68914216D03A680792934ADDF80B
:104DA0001CE093481960C2F800E00AF073FC9048D8
:104DB0000AF020FC3B6806938E4A8F4B06981060E1
:104DC000316801221A70012900F0E180042900F005
:104DD000DE808A4F29603D78002D00F0CD80236869
:104DE00082490B93864A0B9B096812687B485B1AC1
:104DF00093423FD9834E84488449854A854D864CE9
:104E0000DFF864C2DFF864E201233370002303702B
:104E10000B70137081488249824A2B702370037093
:104E20000B701370804D814C81488249824A2B70EF
:104E3000237003700B701370804D814C8148824940
:104E4000824A8CF800303B708EF800302B70237053
:104E500003700B701370AE217D48674C07F08CFC1B
:104E6000002333702378002B40F004810DF5257D5D
:104E7000BDE8F083022D00F03381012D00F0E681C2
:104E8000642D00F089810A2D00F02A820B2D01F09B
:104E90003B800C2D01F04781142D01F05482152D1B
:104EA00000F0B883162D01F0B7841E2D01F0BE86E8
:104EB0001F2D01F06487202D02F07480282D02F050
:104EC000D181292D02F078822A2D02F085833C2D94
:104ED00002F073843D2D02F02185502D02F08C8666
:104EE0005A2D02F0D3866E2DC0D1464E3378002B5A
:104EF00043F078804A4D2A78002A02F076872368AA
:104F0000DFF86C818E93534A8E9BD8F8001012689C
:104F10005B1A934211D9504B1A78012A0CBF002218
:104F200001221A701878FDF797FD494807F0BEFD79
:104F300023688F938F9BC8F800302F4A1378002B7B
:104F400094D0294B1B680021013B1170072B8DD891
:104F500001A252F823F000BF35950000079500002C
:104F60006D4E0000D19400006D4E00006D4E0000AB
:104F70006D4E0000A3940000224E3378002B7FF486
:104F80006AAF1D4C2378002B3FF470AF72E02368AA
:104F90001848324A08930668089B10680F4A9B1B02
:104FA00083427FF616AF13682D4809932D4E099B57
:104FB00007683668DB1BB3427FF60BAF13680A93B2
:104FC0000A9A0D4B026001221A7002E7044B034C4F
:104FD0001A68D4E6249EFF1FEC9EFF1F3C9FFF1F14
:104FE000949EFF1F608CFF1F8C9EFF1F909DFF1FD4
:104FF0001094FF1F089EFF1FF49DFF1F0C9EFF1FB4
:10500000F08DFF1F588CFF1F5A9DFF1FD09EFF1F62
:105010008C9DFF1F449EFF1F589DFF1F649DFF1F17
:105020002E9EFF1FC19DFF1F969DFF1FB69DFF1F58
:10503000EC9DFF1F3D9EFF1FE09EFF1F509EFF1F28
:10504000009EFF1FDC9DFF1FDC9EFF1FDD9EFF1FDC
:10505000009FFF1F908DFF1F889EFF1F508AFF1F1C
:10506000889DFF1FB48CFF1FA69EFF1FED9DFF1F95
:10507000389EFF1F00232370FBF782FBB94ABA4B0F
:10508000BA49BB4812781B780968007802EB4303E1
:105090004A1E03EB80030E2A3FF6E8AE01A151F849
:1050A00022F000BF4F550000675500006D4E000014
:1050B000175500006D4E00006D4E00006D4E000053
:1050C000DD5400006D4E00006D4E00006D4E00007E
:1050D0006D4E00006D4E00006D4E0000D954000072
:1050E000A44E3378002B40F00287A34D2A68236832
:1050F0000D93A2490D9B09689B1A8B4211D9A048B8
:10510000A04901220023027026200B703B703270F0
:10511000FBF700FD9C4B1988884202D02620FBF744
:10512000EDFC9A4B1A78002A3FF4A0AE00221A70C8
:10513000FBF726FB8B4A8C4B8C498D4812781B78E9
:105140000968007802EB43034A1E03EB80030E2A32
:105150003FF68CAE01A151F822F000BF9557000038
:10516000655700006D4E00001F5700006D4E000097
:105170006D4E00006D4E0000F95600006D4E0000AF
:10518000DB5700006D4E00006D4E00006D4E0000BC
:105190006D4E0000D9540000764E3378002B41F05C
:1051A000CC807B4D2B78002B40F05081DFF8F891BC
:1051B00099F80050002D01F05D812368DFF8EC8143
:1051C0002493744AD8F80010249B12685B1A934207
:1051D000714A117800D8C1B1704B1878012802F0DB
:1051E000D78001201870002941F0D68618786C4BC2
:1051F000013D53F82510FDF76DFD6A4807F056FC98
:1052000023682593259BC8F80030604A1378002B4B
:105210003FF42CAE554B1B680021013B1170072B4E
:105220003FF624AE01A252F823F000BF635C0000F9
:10523000235C00006D4E0000D95B00006D4E000045
:105240006D4E00006D4E00008B5B0000494E3378C0
:10525000002B40F06287DFF8589199F80000002891
:1052600000F0A8802368DFF844811293494A129B1A
:10527000D8F8001012685B1A934210D9474B1A787D
:10528000012A0CBF002001201870FDF7B7FE454829
:1052900007F00CFC23681393139BC8F800303B4ABB
:1052A0001378002B3FF4E2AD304B1B680021013B2B
:1052B0001170072B3FF6DAAD01A252F823F000BFC0
:1052C00079590000495900006D4E00001359000043
:1052D0006D4E00006D4E00006D4E0000E358000062
:1052E000244E3378002B40F08D812368DFF8BC809A
:1052F0002E93284A2E9BD8F8001012685B1A93420E
:1053000010D9264B1A78012A0CBF002001201870F2
:10531000FBF77AFB234807F0C9FB23682F932F9BE9
:10532000C8F80030194A1378002B3FF49FAD0F4B9B
:105330001B680021013B1170072B3FF697AD01A2BE
:1053400052F823F0AD580000A55800006D4E000043
:105350006F5800006D4E00006D4E00006D4E000055
:105360003B580000D19EFF1F2C9FFF1F8C9EFF1FEC
:105370002D9FFF1F588CFF1FA89DFF1FEC8DFF1F47
:10538000959DFF1F669DFF1F649EFF1FF49DFF1FDD
:105390003D9EFF1F908DFF1FF89EFF1F889EFF1FE1
:1053A000448CFF1F009FFF1FE09EFF1F389EFF1FC2
:1053B000A69EFF1FDFF8349399F80030002B40F0D1
:1053C000E580DFF82C9399F80020002A01F0508145
:1053D0002268DFF820831A92B1491A9AD8F800009F
:1053E0000968121A8A4211D9AE4A117801290BBFF5
:1053F0001846012013701070FCF79AFDAA4807F0B8
:1054000055FB23681B931B9BC8F80030A74A1378F1
:10541000002B3FF42BADA64B1B680021013B117004
:10542000072B3FF623AD01A252F823F0835E000064
:10543000475E00006D4E0000B95E00006D4E00003A
:105440006D4E00006D4E0000175E00002368DFF80F
:10545000A4822093924AD8F80010209B12685B1A0D
:105460009342944A117800D8B1B18E4B1878012834
:1054700001F08E8501201870002941F0AB83187867
:105480008D4B1968FDF726FC874807F00FFB236852
:105490002193219BC8F80030844A1378002B3FF4F5
:1054A000E5AC834B1B680021013B1170072B3FF6D5
:1054B000DDAC01A252F823F0855A0000515A0000D9
:1054C0006D4E0000195A00006D4E00006D4E000038
:1054D0006D4E0000AF59000008F0B8FE774B7849D8
:1054E0001C78784B784A09881B8812680B44002C7A
:1054F00001F08C80B2EB630F81F28A86734B1B78CC
:10550000002B01F03284AF21674807F035F9012301
:105510003B703370AAE4002B01F0A680013B6C4A7B
:1055200032F813304BB16B4D6B486C496C4A2B8091
:105530000123002505700B701370AF215A4807F046
:105540001BF9012302223A70237033708EE463B991
:1055500001232370AF21544807F00EF902220123E2
:105560003A70337082E4002BF4D0013B584A32F891
:105570001330002BEED0574C57485849584A2380D7
:105580000123002404700B701370E3E72368DFF835
:1055900064811693424A169BD8F8001012685B1A71
:1055A00093420FD93F4B1A78012A18BF0120187077
:1055B000FDF7A8FD3C4807F079FA23681793179B7D
:1055C000C8F80030394A1378002B3FF44FAC384B01
:1055D0001B680021013B1170072B3FF647AC01A26D
:1055E00052F823F0555B0000255B00006D4E000073
:1055F000EF5A00006D4E00006D4E00006D4E000031
:10560000BF5A0000FEF7B8FD364A01210023117091
:1056100033706AE62368DFF8DC803A93204A3A9BCD
:10562000D8F8001012685B1A934219D91D4A1E4817
:105630001378012B0CBF0023012313702A4A019316
:10564000B2F900301A2219460092142206F042FAEA
:10565000154807F02BFA23683B933B9BC8F80030B2
:10566000124A1378002B3FF401AC114B1B68002148
:10567000013B1170072B3FF6F9AB01A252F823F062
:10568000975D0000715D00006D4E0000F15C000050
:105690006D4E00006D4E00006D4E0000AF5C0000CE
:1056A000908DFF1F889EFF1F009FFF1FF49DFF1F0F
:1056B0008C9EFF1FF89EFF1F048BFF1F949DFF1FF2
:1056C0008E9DFF1F469EFF1FBC9DFF1FB79DFF1FA6
:1056D000709DFF1F649EFF1FEE9DFF1F959DFF1F86
:1056E000669DFF1F679DFF1F609DFF1FAC9DFF1FF5
:1056F000ED9DFF1F389EFF1FBA4C2378012B41F20E
:1057000053862620FBF706FAB74B1988884202D049
:105710002620FBF7F3F900232370FFF7A7BB002B2C
:1057200001F04185013BB14A32F8136096B1AE4BAE
:10573000AF48B049AB4A1E800027012307702620DE
:105740000B701370FBF7E6F9864203D03146262032
:10575000FBF7D4F9FFF730F823681093109B2B6008
:10576000FFF784BB83B1013BA04A32F813305BB131
:105770009D4E9F489F499B4A338001230026067017
:105780000B701370FFF718F823680F930F9B2B60B3
:10579000FFF76CBB002B01F0F484013B934A32F815
:1057A000136096B1904B924892498E4A1E80002712
:1057B0000123077026200B701370FBF7ABF98642AC
:1057C00003D031462620FBF799F9FEF7F5FF236851
:1057D0000E930E9B2B60FFF749BBFBF74BFD8648F2
:1057E00006F0C2FF0121844806F010FD0221824824
:1057F00006F006FD0F2223217F4806F0FDFC05225E
:105800007E497D4809F0E2FE7B4809F0F3FE1E2246
:105810002321794806F0F0FC05227949764809F001
:10582000D5FE754809F0E6FE734807F03FF9236896
:105830001193119B2B60FFF719BB012302203B70D2
:105840003370FBF767F96F4B1988884202D002204A
:10585000FBF754F90420FBF75DF96B4B198888427C
:105860003FF404AB0420FBF749F9FFF7FFBA01232B
:105870003C22022033703A70FBF74CF9614B1988D7
:10588000884202D00220FBF739F90420FBF742F9E5
:105890005D4B198888423FF4E9AA0420FBF72EF9F2
:1058A000FFF7E4BA0B233B70FFF7E0BA01231422A1
:1058B000022033703A70FBF72DF9524B1988884259
:1058C00002D00220FBF71AF90420FBF723F94E4B14
:1058D000198888423FF4CAAA0420FBF70FF9FFF7A2
:1058E000C5BA0120FDF78AFB484B434800241C70D1
:1058F00007F0DCF80E2089F80040FBF70BF9444B69
:10590000198888423FF4B2AA0E20FBF7F7F8FFF798
:10591000ADBA3F4D2B88172B3FF6A8AA0020FDF704
:105920006DFB2B88012003442B80FDF767FB374B71
:10593000314800221A7007F0B9F823681593159BB7
:10594000C8F80030FFF792BA0120FDF757FB2F4B44
:10595000294800241C7007F0A9F80E2089F800409F
:10596000FBF7D8F82A4B198888423FF47FAA0E200B
:10597000FBF7C4F8FFF77ABA254D2B88002B3FF4CC
:1059800075AA0020FDF73AFB2B880120013B2B80F4
:10599000FDF734FB1D4B184800221A7007F086F8FB
:1059A00023681493149BC8F80030FFF75FBA194CB2
:1059B00001202168FDF78EF9144B0F4800261E7058
:1059C00007F074F844202E70FBF7A4F82168183112
:1059D00088423FF44BAA89B24420FBF78FF8FFF7C7
:1059E00045BA00BF669DFF1F649EFF1F709DFF1F8D
:1059F000EE9DFF1F959DFF1F009FFF1FB037010009
:105A0000B8370100169EFF1FE89EFF1F889EFF1FEC
:105A1000A49DFF1F048BFF1FAE4D296817293FF778
:105A200025AA0020FDF756F92B68013319460120FD
:105A30002B60FDF74FF9A84BA84800221A7007F019
:105A400035F823682393239BC8F80030FFF70EBA7C
:105A5000A04C01202168FDF73DF99F4B9F4800268F
:105A60001E7007F023F844202E70FBF753F82168CE
:105A7000183188423FF4FAA989B24420FBF73EF876
:105A8000FFF7F4B9934D296811F1170FFFF6EEA94E
:105A90000020FDF71FF92B68013B194601202B6000
:105AA000FDF718F98C4B8D4800221A7006F0FEFFA6
:105AB00023682293229BC8F80030FFF7D7B9012052
:105AC000FDF720FB844B854800241C7006F0EEFF98
:105AD000282089F80040FBF71DF8814B198888427F
:105AE0003FF4C4A92820FBF709F8FFF7BFB97C4DA4
:105AF0002B88052B3FF6BAA90020FDF703FB2B8866
:105B0000012003442B80FDF7FDFA734B73480022FC
:105B10001A7006F0CBFF23681993199BC8F8003060
:105B2000FFF7A4B90120FDF7EDFA6B4B6B48002499
:105B30001C7006F0BBFF282089F80040FAF7EAFF46
:105B4000674B198888423FF491A92820FAF7D6FFBD
:105B5000FFF78CB9624D2B88002B3FF487A90020FA
:105B6000FDF7D0FA2B880120013B2B80FDF7CAFA04
:105B7000594B5A4800221A7006F098FF2368189370
:105B8000189BC8F80030FFF771B999F80030554EEE
:105B9000013B012056F82310FDF79CF84E4B4F486F
:105BA00000221A7006F082FF99F8005005F12204D5
:105BB0006400E4B2013D2046FAF7ACFF56F8251028
:105BC0001831884203D089B22046FAF797FF0023A4
:105BD00089F80030FFF74AB999F80030414D424E3C
:105BE000013B55F8231017293FF740A90020FDF786
:105BF00071F83378013B012055F823200244114607
:105C000045F82320FDF766F8334B344800221A701C
:105C100006F04CFF23682793279BC8F80030FFF756
:105C200025B999F800302F4E013B012056F823107A
:105C3000FDF750F8284B294800221A7006F036FF6D
:105C400099F8005005F122046400E4B22046013DB9
:105C5000FAF760FF56F825309842B8D003F11801E2
:105C6000B1E799F800301F4D1F4E013B55F8231046
:105C700011F1170FFFF6FAA80020FDF72BF8337883
:105C8000013B012055F82320013A114645F8232015
:105C9000FDF720F8104B114800221A7006F006FF9D
:105CA00023682693269BC8F80030FFF7DFB80F4B18
:105CB0000A48B3F90030142401221A2501920095F4
:105CC000194622463C7005F005FF044806F0EEFE3A
:105CD000FFF7CCB8048BFF1F889EFF1F009FFF1F9C
:105CE000B29EFF1F448CFF1FE09EFF1F609DFF1FA1
:105CF000B24EB34BB34F32881B6839681A448A429C
:105D0000BFF6B4A8B04D3280B5F90030AF484FF0BF
:105D1000000E1A2219468DE80440142205F0DAFE1E
:105D2000AB4B3A6819683388521A5C2A42F34280B6
:105D3000591A5D23561C03FB01F393FBF6F61B3641
:105D400033B201211A2201910092194614229F4870
:105D50002E6005F0BFFE9D4806F0A8FE23683D9327
:105D60003D9A9C4BC8F8002000221A70FFF77EB8BD
:105D7000954B9648B3F9003001241A228DE814009F
:105D80001624194614223C7005F0A4FE8F4806F034
:105D90008DFEFFF76BB8894E894A8D4F33881268A4
:105DA00039689A1A8A427FF761A8874D3280B5F91F
:105DB000003086484FF0000E1A2219468DE8044044
:105DC000142205F087FE7F4B39681A683388521A0F
:105DD0005C2A41F3F887591A5D23561C03FB01F333
:105DE00093FBF6F61B3633B201211A220191009281
:105DF0001946142275482E6005F06CFE734806F0B3
:105E000055FE23683C933C9A724BC8F80020002250
:105E10001A70FFF72BB80120FCF78AF86D4B6B481E
:105E200000241C7006F042FE102089F80040FAF7AA
:105E300071FE694B198888423FF418A81020FAF7C0
:105E40005DFEFFF713B8FAF79BFC644B1C78002C3F
:105E500041F0B8860120FCF76BF85E4B5B481C7084
:105E600006F024FE102089F80040FAF753FE5A4B42
:105E7000198888423EF4FAAF1020FAF73FFEFEF789
:105E8000F5BF554D2B88012B7EF6F0AF0020FCF7B7
:105E90004FF82B880120013B2B80FCF749F84D4B34
:105EA0004A4800221A7006F001FE23681C931C9BCE
:105EB000C8F80030FEF7DABF474D2B880F2B3EF6AF
:105EC000D5AF0020FCF734F82B88012003442B8049
:105ED000FCF72EF83F4B3D4800221A7006F0E6FD15
:105EE00023681D931D9BC8F80030FEF7BFBF0390C9
:105EF000FEF762FC03983A4D03680C930C9A2A60F3
:105F000000233370FFF7F3B80368DFF8E4803093C1
:105F1000344A309BD8F8001012685B1A934219D9A2
:105F20002C4A2A481378012B0CBF0023012313703D
:105F3000254A0193B2F900301A2219460092142220
:105F400005F0C8FD214806F0B1FD23683193319B6F
:105F5000C8F80030244A1378002B3EF487AF234B57
:105F60001B680021013B1170072B3EF67FAF01A299
:105F700052F823F09B600000756000006D4E000039
:105F8000F55F00006D4E00006D4E00006D4E00008C
:105F9000955F00000C4B0D48B3F9003001241A2224
:105FA0008DE814000A24194614223C7005F092FD75
:105FB000064806F07BFDFEF759BF00BFE49DFF1FBA
:105FC000B49EFF1FE48DFF1F609DFF1F009FFF1FFA
:105FD000688AFF1F889EFF1F589EFF1F949DFF1F0A
:105FE000A89DFF1F908DFF1FF49DFF1F8C9EFF1F1C
:105FF000389EFF1FA24EA34BA34F32881B683968FF
:106000001A448A42BEF632AFA04D3280B5F9003054
:106010009F484FF0000E1A2219468DE804401422C2
:1060200005F058FD9B4B3A6819683388521A5C2A70
:1060300041F35A84591A5D23561C03FB01F393FB69
:10604000F6F61B3633B201211A220191009219464D
:1060500014228F482E6005F03DFD8D4806F026FD88
:1060600023683393339A8C4BC8F8002000221A70AF
:10607000FEF7FCBE854B8648B3F9003001241A2296
:106080008DE814000C24194614223C7005F022FD02
:106090007F4806F00BFDFEF7E9BE794E794A7D4F49
:1060A0003388126839689A1A8A427EF7DFAE774DD4
:1060B0003280B5F9003076484FF0000E1A221946AA
:1060C0008DE80440142205F005FD6F4B39681A680D
:1060D0003388521A5C2A41F31084591A5D23561CE6
:1060E00003FB01F393FBF6F61B3633B201211A22B0
:1060F000019100921946142265482E6005F0EAFCD1
:10610000634806F0D3FC23683293329A624BC8F896
:10611000002000221A70FEF7A9BEFCF773FE0023D0
:106120003370FFF798B80368DFF8848134935B4AD3
:10613000349BD8F8001012685B1A934219D9564B59
:1061400053481A78012A0CBF002201221A70544BBE
:106150000192B3F90030392219460092322205F03B
:10616000B9FC4B4806F0A2FC23683593359BC8F870
:1061700000304C4A1378002B3EF478AE4A4B1B6833
:106180000021013B1170072B3EF670AE01A252F8C0
:1061900023F000BFB56200005B6200006D4E00009E
:1061A000DB6100006D4E00006D4E00006D4E000082
:1061B000B56100003A4B3648B3F90030012439226A
:1061C0008DE814000A24194632223C7005F082FC46
:1061D0002F4806F06BFCFEF749BE344E294B2A4F80
:1061E00032881B6839681A448A42BEF63FAE2C4D8D
:1061F0003280B5F9003026484FF0000E392219469A
:106200008DE80440322205F065FC224B3A6819689B
:106210003388521A5C2A41F3A484591A5D23561C10
:1062200003FB01F393FBF6F61B3633B2012139224F
:10623000019100921946322215482E6005F04AFC61
:10624000134806F033FC23683793379A124BC8F88B
:10625000002000221A70FEF709BE114B0C48B3F95A
:106260000030012439228DE814000A241946322214
:106270003C7005F02FFC064806F018FCFEF7F6BD52
:10628000169EFF1F9C9EFF1F588AFF1F609DFF1FC9
:10629000009FFF1F309EFF1F889EFF1F908DFF1FD6
:1062A000A89EFF1FF49DFF1F8C9EFF1FE89EFF1FEF
:1062B000389EFF1FC34FC44AC448C5493B88126873
:1062C000008809689A1A43189A427EF7CFADC14DEB
:1062D0003A80B5F90030C0483922002619468DE8C9
:1062E0004400322205F0F6FBBC4ABD4B11681A6827
:1062F0003B88521A5C2A41F33D84591A5D23561C8F
:1063000003FB01F393FBF6F61B3633B2012139226E
:106310000191009219463222AF482E6005F0DAFB57
:10632000AD4806F0C3FB23683693369AAD4BC8F8E8
:10633000002000221A70FEF799BDFCF7D5FD00235E
:106340003370FEF72EBFA84E3378002B40F0048543
:106350002368DFF8B0823893A44A389BD8F800103D
:1063600012685B1A934210D99E4B1A78012A0CBF0F
:10637000002001201870FAF747FB974806F096FBBB
:1063800023683993399BC8F80030994A1378002B59
:106390003EF46CAD974B1B680021013B1170072B3D
:1063A0003EF664AD01A252F823F000BF3F64000046
:1063B000376400006D4E0000016400006D4E000067
:1063C0006D4E00006D4E0000CD63000001230620DD
:1063D0003B703370FAF79EFB874B1988884202D0D6
:1063E0000620FAF78BFB0820FAF794FB834B1988F9
:1063F00088423EF43BAD0820FAF780FBFEF736BD3D
:1064000001230A22062033703A70FAF783FB7A4B95
:106410001988884202D00620FAF770FB0820FAF7A4
:1064200079FB764B198888423EF420AD0820FAF7B4
:1064300065FBFEF71BBD15233B70FEF717BD01235F
:106440001E22062033703A70FAF764FB6A4B1988F3
:10645000884202D00620FAF751FB0820FAF75AFBCF
:10646000664B198888423EF401AD0820FAF746FBD6
:10647000FEF7FCBCDFF89091236899F80010DFF874
:106480008481002900F0D8822893584A289BD8F8A4
:10649000001012685B1A934211D9524B1A78012AE4
:1064A00015BF0120284618701D70FDF76BF84A488B
:1064B00006F0FCFA23682993299BC8F800304C4A5F
:1064C0001378002B3EF4D2AC4A4B1B680021013BF1
:1064D0001170072B3EF6CAAC01A252F823F000BFA0
:1064E00093650000636500006D4E0000316500009B
:1064F0006D4E00006D4E00006D4E00000165000005
:106500000120FDF73FF8374B334800241C7006F09C
:10651000CDFA4E2089F80040FAF7FCFA384B19887A
:1065200088423EF4A3AC4E20FAF7E8FAFEF79EBC90
:106530000020FDF727F8324A1388B3FA83F35B098A
:1065400001201380FDF71EF8264B234800221A7005
:1065500006F0ACFA23682B932B9BC8F80030FEF7AB
:1065600085BC0120FDF70EF81E4B1B4800241C7053
:1065700006F09CFA4E2089F80040FAF7CBFA204B3F
:10658000198888423EF472AC4E20FAF7B7FAFEF74B
:106590006DBC0020FCF7F6FF194A1388B3FA83F3A9
:1065A0005B0901201380FCF7EDFF0E4B0A48002227
:1065B0001A7006F07BFA23682A932A9BC8F80030E9
:1065C000FEF754BCE89EFF1F9C9EFF1F169EFF1FF8
:1065D0009C8DFF1FA89EFF1F009FFF1F309EFF1F67
:1065E000588AFF1F889EFF1F588CFF1F908DFF1F2A
:1065F000F49DFF1F8C9EFF1FE49DFF1FC89EFF1F81
:10660000C29DFF1F389EFF1F509EFF1FB2EB630FFE
:10661000FEF679AFAD4EAE4D33782A88B3FA83F3E8
:1066200082F002025B091146422033702A80FAF799
:1066300065FA21460D2007F0DDFA962007F016FBDB
:1066400001210D2007F0D6FA962007F00FFB214616
:106650000D2007F0CFFA962007F008FB01210D204E
:1066600007F0C8FAFEF702BC01232370FEF765BFEE
:106670002368DFF894821E9396481E9BD8F800107A
:1066800000685B1A834215D9934B1978012916BF0C
:1066900001221A701A70914B08BF154618782946C6
:1066A000FAF79CF98E4806F001FA23681F931F9BA6
:1066B000C8F800308B4B1A78002A3EF4D7AB002282
:1066C0001A70FAF75DF8884A884B89498948127828
:1066D0001B780968007802EB43034A1E03EB800332
:1066E0000B2A3EF6C3AB01A151F822F0D767000098
:1066F000CF6700006D4E00008D6700006D4E0000FA
:106700006D4E00006D4E0000816700006D4E000070
:106710001D6700006D4E00004F670000002B3EF427
:10672000A5AB754A754D128803F11900013B400075
:10673000022425F813201146012300F0FE003370D7
:106740003C70FAF7DBF96E4B1C70FEF78FBB002B29
:106750003EF48CAB03F11900684D013B0022400070
:1067600025F813201146012300F0FE0002243370A7
:106770003C70FAF7C3F9624B03221A70FEF776BB3E
:10678000002201233A703370FEF770BB534C20781F
:1067900001287EF66BAB0021FAF720F923784E4DE5
:1067A000013BDBB2184601212370FAF717F90024E8
:1067B00034238DE818004A482C7040230B223F21D7
:1067C00005F056F9464806F071F9FEF74FBBFCF7A5
:1067D0001DFDFEF74BBB414C207805283EF646AB2D
:1067E0000021FAF7FBF823783B4D0133DBB2184662
:1067F00001212370FAF7F2F8002434238DE8180001
:1068000037482C7040230B223F2105F031F93448E2
:1068100006F04CF9FEF72ABB2368DFF8EC803E93C4
:106820002C4A3E9BD8F8001012685B1A934219D983
:10683000294A2B481378012B0CBF00230123137026
:10684000304A0193B2F900303922194600923222BF
:1068500005F040F9224806F029F923683F933F9B51
:10686000C8F800301F4A1378002B3EF4FFAA204BD3
:106870001B680021013B1170072B3EF6F7AA01A20D
:1068800052F823F0B36900008D6900006D4E0000DE
:106890000D6900006D4E00006D4E00006D4E000051
:1068A000A5680000174B0E48B3F9003001243922C7
:1068B0008DE814001424194632223C7005F00AF9C0
:1068C000074806F0F3F8FEF7D1BA00BFBA9DFF1FE4
:1068D000EA9EFF1F908DFF1F889EFF1F3289FF1FBA
:1068E000009FFF1FF49DFF1FD19EFF1F2C9FFF1FC6
:1068F0008C9EFF1F2D9FFF1F649EFF1F709DFF1F1B
:10690000669DFF1FA89EFF1F389EFF1FB44EB54B0C
:10691000B54F32881B6839681A448A42BEF6A6AA67
:10692000B24D3280B5F90030B1484FF0000E392237
:1069300019468DE80440322205F0CCF8AD4B3A6898
:1069400019683388521A5C2A41F34682591A5D232A
:10695000561C03FB01F393FBF6F61B3633B2012101
:1069600039220191009219463222A1482E6005F089
:10697000B1F89F4806F09AF823684193419A9E4BDC
:10698000C8F8002000221A70FEF770BA974B98489A
:10699000B3F90030012439228DE81400142419467B
:1069A00032223C7005F096F8914806F07FF8FEF729
:1069B0005DBA8B4E8B4A91489149338812680088A2
:1069C00009689A1A43189A427EF750AA874D328076
:1069D000B5F9003086483922002719468DE8840031
:1069E000322205F077F8834A7F4B11681A683388A2
:1069F000521A5C2A41F33C82591A5D23561C03FB50
:106A000001F393FBF6F61B3633B2012139220191D3
:106A100000921946322276482E6005F05BF87448E1
:106A200006F044F823684093409A734BC8F800205E
:106A300000221A70FEF71ABA2C93724A2C9BD8F8CF
:106A4000000012681B1A934211D96B4B1A78012A65
:106A500018BF012119706C4B1878F9F7BFFF644813
:106A600006F024F823682D932D9BC8F80030674B5F
:106A70001A78002A3EF4FAA900221A70F9F780FE6B
:106A8000634A644B6449654812781B78096800784A
:106A900002EB43034A1E03EB80030B2A3EF6E6A9F2
:106AA00001A151F822F000BF936B00008B6B000036
:106AB0006D4E0000496B00006D4E00006D4E0000F1
:106AC0006D4E00003D6B00006D4E0000D96A000065
:106AD0006D4E00000B6B0000002B3EF4C7A9504A1E
:106AE000504D128803F11900013B4000022425F8A3
:106AF00013201146012300F0FE0033703C70F9F7BB
:106B0000FDFF494B1C70FEF7B1B9002B3EF4AEA956
:106B100003F11900434D013B0022400025F81320EA
:106B20001146012300F0FE00022433703C70F9F797
:106B3000E5FF3D4B03221A70FEF798B900220123AE
:106B40003A703370FEF792B92F4C207801287EF608
:106B50008DA90021F9F742FF2378274D013BDBB2D5
:106B6000184601212370F9F739FF002434238DE8FA
:106B700018001F482C7040230B223F2104F078FF9F
:106B80001B4805F093FFFEF771B9FCF759FDFEF7BE
:106B90006DB91D4C207805283EF668A90021F9F74B
:106BA0001DFF2378144D0133DBB2184601212370F9
:106BB000F9F714FF002434238DE818000C482C70DA
:106BC00040230B223F2104F053FF094805F06EFFDC
:106BD000FEF74CB90021012011701870FEF750BC6F
:106BE000C89EFF1FB49EFF1FE48DFF1FA89EFF1FBE
:106BF000009FFF1F688AFF1F889EFF1FE49DFF1FE5
:106C00009C8DFF1F908DFF1F948DFF1FF49DFF1F14
:106C1000D19EFF1F2C9FFF1F8C9EFF1F2D9FFF1FCC
:106C2000649EFF1F709DFF1F669DFF1FAA4E337855
:106C3000002B40F0B1832368DFF8D0824293A74A4B
:106C4000429BD8F8001012685B1A934210D9A44BEB
:106C50001A78012A0CBF002001201870F9F7D4FE21
:106C6000A04805F023FF23684393439BC8F80030F6
:106C70009D4A1378002B3EF4F9A89C4B1B68002119
:106C8000013B1170072B3EF6F1A801A252F823F048
:106C9000236D00001B6D00006D4E0000E56C0000D0
:106CA0006D4E00006D4E00006D4E0000B16C000096
:106CB00001230A203B703370F9F72CFF8C4B1988A5
:106CC000884202D00A20F9F719FF0C20F9F722FFB9
:106CD000884B198888423EF4C9A80C20F9F70EFFAA
:106CE000FEF7C4B8012314220A2033703A70F9F772
:106CF00011FF7F4B1988884202D00A20F9F7FEFE67
:106D00000C20F9F707FF7B4B198888423EF4AEA8A8
:106D10000C20F9F7F3FEFEF7A9B81F233B70FEF72E
:106D2000A5B8012328220A2033703A70F9F7F2FE41
:106D30006F4B1988884202D00A20F9F7DFFE0C2039
:106D4000F9F7E8FE6B4B198888423EF48FA80C20B7
:106D5000F9F7D4FEFEF78AB8FCF7C6FF664A0121B0
:106D6000002311703370FFF7F3BAAF215D4805F0CF
:106D700003FD642201233A703370FEF777B823686D
:106D8000DFF888814493554A449BD8F80010126874
:106D90005B1A934219D9524A52481378012B0CBFFF
:106DA000002301231370554A0193B2F900301A22CF
:106DB00019460092142204F08DFE4A4805F076FE32
:106DC00023684593459BC8F80030474A1378002B49
:106DD0003EF44CA8454B1B680021013B1170072B6A
:106DE0003EF644A801A252F823F000BF116F000044
:106DF000B36E00006D4E0000336E00006D4E00005B
:106E00006D4E00006D4E00000D6E00003B4B35488E
:106E1000B3F9003001241A228DE814001E2419460B
:106E200014223C7004F056FE2E4805F03FFEFEF79B
:106E30001DB82F4E324B334F32881B6839681A44C5
:106E40008A42BEF613A82D4D3280B5F90030254890
:106E50004FF0000E1A2219468DE80440142204F067
:106E600039FE294B3A6819683388521A5C2A41F373
:106E7000AB80591A5D23561C03FB01F393FBF6F616
:106E80001B3633B201211A220191009219461422B5
:106E900014482E6004F01EFE124805F007FE236819
:106EA0004793479A0E4BC8F8002000221A70FDF74E
:106EB000DDBF124B0B48B3F9003001241A228DE8D4
:106EC00014002024194614223C7004F003FE0548E7
:106ED00005F0ECFDFDF7CABF588CFF1F908DFF1F1A
:106EE000889EFF1F009FFF1FF49DFF1F8C9EFF1FAA
:106EF0002C9EFF1FB49DFF1F679DFF1F609DFF1FFE
:106F0000A09EFF1F3C8BFF1FE88DFF1F389EFF1FB9
:106F1000AD4EAE4AAE4F3388126839689A1A8A422B
:106F20007DF7A4AFAB4D3280B5F90030AA484FF0E1
:106F3000000E1A2219468DE80440142204F0CAFDFE
:106F4000A64B39681A683388521A5C2A41F3948038
:106F5000591A5D23561C03FB01F393FBF6F61B360F
:106F600033B201211A2201910092194614229A4843
:106F70002E6004F0AFFD984805F098FD2368469315
:106F8000469A974BC8F8002000221A70FDF76EBF92
:106F900000201870FEF770BA0021012011701870DF
:106FA000FEF725B92368DFF8648248938D4A489B31
:106FB000D8F8001012685B1A934219D9884A86489B
:106FC0001378012B0CBF002301231370864A019311
:106FD000B2F90030392219460092322204F07AFDCB
:106FE0007D4805F063FD23684993499BC8F800304C
:106FF0007E4A1378002B3DF439AF7D4B1B6800218E
:10700000013B1170072B3DF631AF01A252F823F07E
:10701000FD700000D77000006D4E0000577000003A
:107020006D4E00006D4E00006D4E0000317000008E
:107030006D4B6948B3F90030012439228DE8140002
:107040001E24194632223C7004F044FD624805F0CB
:107050002DFDFDF70BBF674E5C4B604F32881B6800
:1070600039681A448A42BDF601AF5F4D3280B5F9E6
:10707000003059484FF0000E392219468DE804407F
:10708000322204F027FD524B3A6819683388521AAD
:107090005C2A41F37D80591A5D23561C03FB01F3E2
:1070A00093FBF6F61B3633B201213922019100928F
:1070B0001946322248482E6004F00CFD464805F07F
:1070C000F5FC23684B934B9A454BC8F800200022EF
:1070D0001A70FDF7CBBE444B3F48B3F90030012492
:1070E00039228DE814001E24194632223C7004F027
:1070F000F1FC394805F0DAFCFDF7B8BE3D4E334AE5
:1071000031483D4933881268008809689A1A431843
:107110009A427DF7ABAE344D3280B5F900302E483F
:107120003922002719468DE88400322204F0D2FC6F
:10713000274A2A4B11681A683388521A5C2A41F38D
:107140004780591A5D23561C03FB01F393FBF6F6A7
:107150001B3633B2012139220191009219463222A5
:107160001D482E6004F0B6FC1B4805F09FFC236808
:107170004A934A9A1A4BC8F8002000221A70FDF769
:1071800075BE1E4A1E4E13881E48012B8CBF03F18C
:10719000FF33802313801C4A0023012133700370C6
:1071A0001170FEF712BB154A154E138815487F2B38
:1071B00094BF013301231380134A0023012133704C
:1071C00003701170FEF7C6BA2C9EFF1FA09EFF1F12
:1071D000E88DFF1F609DFF1F009FFF1F3C8BFF1F5F
:1071E000889EFF1F908DFF1FA89EFF1FF49DFF1F0D
:1071F0008C9EFF1FB49DFF1F9C8DFF1F649EFF1F71
:10720000EE9DFF1F669DFF1F959DFF1F389EFF1F70
:10721000C04DC14C2B782288B3FA83F382F004026C
:107220005B09114642202B702280F9F767FC002190
:107230000D2006F0DFFC962006F018FD01210D2040
:1072400006F0D8FC962006F011FD00210D2006F076
:10725000D1FC962006F00AFD01210D2006F0CAFCA3
:10726000FDF704BEAD4E3378002B40F04F8323680A
:10727000DFF8E0824C93AA4A4C9BD8F800101268C1
:107280005B1A934210D9A74B1A78012A0CBF002031
:1072900001201870F9F7B8FBA34805F007FC236834
:1072A0004D934D9BC8F80030A04A1378002B3DF455
:1072B000DDAD9F4B1B680021013B1170072B3DF694
:1072C000D5AD01A252F823F05B73000053730000A8
:1072D0006D4E00001D7300006D4E00006D4E0000ED
:1072E0006D4E0000E9720000012322203B703370D4
:1072F000F9F710FC8F4B1988884202D02220F9F749
:10730000FDFB2420F9F706FC8B4B198888423DF4DD
:10731000ADAD2420F9F7F2FBFDF7A8BD01231E2235
:10732000222033703A70F9F7F5FB824B19888842B6
:1073300002D02220F9F7E2FB2420F9F7EBFB7E4B89
:10734000198888423DF492AD2420F9F7D7FBFDF768
:107350008DBD29233B70FDF789BD01233C222220EE
:1073600033703A70F9F7D6FB724B1988884202D015
:107370002220F9F7C3FB2420F9F7CCFB6E4B1988C8
:1073800088423DF473AD2420F9F7B8FBFDF76EBDDC
:1073900000201870FDF727BFFCF782FB674A012128
:1073A00000231170337046E46549012300220B70FD
:1073B00033703A70FEF7A5B92368DFF898814E93D1
:1073C000574A4E9BD8F8001012685B1A93421AD99C
:1073D000544B5C491A785448012A0CBF0022012200
:1073E0001A701A78B1F9003001921A2219460092E7
:1073F000142204F06FFB4C4805F058FB23684F93B0
:107400004F9BC8F80030494A1378002B3DF42EAD4D
:10741000474B1B680021013B1170072B3DF626AD41
:1074200001A252F823F000BF59750000EF7400006C
:107430006D4E00006F7400006D4E00006D4E000038
:107440006D4E0000497400003E4B3748B3F90030E0
:1074500001241A228DE814002824194614223C70B5
:1074600004F038FB304805F021FBFDF7FFBC314E3E
:10747000354B364F32881B6839681A448A42BDF64C
:10748000F5AC304D3280B5F9003027484FF0000E92
:107490001A2219468DE80440142204F01BFB2C4BE1
:1074A0003A6819683388521A5C2A41F32882591ABB
:1074B0005D23561C03FB01F393FBF6F61B3633B238
:1074C00001211A22019100921946142216482E60B9
:1074D00004F000FB144805F0E9FA23685193519A2F
:1074E000104BC8F8002000221A70FDF7BFBC154BE6
:1074F0000D48B3F9003001241A228DE814002A2423
:10750000194614223C7004F0E5FA074805F0CEFA5B
:10751000FDF7ACBC149EFF1FEA9EFF1F588CFF1F97
:10752000908DFF1F889EFF1F009FFF1FF49DFF1F70
:107530008C9EFF1F8E9DFF1F469EFF1F679DFF1F96
:10754000959DFF1F609DFF1F4C9EFF1F5C8AFF1FC4
:10755000FC8DFF1F389EFF1FB94EBA4ABA4F3388C1
:10756000126839689A1A8A427DF780ACB74D32802A
:10757000B5F90030B6484FF0000E1A2219468DE8D2
:107580000440142204F0A6FAB24B39681A68338812
:10759000521A5C2A41F3C581591A5D23561C03FB1C
:1075A00001F393FBF6F61B3633B201211A22019147
:1075B000009219461422A6482E6004F08BFAA448C3
:1075C00005F074FA23685093509AA34BC8F8002032
:1075D00000221A70FDF74ABC2368DFF89C825293A0
:1075E0009E4A529BD8F8001012685B1A93421AD92F
:1075F000994B9B491A789648012A0CBF0022012218
:107600001A701A78B1F900300192392219460092A5
:10761000322204F05FFA8E4805F048FA236853934B
:10762000539BC8F800308F4A1378002B3DF41EACF2
:107630008D4B1B680021013B1170072B3DF616ACEA
:1076400001A252F823F000BF357700000F77000049
:107650006D4E00008F7600006D4E00006D4E0000F4
:107660006D4E0000697600007D4B7948B3F900301B
:10767000012439228DE814002824194632223C7056
:1076800004F028FA724805F011FAFDF7EFBB774EC7
:107690006C4B704F32881B6839681A448A42BDF6B9
:1076A000E5AB6F4D3280B5F9003069484FF0000E00
:1076B000392219468DE80440322204F00BFA624B5D
:1076C0003A6819683388521A5C2A40F34986591A75
:1076D0005D23561C03FB01F393FBF6F61B3633B216
:1076E00001213922019100921946322258482E6018
:1076F00004F0F0F9564805F0D9F923685593559AE6
:10770000554BC8F8002000221A70FDF7AFBB544B50
:107710004F48B3F90030012439228DE814002824A1
:10772000194632223C7004F0D5F9494805F0BEF9FB
:10773000FDF79CBB4D4E434A41484D493388126882
:10774000008809689A1A43189A427DF78FAB444D16
:107750003280B5F900303E483922002719468DE8BD
:107760008400322204F0B6F9374A3A4B11681A689D
:107770003388521A5C2A41F3DD80591A5D23561C66
:1077800003FB01F393FBF6F61B3633B201213922DA
:1077900001910092194632222D482E6004F09AF988
:1077A0002B4805F083F923685493549A2A4BC8F860
:1077B000002000221A70FDF759BB2E4E3378002BA3
:1077C00040F0F0822368DFF8B0805693234A569B3E
:1077D000D8F8001012685B1A934211D91E4B1A7820
:1077E000012A0CBF002201221A701878F9F70CF94F
:1077F000174805F05BF923685793579BC8F800308A
:10780000184A1378002B3DF431AB174B1B6800214D
:10781000013B1170072B3DF629AB01A252F823F072
:10782000C7780000BF7800006D4E00009D78000012
:107830006D4E00006D4E00006D4E00007D78000022
:107840008E9DFF1F4C9EFF1FFC8DFF1F609DFF1F25
:10785000009FFF1F5C8AFF1F889EFF1F908DFF1FE8
:10786000A89EFF1FF49DFF1F8C9EFF1F469EFF1FBB
:107870009C8DFF1F588CFF1F389EFF1F01232A205D
:107880003B703370F9F746F9BF4B198888423DF4D5
:10789000EDAA2A20F9F732F9FDF7E8BA01232822E8
:1078A0002A2033703A70F9F735F9B74B19888842B6
:1078B0003DF4DCAA2A20F9F721F9FDF7D7BA3D23D8
:1078C0003B70FDF7D3BA01230A222A2033703A70A5
:1078D000F9F720F9AC4B198888423DF4C7AA2A2051
:1078E000F9F70CF9FDF7C2BA5E1A5C2303FB06F345
:1078F00093FBF2F61B36FEF7A5BB5E1A5C2303FB77
:1079000006F393FBF2F61B36FEF7EFBBFCF710FB1A
:107910009E4A0121002311703370A8E42368DFF828
:107920009C8258939A4A589BD8F8001012685B1AA8
:1079300093421AD9974B98491A789848012A0CBF54
:10794000002201221A701A78B1F9003001921A222D
:1079500019460092142204F0BDF8904805F0A6F8EC
:1079600023685993599BC8F800308D4A1378002B2F
:107970003DF47CAA8B4B1B680021013B1170072B47
:107980003DF674AA01A252F823F000BFAF7A0000BE
:10799000897A00006D4E0000D37900006D4E000022
:1079A0006D4E00006D4E0000AD7900007A4B7B48B3
:1079B000B3F9003001241A228DE814003C24194642
:1079C00014223C7004F086F8744805F06FF8FDF757
:1079D0004DBA6D4E744A754F33881268D7F800E07F
:1079E0001A447245BDF642AA7149724BDFF8D09134
:1079F00008681D68D9F8001093B2CEEB01012A1A6D
:107A000091423380644DCEEB0303CCBF02FB0333C2
:107A10005343694AC8BF013193FBF1F3B5F9001034
:107A2000034413604FF0000E1A220B468DE8044009
:107A30005A48142204F04EF8D9F800103A683388F6
:107A4000521A5C2A40F36487591A5D23561C03FBC3
:107A500001F393FBF6F61B3633B201211A22019192
:107A60000092194614224D482E6004F033F84B481A
:107A700005F01CF823685B935B9A464BC8F800201E
:107A800000221A70FDF7F2B9434B4448B3F90030B5
:107A900001241A228DE814003C24194614223C705B
:107AA00004F018F83D4805F001F8FDF7DFB9364E4F
:107AB0003D4ADFF80C9133881268D9F800509A1AC1
:107AC000AA427DF7D3A93B4B384F3949D7F800E09C
:107AD0001868096893B2CEEB0505421A95423380C7
:107AE000CEEB030341F3A08302FB03336A1C93FB39
:107AF000F2F31944284D304AB5F9003011604FF0C7
:107B0000000E1A2219468DE804402448142203F07E
:107B1000E1FFD9F800103A683388521A5C2A41F321
:107B20007A83591A5D23561C03FB01F393FBF6F687
:107B30001B3633B201211A220191009219461422F8
:107B400016482E6003F0C6FF144804F0AFFF236808
:107B50005A935A9A0F4BC8F8002000221A70FDF76A
:107B600085B95E1A5C2303FB06F393FBF2F61B3622
:107B7000FEF75BBB5E1A5C2303FB06F393FBF2F696
:107B80001B36FEF7C2BB00BFF09EFF1F679DFF1FA5
:107B9000908DFF1F889EFF1F609DFF1F009FFF1F8E
:107BA000F49DFF1F8C9EFF1FD89DFF1F408CFF1F61
:107BB000608AFF1F5C8CFF1F548CFF1F389EFF1FC5
:107BC000F48DFF1FAF4A1378B3FA83F35B090120EA
:107BD0001370FAF7ADF9AC4BAC4800221A7004F000
:107BE00065FFAB4A138883F00803194642201380CF
:107BF000F8F784FFFDF73AB9A64E33781BB1FBF7CF
:107C000099F900233370A44D2978002900F086806B
:107C10002368DFF8A4825C93A04A5C9BD8F800102C
:107C200012685B1A934211D9974B1A78012A0CBF3C
:107C3000002201221A701878FCF730FE934804F0F5
:107C400035FF23685D935D9BC8F80030944A137834
:107C5000002B3DF40BA9934B1B680021013B1170D5
:107C6000072B3DF603A901A252F823F0E189000099
:107C7000AF8900006D4E0000798900006D4E000054
:107C80006D4E00006D4E000047890000814E337834
:107C9000002B40F0A281844D2A78002A00F00E814A
:107CA0002368DFF8148278937C4A789BD8F8001018
:107CB00012685B1A934211D9734B1A78012A0CBFD0
:107CC000002201221A701878FCF7F0FB6F4804F0CC
:107CD000EDFE23687993799BC8F80030704A1378D9
:107CE000002B3DF4C3A86F4B1B680021013B1170B2
:107CF000072B3DF6BBA801A252F823F0F18A000041
:107D0000C38A00006D4E00008F8A00006D4E000097
:107D10006D4E00006D4E0000618A0000634D2A78B0
:107D2000002A00F0B2812368DFF88C8162935B4AFD
:107D3000629BD8F8000012681B1A934211D9524B6B
:107D40001A78012A16BF012219701A701878FBF7E9
:107D5000D5FA4E4804F0AAFE23686393639BC8F8E3
:107D600000304F4A1378002B3DF480A84D4B1B6820
:107D70000021013B1170072B3DF678A801A252F8B3
:107D800023F000BF8D9300005B9300006D4E000058
:107D9000299300006D4E00006D4E00006D4E0000F6
:107DA000F7920000FBF7C0FD414A0121002311704A
:107DB000337007E55E1A5C2303FB06F393FBF2F6D0
:107DC0001B36FDF7BDBF5E1A5C2303FB06F393FB76
:107DD000F2F61B36FEF707B85E1A5C2303FB06F3C8
:107DE00093FBF2F61B36FEF7B9BD324D2978002918
:107DF00000F0FE802368DFF8C08092932749929BB1
:107E0000D8F8000009681B1A8B4210D91E4B19784C
:107E1000012918BF01221A701878F8F715FE1B48BF
:107E200004F044FE23689393939BC8F800301C4AE7
:107E30001378002B3DF41AA81A4B1B680021013B54
:107E40001170072B3DF612A801A252F823F000BFD3
:107E50006D940000239400006D4E0000ED9300002F
:107E60006D4E00006D4E00006D4E0000BF9300008F
:107E70005E1A5C2303FB06F393FBF2F61B36FEF758
:107E8000C3BD00BFDE9EFF1F889EFF1F009FFF1F18
:107E9000EA9EFF1F588CFF1F5A9DFF1F908DFF1FEA
:107EA000F49DFF1F8C9EFF1F449EFF1FD09EFF1F4F
:107EB000679DFF1F009EFF1F389EFF1FB94D297849
:107EC00000293DD02368DFF804837C93B6497C9B6E
:107ED000D8F8000009681B1A8B4210D9B34B1978E7
:107EE000012918BF01221A701878FAF71BFEB04852
:107EF00004F0DCFD23687D937D9BC8F80030AD4A1B
:107F00001378002B3CF4B2AFAB4B1B680021013B54
:107F10001170072B3CF6AAAF01A252F823F000BF64
:107F200055860000278600006D4E0000F185000098
:107F30006D4E00006D4E00006D4E0000C3850000C8
:107F40009E4D2A78002A00F01D872368DFF87C8286
:107F50008093954A809BD8F8000012681B1A9342C0
:107F600011D9924B1A78012A16BF012219701A7082
:107F70001878FCF7FFFA8E4804F098FD2368819387
:107F8000819BC8F800308B4A1378002B3CF46EAF0D
:107F9000894B1B680021013B1170072B3CF666AF33
:107FA00001A252F823F000BF1B870000ED860000FD
:107FB0006D4E0000B98600006D4E00006D4E000051
:107FC0006D4E00008B8600005E1A5C2303FB06F3F7
:107FD00093FBF2F61B36FEF754BFFAF7CDFF0023F2
:107FE000337058E6FAF7EAFF00233370FCF782BFDC
:107FF000734D2A78002A00F005862368DFF8CC81CB
:108000009693694A969BD8F8000012681B1A93420F
:1080100011D9664B1A78012A16BF012219701A70FD
:108020001878F8F72FFD624804F040FD2368979315
:10803000979BC8F800305F4A1378002B3CF416AFCA
:108040005D4B1B680021013B1170072B3CF60EAF06
:1080500001A252F823F000BF998B00006B8B000047
:108060006D4E0000C98B00006D4E00006D4E00008B
:108070006D4E00003D8B00005E1A5C2303FB06F38F
:1080800093FBF2F61B36FEF76BBF4E4D29780029A5
:108090003CD02368DFF8348166934349669BD8F867
:1080A000000009681B1A8B4210D9404B197801292E
:1080B00018BF01221A701878FAF76CFC3C4804F0DB
:1080C000F5FC23686793679BC8F80030394A13783A
:1080D000002B3CF4CBAE384B1B680021013B1170E8
:1080E000072B3CF6C3AE01A252F823F0C388000070
:1080F0005B8800006D4E0000898800006D4E000016
:108100006D4E00006D4E00004F8700002E4D2A7806
:10811000002A66D02368DFF8B4806A93224A6A9BFB
:10812000D8F8000012681B1A934211D91F4B1A7815
:10813000012A16BF012219701A701878FCF776FC14
:108140001B4804F0B3FC23686B936B9BC8F80030AA
:10815000184A1378002B3CF489AE174B1B6800219A
:10816000013B1170072B3CF681AE01A252F823F0BF
:1081700029880000DF8700006D4E0000AB870000FB
:108180006D4E00006D4E00006D4E00007D870000BA
:108190005E1A5C2303FB06F393FBF2F61B36FEF735
:1081A00082BF00BF589DFF1F908DFF1F889EFF1F3D
:1081B000009FFF1FF49DFF1F8C9EFF1F649DFF1FEC
:1081C000DC9DFF1F8C9DFF1F2B9FFF1F389EFF1FF5
:1081D0005E1A5C2303FB06F393FBF2F61B36FEF7F5
:1081E000B8BFBA4D297800293CD02368DFF8008356
:1081F0006E93B7496E9BD8F8000009681B1A8B4232
:1082000010D9B44B1978012918BF01221A701878B7
:10821000FBF7AEFAB04804F049FC23686F936F9BFC
:10822000C8F80030AD4A1378002B3CF41FAEAC4BBD
:108230001B680021013B1170072B3CF617AE01A211
:1082400052F823F051850000238500006D4E000098
:10825000838500006D4E00006D4E00006D4E0000E5
:10826000F58400009F4D23682A78DFF88482002A75
:108270003AD07293964A729BD8F8000012681B1A83
:10828000934211D9934B1A78012A16BF0122197013
:108290001A701878FAF7B8FC8F4804F007FC2368C6
:1082A0007393739BC8F800308C4A1378002B3CF40E
:1082B000DDAD8B4B1B680021013B1170072B3CF699
:1082C000D5AD01A252F823F0998400006B84000020
:1082D0006D4E0000378400006D4E00006D4E0000B2
:1082E0006D4E00000984000076937949769BD8F89A
:1082F000000009681B1A8B4212D9764B19780129A4
:1083000018BF01221A70784A19781078F8F766FBBE
:10831000714804F0CBFB23687793779BC8F8003053
:108320006E4A1378002B3CF4A1AD6D4B1B68002105
:10833000013B1170072B3CF699AD01A252F823F0D6
:10834000C7830000BF8300006D4E00007D830000E6
:108350006D4E00006D4E00006D4E000073830000F6
:108360005E1A5C2303FB06F393FBF2F61B36FFF762
:10837000B6B901233B703370FCF778BD5A4C2078B6
:1083800001287CF673AD0021F8F728FB2378514DC6
:10839000013BDBB2184601212370F8F71FFB0024D4
:1083A00034238DE818004C482C7040230B223F21C9
:1083B00003F05EFB484804F079FBFCF757BDFCF77F
:1083C00011FCFCF753BD484C207805283CF64EAD17
:1083D0000021F8F703FB23783E4D0133DBB218464A
:1083E00001212370F8F7FAFA002434238DE81800ED
:1083F00039482C7040230B223F2103F039FB3648CB
:1084000004F054FBFCF732BD0120FAF7FDFB314BC1
:10841000314800241C7004F049FB30202C70F8F720
:1084200079FB324B198888423CF420AD3020F8F7B4
:1084300065FBFCF71BBD0020FAF7E6FB2B4A13880F
:10844000082B94BF0133002301201380FAF7DCFBD3
:10845000204B214800221A7004F028FB23687593F2
:10846000759BC8F80030FCF701BD0120FAF7CCFB82
:10847000184B194800241C7004F018FB30202C7095
:10848000F8F748FB194B198888423CF4EFAC3020D0
:10849000F8F734FBFCF7EABC0020FAF7B5FB134A07
:1084A0001388002B00F08780013B13800120FAF72E
:1084B000ABFB084B084800221A7004F0F7FA236857
:1084C0007493749BC8F80030FCF7D0BCB69DFF1FB6
:1084D000908DFF1F889EFF1F009FFF1FF49DFF1FB1
:1084E0008C9EFF1FEC9DFF1F648AFF1FA29DFF1F34
:1084F000389EFF1F0120FBF73BF9C44BC448002402
:108500001C7004F0D3FA2E202C70F8F703FBC14B3B
:10851000198888423CF4AAAC2E20F8F7EFFAFCF751
:10852000A5BC0120FBF724F9B84BB94800241C7006
:1085300004F0BCFA2E202C70F8F7ECFAB54B198831
:1085400088423CF493AC2E20F8F7D8FAFCF78EBCA6
:108550000020FBF70DF9AF4A1388002B2ED0013B0A
:1085600013800120FBF704F9A84BA94800221A70D8
:1085700004F09CFA23687093709BC8F80030FCF7F5
:1085800075BC0020FBF7F4F8A24A13881D2B94BF9A
:108590000133002301201380FBF7EAF89B4B9C4832
:1085A00000221A7004F082FA23687193719BC8F854
:1085B0000030FCF75BBC0923138077E71E23138090
:1085C000CFE70120FAF7AEFA904B914800241C70D7
:1085D00004F06CFA1A202C70F8F79CFA8E4B19886C
:1085E00088423CF443AC1A20F8F788FAFCF73EBC0A
:1085F000894D2B880B2B3CF639AC0020FAF792FA08
:108600002B88012003442B80FAF78CFA7F4B80489B
:1086100000221A7004F04AFA23687F937F9BC8F8FF
:108620000030FCF723BC0120FAF77CFA774B78483E
:1086300000241C7004F03AFA1A202C70F8F76AFA39
:10864000754B198888423CF411AC1A20F8F756FA99
:10865000FCF70CBC704D2B88002B3CF407AC0020C1
:10866000FAF760FA2B880120013B2B80FAF75AFABF
:10867000664B674800221A7004F018FA23687E934C
:108680007E9BC8F80030FCF7F1BB0120FBF772FFBE
:108690005E4B5F4800241C7004F008FA1C202C700C
:1086A000F8F738FA5D4B198888423CF4DFAB1C20A0
:1086B000F8F724FAFCF7DABB0020FBF75BFF574A18
:1086C0001388032B94BF0133002301201380FBF791
:1086D00051FF4E4B4E4800221A7004F0E7F9236810
:1086E0008393839BC8F80030FCF7C0BB0120FBF7E5
:1086F00041FF464B464800241C7004F0D7F91C206B
:108700002C70F8F707FA454B198888423CF4AEAB59
:108710001C20F8F7F3F9FCF7A9BB0020FBF72AFFB0
:108720003E4A1388002B00F0C980013B13800120D2
:10873000FBF720FF354B364800221A7004F0B6F9DB
:1087400023688293829BC8F80030FCF78FBB01201E
:10875000FAF720F92D4B2E4800241C7004F0A6F9DE
:1087600016202C70F8F7D6F92D4B198888423CF466
:108770007DAB1620F8F7C2F9FCF778BB0120FCF7B7
:1087800055F9224B224800241C7004F08FF92C204C
:108790002C70F8F7BFF9234B198888423CF466AB7C
:1087A0002C20F8F7ABF9FCF761BB0020FCF73EF991
:1087B0001C4A13880B2B94BF013300230120138024
:1087C000FCF734F9114B124800221A7004F06EF9CC
:1087D00023686D936D9BC8F80030FCF747BB012000
:1087E000FCF724F9094B0A4800241C7004F05EF9D8
:1087F0002C202C70F8F78EF90A4B198888423CF42B
:1088000035AB2C20F8F77AF9FCF730BB889EFF1FB8
:10881000009FFF1FB89EFF1FCC9DFF1FC49DFF1F21
:108820005C9DFF1F989EFF1F0020FCF7FFF8BD4ACC
:108830001388002B5DD0013B13800120FCF7F6F874
:10884000B94BBA4800221A7004F030F923686C93CF
:108850006C9BC8F80030FCF709BB0120FAF79AF8C6
:10886000B14BB24800241C7004F020F916202C7083
:10887000F8F750F9AE4B198888423CF4F7AA162055
:10888000F8F73CF9FCF7F2BA0020FAF783F8A84AA7
:1088900013887E2B94BF0133002301201380FAF745
:1088A00079F8A14BA14800221A7004F0FFF8236860
:1088B0006993699BC8F80030FCF7D8BA0423138089
:1088C00035E70020FAF766F8994A1388A3B1013B0F
:1088D00013800120FAF75EF8934B944800221A7037
:1088E00004F0E4F823686893689BC8F80030FCF74C
:1088F000BDBA0C231380A0E77F231380E9E75E1A3B
:108900005C2303FB06F393FBF2F61B36FEF7D7BDA1
:108910005E1A5C2303FB06F393FBF2F61B36FFF7AC
:108920009BB85E1A5C2303FB06F393FBF2F61B363F
:10893000FEF73ABE5E1A5C2303FB06F393FBF2F6E6
:108940001B36FEF722BF0120FBF7A8FF764B7748C6
:1089500000241C7004F0AAF812202C70F8F7DAF842
:10896000744B198888423CF481AA1220F8F7C6F8A3
:10897000F8F774FCFCF77ABA6E4D2B88092B4FF090
:10898000000046D8FBF78AFF2B88012003442B8088
:10899000FBF784FF644B654800221A7004F086F8E8
:1089A00023686093609BC8F80030FCF75FBA012031
:1089B000FBF774FF5C4B5D4800241C7004F076F8F4
:1089C00012202C70F8F7A6F85A4B198888423CF40C
:1089D0004DAA1220F8F792F8F8F740FCFCF746BAD7
:1089E000544D2E8846B30020FBF758FF2B880120FA
:1089F000013B2B80FBF752FF4B4B4C4800221A7077
:108A000004F054F823685E935E9BC8F80030FCF7CE
:108A10002DBAFBF743FF002601202E80FBF73EFF17
:108A2000414B42481E7004F041F823686193619BFA
:108A3000C8F80030FCF71ABA3046FBF72FFF0A23BC
:108A400001202B80FBF72AFF374B38481E7004F0BB
:108A50002DF823685F935F9BC8F80030FCF706BAD7
:108A60000120FBF723FD304B304800241C7004F03C
:108A70001DF818202C70F8F74DF82F4B19888842F4
:108A80003CF4F4A91820F8F739F8FCF7EFB9002006
:108A9000FBF70CFD284A1388012B94BF01330023F8
:108AA00001201380FBF702FD1F4B204800221A70A3
:108AB00003F0FCFF23687B937B9BC8F80030FCF736
:108AC000D5B90120FBF7F2FC174B184800241C70A5
:108AD00003F0ECFF18202C70F8F71CF8164B1988DF
:108AE00088423CF4C3A91820F8F708F8FCF7BEB98F
:108AF0000020FBF7DBFC104A1388002B7FD0013BE2
:108B000013800120FBF7D2FC074B084800221A70A3
:108B100003F0CCFF23687A937A9BC8F80030FCF707
:108B2000A5B900BF989EFF1F889EFF1F009FFF1FD3
:108B30005C9DFF1F909EFF1F209EFF1F0120F7F7E7
:108B4000A1FFB14BB14800241C7003F0AFFF5220CD
:108B50002C70F7F7DFFFAE4B198888423CF486A9EA
:108B60005220F7F7CBFFFCF781B90120F7F78AFF16
:108B7000A54BA64800241C7003F098FF52202C70CF
:108B8000F7F7C8FFA24B198888423CF46FA952201E
:108B9000F7F7B4FFFCF76AB90020F7F773FF9C4AB8
:108BA00013880BB1013B13800120F7F76BFF964B45
:108BB000964800221A7003F079FF23689893989BD7
:108BC000C8F80030FCF752B90020F7F75BFF904A75
:108BD0001388032B98BF01334FF0010098BF138017
:108BE000F7F750FF884B894800221A7003F05EFFA8
:108BF00023689993999BC8F80030FCF737B9022392
:108C000013807EE7834D297800293DD02368DFF863
:108C100020829A9380499A9BD8F8000009681B1A11
:108C20008B4210D9784B1978012918BF01221A708C
:108C30001878F7F745FF754803F038FF23689B93D2
:108C40009B9BC8F80030754A1378002B3CF40EA9A2
:108C5000734B1B680021013B1170072B3CF606A9E2
:108C600001A252F823F000BFFD950000CF9500004F
:108C70006D4E0000999500006D4E00006D4E000095
:108C80006D4E00006B950000664D23682A78DFF872
:108C9000A081002A3AD09E935F4A9E9BD8F800009C
:108CA00012681B1A934211D9574B1A78012A16BF22
:108CB000012219701A701878FAF77EFB534803F0F6
:108CC000F5FE23689F939F9BC8F80030534A1378A2
:108CD000002B3CF4CBA8524B1B680021013B1170C8
:108CE000072B3CF6C3A801A252F823F0C59200005E
:108CF000979200006D4E0000659200006D4E0000DE
:108D00006D4E00006D4E000037920000A293424964
:108D1000A29BD8F8000009681B1A8B4212D93A4B63
:108D20001978012918BF01221A703F4A1978107862
:108D3000F7F754FE354803F0B9FE2368A393A39BCD
:108D4000C8F80030354A1378002B3CF48FA8344B18
:108D50001B680021013B1170072B3CF687A801A27C
:108D600052F823F0D5910000CD9100006D4E000027
:108D70008B9100006D4E00006D4E00006D4E0000A6
:108D80007F910000294D2978002953D02368DFF80E
:108D9000A08084932049849BD8F8000009681B1A9E
:108DA0008B4210D9184B1978012918BF01221A706B
:108DB0001878FAF74BFD154803F078FE2368859381
:108DC000859BC8F80030154A1378002B3CF44EA858
:108DD000134B1B680021013B1170072B3CF646A882
:108DE00001A252F823F000BF49910000F390000067
:108DF0006D4E0000BD9000006D4E00006D4E0000F5
:108E00006D4E00008F900000889EFF1F009FFF1F87
:108E1000948AFF1FDC9EFF1F908DFF1FF49DFF1F94
:108E20008C9EFF1FDD9EFF1F488AFF1FC19DFF1FF5
:108E3000389EFF1FBA4D23682A78DFF80883002A7E
:108E40003AD08893B74A889BD8F8000012681B1A5A
:108E5000934211D9B44B1A78012A16BF0122197016
:108E60001A701878FBF7ACFAB04803F01FFE2368BD
:108E70008993899BC8F80030AD4A1378002B3BF4E6
:108E8000F5AFAC4B1B680021013B1170072B3BF683
:108E9000EDAF01A252F823F0599000002B90000092
:108EA0006D4E00005F8F00006D4E00006D4E0000A3
:108EB0006D4E0000318F00008C939A498C9BD8F83E
:108EC000000009681B1A8B4212D9974B19780129A7
:108ED00018BF01221A70984A19781078F7F77EFDAA
:108EE000924803F0E3FD23688D938D9BC8F8003012
:108EF0008F4A1378002B3BF4B9AF8E4B1B680021CF
:108F0000013B1170072B3BF6B1AF01A252F823F0E1
:108F1000E98F0000E18F00006D4E00009F8F000080
:108F20006D4E00006D4E00006D4E0000958F0000EC
:108F30000120FBF745FA7C4B7C4800241C7003F0B1
:108F4000B5FD32202C70F7F7E5FD7C4B198888427F
:108F50003BF48CAF3220F7F7D1FDFBF787BF774D9D
:108F60002B88172B3BF682AF0020FBF729FA2B88C2
:108F7000012003442B80FBF723FA6B4B6B48002244
:108F80001A7003F093FD23688B938B9BC8F8003015
:108F9000FBF76CBF01233B703370FBF767BF664C78
:108FA000207801287BF662AF0021F7F717FD2378C0
:108FB0005D4D013BDBB2184601212370F7F70EFD32
:108FC000002434238DE8180058482C7040230B22CD
:108FD0003F2102F04DFD554803F068FDFBF746BF09
:108FE000FBF756FBFBF742BF534C207805283BF6B6
:108FF0003DAF0021F7F7F2FC23784B4D0133DBB294
:10900000184601212370F7F7E9FC002434238DE88A
:10901000180046482C7040230B223F2102F028FD07
:10902000424803F043FDFBF721BF0120FBF7C8F9DD
:109030003D4B3E4800241C7003F038FD32202C705C
:10904000F7F768FD3D4B198888423BF40FAF32209B
:10905000F7F754FDFBF70ABF384D2B88002B3BF484
:1090600005AF0020FBF7ACF92B880120013B2B80DA
:10907000FBF7A6F92C4B2D4800221A7003F016FDC1
:1090800023688A938A9BC8F80030FBF7EFBE012063
:10909000FAF7DCFB244B254800241C7003F006FD86
:1090A00020202C70F7F736FD254B198888423BF4B9
:1090B000DDAE2020F7F722FDFBF7D8BE204D2B8830
:1090C000452B3BF6D3AE0020FAF7C0FB2B880120DE
:1090D00003442B80FAF7BAFB134B144800221A7092
:1090E00003F0E4FC23688793879BC8F80030FBF704
:1090F000BDBE0120FAF7AAFB0B4B0C4800241C70E4
:1091000003F0D4FC20202C70F7F704FD0C4B1988D9
:1091100088423BF4ABAE2020F7F7F0FCFBF7A6BE8D
:10912000969DFF1F908DFF1F889EFF1F009FFF1FB2
:10913000F49DFF1F8C9EFF1F548AFF1FCA9EFF1FB6
:10914000DA9EFF1F389EFF1FC14D2B88002B3BF47A
:109150008DAE0020FAF77AFB2B880120013B2B8093
:10916000FAF774FBBB4BBC4800221A7003F09EFC5C
:1091700023688693869BC8F80030FBF777BE5A2297
:1091800001233A703370FBF771BEB44C207801288C
:109190007BF66CAE0021F7F721FC2378AD4D013B47
:1091A000DBB2184601212370F7F718FC00243423A2
:1091B0008DE81800A8482C7040230B223F2102F0B4
:1091C00057FCA54803F072FCFBF750BEFAF752F9C2
:1091D000FBF74CBEA14C207804283BF647AE00219B
:1091E000F7F7FCFB23789B4D0133DBB218460121D6
:1091F0002370F7F7F3FB002434238DE8180096481A
:109200002C7040230B223F2102F032FC924803F0E5
:109210004DFCFBF72BBE5E1A5C2303FB06F393FBAE
:10922000F2F61B36FEF785BC02FB03F393FBF5F267
:109230001144FEF75FBC0120FAF7BEF8854B864863
:1092400000241C7003F032FC56202C70F7F762FCEF
:10925000834B198888423BF409AE5620F7F74EFC41
:10926000FBF704BE0020FAF7A7F87D4A1388B3FA8B
:1092700083F35B0901201380FAF79EF8754B76485B
:1092800000221A7003F012FC2368A193A19BC8F876
:109290000030FBF7EBBD0120FAF78EF86D4B6E48FE
:1092A00000241C7003F002FC56202C70F7F732FCEF
:1092B0006B4B198888423BF4D9AD5620F7F71EFC5A
:1092C000FBF7D4BD0020FAF777F8654A1388B3FAA4
:1092D00083F35B0901201380FAF76EF85D4B5E485B
:1092E00000221A7003F0E2FB2368A093A09BC8F849
:1092F0000030FBF7BBBD0120FAF700F8554B56488C
:1093000000241C7003F0D2FB14202C70F7F702FC31
:10931000544B198888423BF4A9AD1420F7F7EEFBB3
:10932000F7F79CFFFBF7A2BD0020F9F7E7FF4D4AD6
:109330001388B3FA83F35B0901201380F9F7DEFF8A
:10934000444B454800221A7003F0B0FB2368659334
:10935000659BC8F80030FBF789BD0120F9F7CEFF07
:109360003C4B3D4800241C7003F0A0FB14202C70E3
:10937000F7F7D0FB3B4B198888423BF477AD1420BC
:10938000F7F7BCFBF7F76AFFFBF770BD0020F9F7B2
:10939000B5FF344A1388B3FA83F35B0901201380C5
:1093A000F9F7ACFF2B4B2C4800221A7003F07EFB20
:1093B00023686493649BC8F80030FBF757BD012015
:1093C000F7F742FB234B244800241C7003F06EFB8C
:1093D00050202C70F7F79EFB234B198888423BF4F2
:1093E00045AD5020F7F78AFBFBF740BD1E4D2B889B
:1093F0000B2B3BF63BAD0020F7F726FB2B8801201B
:1094000003442B80F7F720FB124B134800221A70FD
:1094100003F04CFB23689593959BC8F80030FBF74D
:1094200025BD0120F7F710FB0A4B0B4800241C70E8
:1094300003F03CFB50202C70F7F76CFB0A4B1988AB
:1094400088423BF413AD5020F7F758FBFBF70EBDF5
:10945000DA9EFF1F889EFF1F009FFF1F488AFF1F85
:10946000F69DFF1F129EFF1FB88CFF1F714D2B88AA
:10947000012B7BF6FBAC0020F7F7E6FA2B880120E6
:10948000013B2B80F7F7E0FA6B4B6C4800221A7017
:1094900003F00CFB23689493949BC8F80030FBF70F
:1094A000E5BC0120F9F7D8FA634B644800241C702E
:1094B00003F0FCFA1E202C70F7F72CFB604B198888
:1094C00088423BF4D3AC1E20F7F718FBFBF7CEBC69
:1094D0005B4D2B88082B3BF6C9AC0020F9F7BCFA92
:1094E0002B88012003442B80F9F7B6FA524B5348DE
:1094F00000221A7003F0DAFA23689193919BC8F85E
:109500000030FBF7B3BC0120F9F7A6FA4A4B4B48F1
:1095100000241C7003F0CAFA1E202C70F7F7FAFA28
:10952000474B198888423BF4A1AC1E20F7F7E6FAB6
:10953000FBF79CBC424D2B88002B3BF497AC0020E2
:10954000F9F78AFA2B880120013B2B80F9F784FA7E
:10955000394B3A4800221A7003F0A8FA2368909316
:10956000909BC8F80030FBF781BC0120F7F7A8FA00
:10957000314B324800241C7003F098FA54202C70B0
:10958000F7F7C8FA2F4B198888423BF46FAC542088
:10959000F7F7B4FAFBF76ABC2A4D2B881D2B3BF674
:1095A00065AC0020F7F78CFA2B88012003442B8050
:1095B000F7F786FA204B214800221A7003F076FA5A
:1095C00023689D939D9BC8F80030FBF74FBC01209A
:1095D000F7F776FA184B194800241C7003F066FA66
:1095E00054202C70F7F796FA164B198888423BF4F2
:1095F0003DAC5420F7F782FAFBF738BC114D2B88AD
:10960000012B7BF633AC0020F7F75AFA2B880120A8
:10961000013B2B80F7F754FA074B084800221A70D9
:1096200003F044FA23689C939C9BC8F80030FBF736
:109630001DBC00BFB88CFF1F889EFF1F009FFF1F2F
:10964000B89DFF1FBA8CFF1F2DE9F04F0E2093B07D
:1096500003F0A4FC07F082F90146AC48AC4FAD4ED4
:1096600002F0B8F8A94802F08BF807F0A7FB3D68B4
:1096700080F30C00012D306000F08380022DDFF8B4
:1096800004B300F08F81032D00F00D82A24CA34D96
:10969000DFF8F492DFF8F4822368A14F0E930E9B5B
:1096A0003A689B1A022B1ED9DFF8E4A29AF8003020
:1096B000002B00F0BC829B4B1A78002A0CBF0122C1
:1096C00000221A7000F0B6829AF80030002B40F0A9
:1096D000B682F7F7C1FEF6F7F1FFF7F7DBFD236877
:1096E0000F930F9B3B6023688F4F10938F4A109B03
:1096F000396812685B1A93422BD83368BBF80000B4
:109700002A68C9F800208342B8F800201ADA00233A
:10971000101AB0F5805FA6BF1B030130C3EB033303
:1097200093FBF0F0F6F7DCFE0146282004F0D2F8B7
:10973000002005F0C7FA0028FAD1FBF7F1FA13B0C0
:10974000BDE8F08F9342D4BFC0EB0303C0EB02032C
:10975000DEE7F8F791F8764B1B7823B9754B1B7849
:10976000002B00F0F5810D2004F04AFAB0FA80F1E8
:1097700049090D2004F03EFA23681193119B3B60C8
:10978000BBE7DFF810926C4AB9F8003011789942C3
:1097900009D0DBB21370002B00F00C82102BA8BF95
:1097A0001023664A1360DFF8F081654AB8F800308C
:1097B0001178994204D0634C2178002940F0EA8165
:1097C000DFF8C0B1544CBBF80030834280F2BA815C
:1097D00022685D4B099209995C4A19600223106066
:1097E0003B605B4B187838BB5A4B1B7823BB5A4BFA
:1097F0001F68002003F0D2FBA7F21F37874202DC6C
:10980000564B00221A70002004F022FC544B554D98
:109810001A682978544F9042D4BF002301238B4209
:109820003B7002D0904200F33C832B70DFF85891DC
:109830003A4DDFF858812FE74C4BDFF860A11F88C5
:10984000BAF80020DFF858E11744DEF800207F1056
:109850009742474A05DA11688F4202DA002840F041
:10986000568302933C4B01921F460020CDF80CE03A
:10987000009303F093FB3F68019A029BA7F5487E93
:10988000704580F2998133480078002800F0948177
:109890001888DDF80CE0BAF80030DEF80010126825
:1098A00003445B108B4280F28D81934240F38A81A6
:1098B000F6F766FF2F490A68531C002B40F34185D9
:1098C000802B00F33D852C4D2C482F882C4D008893
:1098D0002D680B603918B5EB610FC1F24580A2F11C
:1098E00048030F2B00F2A081473A00210D20A9F870
:1098F000002004F07FF9962004F0B8F901210D2032
:1099000004F078F9009B1F6873E700BF689EFF1F93
:10991000C49EFF1FAC9EFF1F3C9FFF1FF49EFF1FB6
:10992000409EFF1FC09DFF1F049EFF1FF88BFF1F5F
:10993000B09EFF1FA59EFF1F2F9EFF1FFC9DFF1FB8
:10994000EE9DFF1F959DFF1FE89DFF1F5C9EFF1F63
:10995000BA9DFF1F149EFF1F6C9DFF1FD99EFF1F06
:10996000548CFF1F599DFF1FB79DFF1FB49DFF1F04
:10997000FC9EFF1FF09DFF1F8E9DFF1F469EFF1F39
:10998000BC9DFF1F169EFF1F1C9EFF1FE89EFF1F12
:10999000DE9EFF1F589EFF1F649EFF1F2C9EFF1F11
:1099A000C89DFF1FBBF80030984240F3EB80A54CE8
:1099B000A54923680A93A54A0A9B096812885B1A7D
:1099C000934202D8002A7FF462AEF6F7D9FEA04A8D
:1099D00033681168BBF80020DFF8C4828B42B8BF3F
:1099E0000B469342B8F800009A4980F2C2859A4B20
:1099F00009881A60002900F0FF82984B04931970BF
:109A0000974DF7F7C3FC28687F2840F3AE85954B48
:109A10007F3883FB0032C317C3EB620303EB4303BE
:109A2000A0EB83007330904B01931B882860002BC0
:109A300040F041878D4B00931B78002B00F0B383DF
:109A40008B4B1A461B78002B00F0AD830294CDF8A7
:109A50000C80DFF82492049CA8464FF0000A1546BB
:109A60000BE003F17300C0B22178F7F777FE2B7893
:109A70000AF1010A534540F39283D8F8003059F8AF
:109A8000040F784A1844A0F17F0382FB032ED917F4
:109A9000C1EB6E0101EB41017F28A3EB8103E0DC08
:109AA000F6F70CFDDFE7BBF80030984280F2FC804F
:109AB000704B1B78002B40F0F780DFF8E8A19AF894
:109AC00000007F2800F38882F6F7F8FC664B0193CC
:109AD0001B88C0B28AF80000002B40F0C986634B97
:109AE00000931B78002B00F0C682614B1A461B784E
:109AF000002B00F0C082604C5A4D4FF00008914698
:109B00000BE003F17300C0B2F7F736F899F80030B4
:109B100008F10108434540F3AE8254F8043F9AF837
:109B200000001844A0F17F0385FB0321DA17C2EB84
:109B3000610202EB42027F28A3EB8203E1DCF6F72D
:109B4000BDFCE0E74B4B1B78002B3FF44AAE3FE6F1
:109B5000464B1B78002B7FF406AE484B1B78002B3E
:109B60007FF401AE434B1B78002B7FF4FCAD0D203E
:109B700004F046F800287FF4FFAD01210D2004F029
:109B800039F8F9E53B4B1B78002B7FF410AF01232C
:109B90003B607BE5DBB218461370F6F7CBFF334B27
:109BA000374A3068194600231370344A23700B700B
:109BB000137005E62B46F4E51988BAF800301268F0
:109BC0000B445B109342BFF614AE002003F0E6F99D
:109BD000009B1F68A7F548739842BFF60AAE294B51
:109BE0001A78002A7FF405AE274F01251D70F6F77D
:109BF000C7FD3B78002B40F00885244B1B78002BD9
:109C000000F0BD86224B1B78002B00F03A87214BD9
:109C10001B784BB9204B1B7833B1B8F800301F4A82
:109C20000A3BA8F800301570009B1F68E1E5F7F7C4
:109C3000ADFB40E5F7F730F8F7F746FD4FE5F7F7EE
:109C4000A5FB46E53C9FFF1FE89DFF1FB89EFF1F39
:109C50005C9EFF1F5C9DFF1FD49EFF1FF89DFF1F92
:109C6000F49EFF1FABAAAA2AC29DFF1FDF9EFF1F03
:109C7000008BFF1FA09DFF1FD88AFF1F5B9DFF1F4A
:109C8000A59EFF1FD99EFF1F3C9EFF1FC09EFF1F6A
:109C9000289FFF1F299FFF1F2A9FFF1F959DFF1FC2
:109CA000E89EFF1FA49EFF1FB14DDFF82093F6F73B
:109CB00067FD2868D9F80030984200F04B84AD4C1D
:109CC000AD4B22680B920B9A1A6023680C93AB4938
:109CD0000C9B09889B1A8B4240F2D4807F2840F36A
:109CE0004084A74B7F3883FB0032C317C3EB62036A
:109CF00003EB4303A0EB83007330DFF8D4A29AF8A0
:109D00000070874200F0BE809E4B1988002900F049
:109D1000B884DFF8C0827F2F40F383859848A7F18D
:109D20007F0280FB0230D317C3EB600000EB4000E2
:109D3000A2EB80007330944B00931B78C0B28AF87A
:109D40000000002B40F0E284904B03931B78002B23
:109D500040F04C868E4B02931B78002B40F0B78668
:109D60008C4B0193029B1B7883B38B4B9AF80000BA
:109D70001B6818447F2840F35586814B7F3883FB4E
:109D80000032C317C3EB620303EB4303A0EB830072
:109D90007330C0B2F6F7F0FE804A814B12789AF821
:109DA000000053F8223018447F2840F33786744B64
:109DB0007F3883FB0032C317C3EB620303EB43031B
:109DC000A0EB83007330C0B2F6F7D6FE009B1B7881
:109DD000002B00F07785019B6E4F1B880493002BAE
:109DE00000F00D8628687F2840F31785644B7F3884
:109DF00083FB0032C317C3EB620303EB4303A0EB07
:109E000083007330049B2860002B40F0D085009BBA
:109E10001B78002B00F0C482624B1A461B78002B83
:109E200000F0BE82604B614904940027CDF814A075
:109E3000CDF818801C46B8468A462F4615460CE0D9
:109E400003F17300C0B29AF80010F7F787FC2B7883
:109E500008F10108434540F39D823B6854F8040F24
:109E6000474A1844A0F17F0382FB032ED917C1EBA8
:109E70006E0101EB41017F28A3EB8103E0DCF6F7E3
:109E80001DFBDFE7DFF84C81BBF8002033689A4206
:109E9000BFF602AC23680D93454B0D9A1A60FFF78D
:109EA000FBBBF6F76DFC434B1978002932D1424BCE
:109EB0001B7843B1344A00921278002A00F0DC8407
:109EC0000098002202703D4A1278002A00F0258393
:109ED0002E4B039319461B78002B40F0C484384A5C
:109EE0002B4812780370012302900B70002A00F0B7
:109EF0002E83254B334A009300211170009A3B7842
:109F00001170029F039A0120387011708DE42E4B5E
:109F10000093CDE42B4A92F800C0BCF1000F40F052
:109F2000BC84194800901A48234B029016481B78AD
:109F300080F800C016484FF0010E80F800C082F88B
:109F400000E0002B40F09B841C4B1B78002BBFD102
:109F50001B4B1B78002B00F0FA820D4B02931B78F1
:109F6000002B00F0F88502993B7800220A705CE42F
:109F7000F49EFF1F3C9FFF1F609EFF1FDA9EFF1F86
:109F8000ABAAAA2A5C9DFF1FDF9EFF1F5B9DFF1FE0
:109F9000B09EFF1FC29DFF1F048BFF1FF99DFF1F77
:109FA000448CFF1F008BFF1FD88AFF1FF89DFF1FE7
:109FB000389EFF1F2A9FFF1FD19EFF1FC09EFF1FBD
:109FC000949DFF1FA59EFF1F6C9DFF1F1C9EFF1FE2
:109FD000A49EFF1FE89EFF1FA3F155337F3803F1B6
:109FE000004383FB0032C317C3EB620303EB43035D
:109FF000A0EB8300733069E513468342D4BFC2EB04
:10A000000303C2EB0003821AB2F5804FAABF9B0381
:10A01000C3EB8333013293FBF2F0F6F761FAC0F33E
:10A02000C61006F09BFCB34B0546188806F096FC5C
:10A03000B1498146284606F0E5FC0146484606F04F
:10A04000E1FC294606F0D6FB4FF07E51054606F0AE
:10A0500077FE002840F01285A849284606F08EFEBB
:10A06000002840F00685284606F0CEFEC0B2A44B7C
:10A0700004931870C4E4A34B1B78002B45D09AF8C6
:10A080000030A3F10C007F2840F311849E4A8B3BE3
:10A0900082FB0321DA17C2EB610202EB4202A3EB5F
:10A0A000820303F17300C0B2F6F766FD009B1B78D4
:10A0B0005BB3964B1A461B783BB3954C924D4FF0D1
:10A0C000000891460AE003F17300C0B2F6F754FDB0
:10A0D00099F8003008F10108434516DD54F8043FB3
:10A0E0009AF800201A44A2F18B0385FB0310D917BC
:10A0F000C1EB6001A2F10C0001EB41017F28A3EB51
:10A100008103E0DCF6F7DAF9DFE7824B1B7883B3F3
:10A11000814B9AF800001B6818447F2840F3C483E1
:10A12000794B7F3883FB0032C317C3EB620303EB29
:10A130004303A0EB83007330C0B2F6F71DFD774AEE
:10A14000774B12789AF8000053F8223018447F2891
:10A1500040F3A7836C4B7F3883FB0032C317C3EBFC
:10A16000620303EB4303A0EB83007330C0B2F6F746
:10A1700003FD019B1B88002B00F07083694B1B784B
:10A18000002B40F06683684B684C694DDFF8A8915E
:10A19000DFF8A88100221A6001233B6074E645467F
:10A1A000029CDDF80C805F4B1B78002B40F0D183C4
:10A1B0002A68544B1B78002B51D0A2F10C007F2849
:10A1C00040F3DA835049A2F18B0381FB0321DA17B4
:10A1D000C2EB610202EB4202A3EB820303F17300C4
:10A1E000049BC0B21978F7F7B9FA009B1B78ABB3A0
:10A1F000464B1A461B788BB34FF0000A0094CDF8FB
:10A200000880DFF80C91D0461446DDF810A00BE072
:10A2100003F17300C0B29AF80010F7F79FFA2378A1
:10A2200008F10108434516DD2B6859F8041F364A2A
:10A230001944A1F18B03D81782FB032EC0EB6E0EDD
:10A24000A1F10C000EEB4E0E7F28A3EB8E03DFDC9A
:10A25000F6F734F9DEE7009CDDF808802A682D4B1C
:10A260001B78002B38D02C4B1B68D0187F2840F36C
:10A270008083254B7F3883FB0032C317C3EB620317
:10A2800003EB4303A0EB83007330049BC0B2197847
:10A29000F7F764FA21490B78022B9ABF5A1CD2B205
:10A2A00000220A701E492B6851F8220018447F28AA
:10A2B00040F35C83144B7F3883FB0032C317C3EB3E
:10A2C000620303EB4303A0EB83007330049BC0B233
:10A2D0001978F7F743FA2A68019B1B88002B00F0D6
:10A2E0003183144BDFF850901A7003233B60FFF763
:10A2F000D3B900BFA29DFF1FCDCCCC3D0000FE42D4
:10A30000F89DFF1F5B9DFF1FABAAAA2A008BFF1FB2
:10A31000D88AFF1FB09EFF1F048BFF1FF99DFF1FF0
:10A32000448CFF1FA59EFF1FD49EFF1F3C9FFF1F55
:10A33000F49EFF1FA49EFF1F1C9EFF1FE89EFF1F91
:10A340008025934A934B1088934A1B8812680D60AE
:10A350000344B2EB630FBFF667AC904B197800294A
:10A3600040F06482B8F800308D4AAB423FF45CACF8
:10A370008C4B158001250D201D7003F03BFC9620B1
:10A3800003F074FC29460D2003F034FC009B1F6889
:10A39000FFF72FBA049CDDF814A0DDF818803D46C5
:10A3A000039B1B78002B53D02B68A3F10C007F2854
:10A3B00040F34B837C488B3B80FB0320DA17C2EBD6
:10A3C000600000EB4000A3EB800303F17300774BC8
:10A3D00004931978C0B2F7F7C1F9009A1378BBB3A8
:10A3E000734A137811469BB3724A0594CDF81890BE
:10A3F000CDF81C80002714468946DDF810800BE05C
:10A4000003F17300C0B298F80010F7F7A7F999F8B4
:10A4100000300137BB4216DD2B6854F8041F624A36
:10A420001944A1F18B03D81782FB032EC0EB6E0EEB
:10A43000A1F10C000EEB4E0E7F28A3EB8E03DFDCA8
:10A44000F6F73CF8DEE7059CDDF81890DDF81C8097
:10A45000029B1B78002B39D0574B28681B68184487
:10A460007F2840F3B482504B7F3883FB0032C31700
:10A47000C3EB620303EB4303A0EB830073304B4B4E
:10A4800004931978C0B2F7F769F94C490B78022B9D
:10A490009ABF5A1CD2B200220A7049492B6851F85F
:10A4A000220018447F2840F38F823F4B7F3883FB84
:10A4B0000032C317C3EB620303EB4303A0EB83003B
:10A4C0007330049BC0B21978F7F748F9019B1B88D9
:10A4D000002B00F07382009B1B783BB9039B1B7819
:10A4E00023B9029B1B78002B00F03C83354B1B7873
:10A4F000002B34D02E480378082B30D832492A68F4
:10A500000968324F0133DBB203F1FF3E511A47F8BD
:10A510002E1003708AF80020B6E400297FF418ADED
:10A52000002B7FF415AD1D49294891F800E0294919
:10A530000391294902912749224A0B70264900902C
:10A54000137003700B70BEF1000F7FF4D5AC3B7835
:10A55000FFF76BB9214B224C1A68FFF7B6BB2A688C
:10A56000D8E7F5F7ABFFFFF7C8BBF5F7A7FFFFF795
:10A570005ABA1C4D09888342A8BF03462B600029A4
:10A580007FF43BAA9A42C8BF0B463FF73CAD34E587
:10A59000469EFF1F8E9DFF1FBC9DFF1F949DFF1FAA
:10A5A000649EFF1F959DFF1FABAAAA2AF89DFF1F5F
:10A5B000008BFF1FD88AFF1F048BFF1FF99DFF1F11
:10A5C000448CFF1FA59EFF1F989DFF1FDC8AFF1F65
:10A5D000DF9EFF1F5B9DFF1FB09EFF1F609EFF1F42
:10A5E0003C9FFF1FD49EFF1FBE4B1B78002B7FF4A8
:10A5F0001BABBD4BBD4A1B78243B83F34703194675
:10A600005B201360F6F7E8FD3B78032B7FF40CAB7F
:10A61000DFF8288398F80020002A40F08582B44FA4
:10A620003B78002B40F07482AE4D2B78002B40F02D
:10A630006382B04B1B78002B40F05282AE4A1380ED
:10A64000AE4B1B78002B40F07A82AD4B7F221A80F4
:10A6500098F80030002B7FF4E7AA3B78002B7FF4BA
:10A66000E3AA2B78002B7FF4DFAAA64A7F210720DC
:10A670001380F6F7B1FD7F210B20F6F7ADFDFFF754
:10A68000D3BAA14BBBF800001B68DFF8B482834249
:10A69000B8F8002080F2BB810B46101AB0F5804F4D
:10A6A000AABF9B03C3EB8333013093FBF0F0F5F7B4
:10A6B00017FFC0F3C61006F051F9944B00901888AC
:10A6C00006F04CF992490190009806F09BF9019B25
:10A6D0000146184606F096F9009906F08BF84FF0FF
:10A6E0007E51009006F02CFB002840F0F78189494C
:10A6F000009806F043FB002840F0BE81009806F069
:10A7000083FBC0B2844B1870FFF705BB834B0193EA
:10A710001B88002B40F05E81814B0393814B029399
:10A72000814B1A461B783BB3804B04940595002758
:10A730001C46154608E003F17300C0B2F6F71CFA98
:10A740002B780137BB4215DD54F8043F9AF800001E
:10A75000774A1844A0F17F0382FB032ED917C1EB7F
:10A760006E0101EB41017F28A3EB8103E3DCF5F7E8
:10A77000A5FEE2E7049C059D039B1B78002B3FF49C
:10A78000F1AA9AF80030A3F10C007F2840F34E8123
:10A7900067488B3B80FB0320DA17C2EB600000EBBD
:10A7A0004000A3EB800303F17300C0B2F6F7E4F9B5
:10A7B000009B1B78002B00F03C815B4B1A461B78FA
:10A7C000002B00F0D981594B0494002705951C46B5
:10A7D0003D46174609E003F17300C0B2F6F7CCF925
:10A7E0003B780135AB4240F3408154F8043F9AF87E
:10A7F00000104F4A1944A1F18B03D81782FB032E96
:10A80000C0EB6E0EA1F10C000EEB4E0E7F28A3EBF9
:10A810008E03E0DCF5F752FEDFE7F5F74FFEFFF7BA
:10A82000F1BA3846F5F74AFEFFF785BA4B2D00F32B
:10A830000F81243D002DB8F8003040F39881AB42E1
:10A840003FF4F2A9ADB23B4BA8F80050012500211E
:10A8500091E500214020F6F7BFFC94E49AF800004F
:10A86000F6F78AF98AE4039A00231370FFF770BBA6
:10A87000F6F782F9FFF733B92A482F4A02904FF0D2
:10A88000000C82F800C00098029A4FF0010E80F888
:10A8900000E082F800C0FFF716BB00231370FFF73B
:10A8A00006BBF5F70BFE61E4F5F708FE44E4F5F7A7
:10A8B00005FEFFF7F8BB049BC0B21978F6F74EFF10
:10A8C000FFF7B8B8039B1B78002B7FF484AA029B88
:10A8D0001B78002B7FF47FAA019B1B880493FFF752
:10A8E00081BA00BF2A9FFF1FF29EFF1FB09DFF1F6E
:10A8F000299FFF1F289FFF1F129EFF1FD19EFF1F32
:10A900005C9DFF1F909EFF1FD49EFF1FA29DFF1FF7
:10A91000CDCCCC3D0000FE42F89DFF1FC29DFF1F25
:10A920005B9DFF1FB09EFF1F008BFF1FD88AFF1F7C
:10A93000ABAAAA2A959DFF1FA59EFF1FC09EFF1FC1
:10A94000E89EFF1F049BD0B21978F6F707FF2A682C
:10A95000C7E47F214020F6F73FFC8C498C4B2A68E6
:10A960000A600021197024E41D46F6E4F5F7A6FDFF
:10A97000ACE4F5F7A3FD88E4F5F7A0FD30E4854BE2
:10A980001B78002B00F09080834B1B78002B7FF40A
:10A990004BA9824B1B78002B3FF446A9B8F8003036
:10A9A0007F4A0A33A8F800301570FFF73DB97D4B98
:10A9B000C0B21978F6F7D2FEFFF729BA794B28789A
:10A9C0001978F6F7CBFE86E5F5F778FD79E5F5F72A
:10A9D00075FD54E5744B0393744B0293F6F7CCF872
:10A9E000009B1B78002B7FF49BAEC5E6704B019358
:10A9F0001B88002B40F0C7806C4B0293C1E69AF88D
:10AA00000000F6F7B9F83B880493FFF7EBB99342DF
:10AA1000D4BFC0EB0303C0EB02033EE6F5F74EFDE7
:10AA2000FFF7D1B9F5F74AFDFFF7B3B9F5F746FDE2
:10AA3000BBE6029B1B78002B7FF497A9039B1B7836
:10AA4000002B3FF449AFFFF7C6B9F5F737FDBEE479
:10AA50001835802DB8F80030564AA8BF8025AB4283
:10AA60003FF4E2A84E4B1580F0E6049C059DFFF7ED
:10AA700079B97F20FFF7FBBA7F2043E60120FFF77B
:10AA8000F6BA454B1B78002B7FF4CEA8434B1B78BE
:10AA9000002B3FF4C9A8B8F80030414A013BA8F8A0
:10AAA00000301570FFF7C0B83B4B1B78002B7FF4CC
:10AAB0009BAD3A4B1B78002B3FF4B6A8B8F800309A
:10AAC000374A0133A8F800301570FFF7ADB8384B9E
:10AAD00001931B88002B3FF445A97FE7012011E675
:10AAE000354B01227F2107201A80F6F775FB7F2165
:10AAF0000B20F6F771FBA3E5304B04227F210720E2
:10AB00001A80F6F769FB00210B20F6F765FB90E54C
:10AB10002A4B02227F2107201A80F6F75DFB7F2156
:10AB20000B20F6F759FB7FE5244A0021072013800C
:10AB3000F6F752FB7F210B20F6F74EFB6FE5204B1B
:10AB400000227F2107201A80F6F746FB7F210B2089
:10AB5000F6F742FB7CE51B4B0093134B1A4A039319
:10AB6000FFF7CAB99AF80000F6F706F8BEE4012B21
:10AB70003FF45AA8012566E6029B1B78002B3FF4A0
:10AB80002AA9FFF7F2B8094B029327E7989DFF1F08
:10AB9000008BFF1F289FFF1F299FFF1F2A9FFF1F5A
:10ABA000959DFF1FF89DFF1F5B9DFF1FB09EFF1F20
:10ABB000C29DFF1F649EFF1F129EFF1F909EFF1FDE
:10ABC0005C9DFF1FDF9EFF1FA59EFF1F002070479B
:10ABD00090F8392090F83800101A704790F8383003
:10ABE00090F839209A4205D95A1C034480F838203D
:10ABF000187E70474FF0FF30704700BF90F8383034
:10AC000090F839209A4286BF1B18187E4FF0FF300B
:10AC1000704700BF704700BF38B50546B0F85E000A
:10AC200090B195F85D301446C3F1210294420CD8DE
:10AC300005F13B001844224601F0D0FF95F85D3045
:10AC4000234485F85D30204638BD01201446287124
:10AC5000EEE700BFB0F85E306BB190F85D30202BAE
:10AC600007D8C218013380F85D30012082F83B100C
:10AC70007047012303710020704700BF0023426921
:10AC800080F8383080F8393080F85C3080F85D30FA
:10AC900080F85E3080F85F3006CA30B40D68046911
:10ACA00043662A4383660A60A370426990F8613064
:10ACB0001649146813441D7A5B7B01EBC5051B0222
:10ACC0006D6803F4E06343F064032B6090F8623036
:10ACD00013449D7CDB7D01EBC5011B02496803F435
:10ACE000E06343F064030B6021685368194205D0A8
:10ACF000036927225A70036904229A71036920228A
:10AD00005A71036980229A7030BC704790420100EA
:10AD100043690CCB12681A420CD0094B99420AD9EC
:10AD2000084B9942036994BF1A220D225A70036995
:10AD300004229A717047036927225A70F7E700BF0F
:10AD40007F1A06003F420F0010B50269D378DBB2CC
:10AD5000D90604463DD510215806D17038D503F0E8
:10AD6000040303F0FF02002B51D03D49626E002323
:10AD70000B7084F85D30002A5BD0904794F85D300A
:10AD8000002B56D02369D0229A70236994F83B2077
:10AD90001A712369012284F85C200222DA7010BD46
:10ADA000304B84F860009C424AD02F4B9C4252D0DA
:10ADB00094F8391013791F29DBB207D82848007896
:10ADC00020B16018013184F8391003760223D37062
:10ADD00010BD5906C3D4917801F0100101F0FF00B5
:10ADE0000029DDD013F001031ED194F85C1094F813
:10ADF0005D00884281BF4B1C091984F85C3091F8D2
:10AE00003B3013712369D0229A702269DEE72369EF
:10AE100084F83920C0229A702369114A19790121D6
:10AE200011700222DA7010BDC02393702269137969
:10AE3000CCE70122002384F85D2084F83B30A1E7B1
:10AE4000626994F86130094913440322187A02F0C8
:10AE50006FFC2269ACE7626994F861300449F3E75A
:10AE6000349FFF1F008EFF1F6C8EFF1FD1AE0000AE
:10AE7000DDAE00000369DB7803F0200373B190F8C6
:10AE800060300133DBB2012B80F860301AD942699F
:10AE900090F861301344187A02F0C6BC70B542696C
:10AEA00003F0FF0590F8613013440446187A02F06D
:10AEB000BBFCA36E5BB184F8385094F83900BDE850
:10AEC0007040184790F85F30002BE0D0704770BD9D
:10AED0000148FFF7CFBF00BF008EFF1F0148FFF7FB
:10AEE000C9BF00BF6C8EFF1F2DE9F047374FDFF859
:10AEF000E0903B68026982B006460093DDF800806E
:10AF00000021A025D3789B065BD53B680193019B6C
:10AF1000C8EB03030F2BF5D949B1102BF2D0002059
:10AF20009070336980229A7002B0BDE8F087726930
:10AF300096F8613013440521187A02F06FFE7269A9
:10AF400096F861301344012193F812A0504602F0A4
:10AF500065FE09240021504602F04CFE2B46013BC1
:10AF6000FDD10121504602F045FE2B46013BFDD1AB
:10AF7000013CEFD1706996F8611001444FF4A07262
:10AF80000C7A4B7B09EBC4011B02496803F4E063B4
:10AF900043F064030B6096F862300344997CDB7DD8
:10AFA00009EBC1011B02496803F4E06343F0640349
:10AFB0000B60013AFDD13269D3789B064FF0010155
:10AFC000A3D4012002B0BDE8F08700BF3C9FFF1F63
:10AFD00090420100F0B503691222DA700269937899
:10AFE00003F0200385B004460D46002B5ED0B42349
:10AFF00093703C4922690B680093009E05E00B6842
:10B000000193019B9B1B042B42D8D37803F02003B0
:10B0100003F0FF00002BF2D094F85D30002B31D00C
:10B020004FF0000E4FF0020C04EB0E0393F83B3090
:10B0300013710B680393039F206907E09B060DD5EE
:10B040000B680293029BDB1B052B28D8C378DBB26D
:10B0500003F0020202F0FF06002AEFD080F803C0DE
:10B060002669F378DBB2DF0632462DD49F062BD556
:10B07000DB0731D40EF1010E94F85D305FFA8EFEDD
:10B080007345D1D800201DBB002384F85E3004E056
:10B090009070236980229A70042005B0F0BD8670FC
:10B0A0002369802204209A7005B0F0BD03F0FF06EA
:10B0B000FFF71AFF10B9042005B0F0BD236984F82A
:10B0C0005F60B0229A7094E78023B3700420DAE7BF
:10B0D00026698023B370D7E7BEF1000F0CBF0220B2
:10B0E0000320F6E73C9FFF1F2DE9F041066900258C
:10B0F000122780F8385080F83950F770D0F810C017
:10B100009CF802E00EF0200E88B0044688461546F2
:10B110001E46BEF1000F49D0B4238CF80230784BA4
:10B1200021691A680092DDF800E006E01A680192D1
:10B130000198CEEB0000042830D8C87800F0200039
:10B1400000F0FF070028F1D04FEA480242F0010268
:10B15000D2B20A711A680292DDF808E0206906E0AE
:10B160001A6803920399CEEB010105292AD8C17808
:10B1700001F0020101F0FF070029F1D04FF0020CAD
:10B1800080F803C02269D17811F0110722D12DBBBC
:10B19000002E0CBFA0238023937003E08F702369DF
:10B1A00080229A70384608B0BDE8F0810EF0FF07A3
:10B1B000FFF79AFE0028F5D0236984F85F70B0226B
:10B1C0009A70ACE787702369802238469A7008B07D
:10B1D000BDE8F081802393700027E3E7012D75D04F
:10B1E000A021917021690A79BE4667464FF0A80CEC
:10B1F0001A680492049805E01A680592059A121AD2
:10B20000052A4AD8CA7802F0020202F0FF08002A92
:10B21000F2D0CF702169CA78D2B212F0100F08466E
:10B220005AD1920658D5013DEDB2012D49D0BEF15B
:10B230001F0F3BD90A79012DDAD11A680692069DB3
:10B2400005E01A680792079A521B052A46D8C27869
:10B2500002F0020202F0FF01002AF2D00223C370C2
:10B260002269D378DBB2D9063AD49B0634D5B02311
:10B27000BEF11F0F93703FD8226904EB0E031279C1
:10B280001A760EF1010E5FFA8EFE16B12369802246
:10B290009A7084F839E0774684E781F80280236960
:10B2A00080229A70774684F839E07BE704EB0E023F
:10B2B00091F8048082F818800EF1010E5FFA8EFE7C
:10B2C000B9E781F802C021690846B0E7A82191706A
:10B2D0002069BE460279B0E7774663E78170DEE712
:10B2E0001021A023D170013BFDD12269937803F096
:10B2F000F7037746937055E723691B79C5E700BFCD
:10B300003C9FFF1F0148FFF71FBD00BF008EFF1FBE
:10B310000148FFF719BD00BF6C8EFF1F704700BFCB
:10B3200038B5144C037801225B000546204684F8AA
:10B330003B3084F85E2084F85D20FFF78BFC2046CC
:10B340000021FFF747FE0B4C2978012320461A46BF
:10B35000FFF7CAFE0128F6D194F8383094F8392066
:10B360009A4205D9E218013384F83830107E38BD8E
:10B37000FF2038BD008EFF1F38B51B4C037801221B
:10B380005B000546204684F83B3084F85E2084F854
:10B390005D20FFF75FFC20460021FFF71BFE124CEB
:10B3A0002978204601230222FFF79EFE0228F6D1CB
:10B3B00094F8382094F839108A420FD2531CDBB22B
:10B3C000A018994284F83830007E0AD9234402320A
:10B3D0001B7E84F8382040EA032038BD4FF6FF700A
:10B3E00038BD40F47F4038BD008EFF1F0C2901D9C5
:10B3F000002070470231490001F0FE01FFF7BCBF99
:10B4000070B50C4C0378164601255B00204684F885
:10B410003B3084F85E5084F85D50FFF71BFC3146EA
:10B420002046FFF717FC29462046BDE87040FFF78D
:10B43000D1BD00BF008EFF1FF8B505460F4616466A
:10B44000412421463A462846FFF7DAFF611C0234C0
:10B45000C9B232462846E4B2FFF7D2FF592CF0D1E8
:10B46000F8BD00BF38B504460D463548FFF706FC69
:10B470006322802120462570FFF7C2FF012002F0E1
:10B48000F5FB204600225E21FFF7BAFF20465D2132
:10B49000FFF746FF242801D0002038BD20460622B1
:10B4A0000C21FFF7C9FF204601222B21FFF7A8FF3F
:10B4B000204601222C21FFF7A3FF20460E222D213A
:10B4C000FFF79EFF204600222E21FFF799FF20461E
:10B4D00001222F21FFF794FF204605223021FFF79C
:10B4E0008FFF204601223121FFF78AFF20460022EC
:10B4F0003221FFF785FF204600223321FFF780FF2E
:10B50000204600223421FFF77BFF20460022352110
:10B51000FFF776FF204600225B21FFF771FF2046F0
:10B5200010225C21FFF76CFF204620225D21FFF7EF
:10B5300067FF20468F225E21FFF762FF012038BDA2
:10B54000008EFF1F10B4047F4160022CC26002D045
:10B5500010BC03F04FBF836810BC1847F0B4464BD3
:10B56000464A186BDC6A01791170454922790A70E4
:10B570009A6A00790870002A46D05968C9688A42D8
:10B580003ED82168CC8B240402F1FF3065D4C0F38F
:10B590000E00C883C88B80B2C882196B0968C88B3B
:10B5A000000452D4C2F30E00C883C88B002480B2BA
:10B5B00012F1FF32C88218BF01229C62D96A2E485C
:10B5C00009680D6800F12404A54236D00068C468FB
:10B5D00014F0804F0C680D6815BF2488247802355C
:10B5E000013544F000440D604463196B254B097923
:10B5F0001970214912B1CA6A12791A70F0BC7047E9
:10B60000521A9A620122D9E7586B196805681E4CD4
:10B610000A63CC62CC682D681C4E24F0804403275A
:10B62000B542CC6083F825701FD1037F4260022BA6
:10B63000C2601ED0F0BC03F0DDBE016890F82400AB
:10B64000CC6840F000404863CFE7CC8BC2F30800E1
:10B6500004F47E442043C883A7E7CC8BC0F30800E2
:10B6600004F47E442043C88394E72B461146F0BC83
:10B6700018478368F0BC1847D88EFF1F1F80004012
:10B680001C8000401B80004000000FFF45B50000FB
:10B6900090E80C00F0B41C6859682568164F174EE6
:10B6A00029432160164D17491760D6601561116056
:10B6B000417A154A5C180A3194F8244053F8215015
:10B6C00002EBC40149680D60017A5C1803EB81014B
:10B6D000247ECD6902EBC40149680D60817A581857
:10B6E00003EB810390F83000596B02EBC002F0BC11
:10B6F00053681960704700BF01401F0001100038F7
:10B700000110007800001F809042010038B5044607
:10B71000104621700A491D4605F074F901464FF0A4
:10B720007E5005F023FA074905F06CF9E56060608A
:10B730002561656102F078FAE061204638BD00BFFE
:10B74000DB0FC9400024744938B504461046217007
:10B7500009491D4605F056F901464FF07E5005F0A7
:10B7600005FA064905F04EF9E560606025616561FE
:10B7700002F05AFAE06138BDDB0FC9400024744979
:10B7800038B503780446032B20D8DFE803F01A18F5
:10B790001002C168406905F02BF80D490546606844
:10B7A00005F0E4F90146284605F0E0F938BD0849FE
:10B7B000406805F0DBF9E16805F024F938BDC068A0
:10B7C00038BDC168406905F013F838BD002038BDA8
:10B7D0000024744970B504460E4602F025FA054669
:10B7E000E069281A05F0BAF8E3682361E56166614B
:10B7F000A0610146606805F0B9F90146A0601048F3
:10B8000005F0B4F904F08AFC04F02AF904F09CFF76
:10B81000054601464FF07E5004F0EAFF616905F0ED
:10B82000F1F821690646284605F0ECF80146304655
:10B8300004F0E0FFE0602046BDE87040FFF7A0BFE5
:10B84000000080BF704700BF2DE9F04F85B09946DA
:10B85000BDF93870BDF83CA0BB1AC1EB090B002B39
:10B86000B8BF5B42BBF1000FB8BFCBF1000B5B452B
:10B870000D4616460093804648DC4D453A46334611
:10B880004CDC194613460A46C5EB09019B1A89B2DE
:10B89000002B0CB2B8BF5B4204EBD474BE42ACBF09
:10B8A0004FF0FF3201224D45039102924FEA6404AA
:10B8B00029DC9BB201930DE0D8F80070BF69B8474E
:10B8C000019BE41AA3B21CB20135002C2DB211DB8E
:10B8D000A94518DB009B5B452A4653463146404646
:10B8E000EADCD8F80020534697692946324640469C
:10B8F000B847E5E7029A1644039AA94502EB030408
:10B9000036B224B2E6DA05B0BDE8F08F4A462B46DF
:10B91000B94635464D4517461E46B2DD30462946E6
:10B920003E464D4607468946AEE700BF10B4046860
:10B930002469A44610BC604730B40468BDF80850C0
:10B940000295A46BA44630BC604700BF30B40468C5
:10B95000BDF808500295E46BA44630BC604700BFB8
:10B9600070B40468BDF90C60BDF8105003960495DE
:10B97000246CA44670BC6047704700BF10B582B00D
:10B98000B0F90C2001910168009200220C6CB0F912
:10B990000A301146A04702B010BD00BF704700BF7B
:10B9A00001F003010129C17506D0032904D0C28822
:10B9B00003894281838170470289C38842818381E0
:10B9C000704700BF2DE9F0410568134E6F6986B0DE
:10B9D000B7420446BDF8308010D1013B13441BB27E
:10B9E0000093CDF804800B46AD6A2046A847236833
:10B9F000DB6AB3420AD106B0BDE8F0810593049238
:10BA00000391B84703A925680EC9E6E7204606B0AA
:10BA1000BDE8F041184700BF79B900002DE9F041B9
:10BA20000568124E6F6986B0B7420446BDF8308093
:10BA30000FD1013BCDF804800B4400921BB2AD6ADC
:10BA40002046A8472368DB6AB3420AD106B0BDE8A6
:10BA5000F081059304920391B84703A925680EC9A4
:10BA6000E7E7204606B0BDE8F041184779B9000085
:10BA70002DE9F04F0568DFF858B06F6985B05F4574
:10BA80000646BDF93890BDF83CA00C46904615D14D
:10BA90001F19BC420CDACDF800A0214601342D6AF2
:10BAA0004B464246304624B2A847BC423568F2DBDA
:10BAB000EB6A5B4507D105B0BDE8F08F0393B8474B
:10BAC0003568039BE4E7304605B0BDE8F04F184702
:10BAD00079B900002DE9F04387B099420546BDF9D8
:10BAE0003840BDF83C6025D0A24212D00768DFF88C
:10BAF0008080D7F81490C14532D18DE85000284697
:10BB0000BC6AA0472B68DB6A434524D107B0BDE877
:10BB1000F083994202DD08461946034628680E96CE
:10BB2000C46B01335B1A1BB22846A44607B0BDE8BC
:10BB3000F0436047A24202DD134622461C462868B5
:10BB40000E96631C846B9B1A1BB22846A44607B052
:10BB5000BDE8F0436047284607B0BDE8F04318470A
:10BB6000059304920391C84703A92F680EC9C4E73F
:10BB700079B900002DE9F04FD0F800E0DFF890909F
:10BB8000DEF814B083B0CB450446BDF93080BDF873
:10BB900034A00D4617461E4631D1CDF800A0DEF880
:10BBA00024B0294633463A462046D8472368CDF884
:10BBB00000A008F1FF323A44D3F824B0294612B26B
:10BBC00033462046D8472368CDF800A02946D3F84D
:10BBD00020B03A4643462046D8472068CDF800A01A
:10BBE000711E29444346056A09B23A462046A847D1
:10BBF0002368DB6A4B4506D103B0BDE8F08FD84718
:10BC0000D4F800E0C9E7204603B0BDE8F04F18477C
:10BC100079B90000F0B4002401264FF6FF75094FF2
:10BC200007600471C475C48104824476C46186755A
:10BC3000067685824582C180028141818281F0BC85
:10BC4000704700BFA43C01002DE9F04F85B00668A5
:10BC5000BDF84450BDF93880CDF800800446019508
:10BC6000D6F848B00392BDF93C60BDF940708946F2
:10BC70009A46D84723680195009742465146D3F823
:10BC8000488020463346C0472068039B0E930F959B
:10BC9000856C4B463A4631462046AC4605B0BDE879
:10BCA000F04F60472DE9F04F87B01746BDF940408F
:10BCB00000912546E91D059344BF2B4603F10E0173
:10BCC0000268BDF8486053690294C91003912B497A
:10BCD000BDF9444001968B42824645D1002C3CDDA3
:10BCE000029B3C445E1EB6B24FF0000923B204939F
:10BCF00001364D46029B002B28DD059B002403EBFB
:10BD0000090806E0EDB22B0604F1010411D4A642A5
:10BD10001CD0A1B211F0070F23B24FEA4505F1D1B3
:10BD2000002BB8BF0733DB10013418F803502B0683
:10BD3000EDD5009BD2F818B019443A4609B2019BE0
:10BD40005046D847A642DAF80020E2D1039B0137DB
:10BD50009944049B3FB2BB42CCD1D36A074A934279
:10BD600006D107B0BDE8F08F9847DAF80020B5E7B4
:10BD7000504607B0BDE8F04F184700BF79B9000042
:10BD800070B4BDF90C60BDF91050BDF814400396B5
:10BD90000495059470BCFFF785BF00BF2DE9F04FF7
:10BDA00093B090460591C1691090BDF8700007905E
:10BDB000BDF874909DF878A00493002900F0CD8020
:10BDC0000A7A0AC9894604998A1AD2B203EBC203D5
:10BDD000BAF1010FDA780B9293F905201E8893F8D7
:10BDE00002B00F9293F9064079D913B2099323B2A6
:10BDF0000C93109B1A68A94B1193194653698B42F7
:10BE000040F0A6800B9B002B55D01FFA88F3002131
:10BE10000D93C8462344DDF8409006910E930F46DB
:10BE20000C46BBF1000F3FD0BDF818100C9B0397D8
:10BE30001FFA8AF0CB1813FB00F304900E9801440C
:10BE40000D98034409B21BB20A910893002505E03E
:10BE50000135EBB264009B45E4B222D9039B2B442D
:10BE6000590703D1731C18F806409EB22306EFD57C
:10BE7000099BBDF81000E91811FB00F10598BAF113
:10BE8000010F0FFA8AF301441CD007980190009328
:10BE9000D26909B217464846089AB847D9F800202F
:10BEA000D6E7039F5F44FFB2069B0B9901330693CD
:10BEB000DBB29942B5D8D36A119A934243D113B0F9
:10BEC000BDE8F08F0F9B191893690A9A29441F4601
:10BED00009B2079B4846B847D9F80020B8E70023C5
:10BEE0000C93099385E70A9A0D9B0132013B52B2EC
:10BEF00013F0FF030A920D936FD1DDF81890079BA2
:10BF0000DDF83C80DDF820A04B4517D0BAF1010FD9
:10BF100000F0C8800B9A109DCDF804900BEB8B01BC
:10BF20004FEACB030A4400931146DEF81C40534607
:10BF3000424609B22846A047D5F800E0DEF82C308A
:10BF4000119A9342BBD0109813B0BDE8F04F184738
:10BF5000109D284698472A6854E7109A0598B2F928
:10BF60000A308342ABDDB2F90C304345A7DD06232E
:10BF700013FB0A03002BA2DD08EBCA03002B9EDD96
:10BF8000537E2BB9049BAF2B02D90133DBB2049350
:10BF9000109BD3F800E0414B11931A46DEF81430A1
:10BFA000934240F08E801FFA88F30E9308339BB2C1
:10BFB000BDF81420059305230D9300230A93CDF8B3
:10BFC0003C800FFA8AF3DDF84080CDF818900B9290
:10BFD0001FFA8AFBCDF820A099460A9ABDF81000F6
:10BFE0000B9C0E9D0523194611FB00232C4811467E
:10BFF000C75C039702FB0B4214FA81F312B21BB227
:10C0000009920C932C462E461CE0089B0999012BA3
:10C010002AB24B4640462DD0079F0197CDF800909D
:10C02000DEF81CA0D047D8F800E0039B5B08013481
:10C030000393059BA4B25D445E44A342ADB2B6B285
:10C040003FF451AF039BD807DFD4079B069A934276
:10C05000EBD0089B012B16D0069B0193CDF80090E6
:10C06000DEF81CA009994B4632B24046D047D8F8BA
:10C0700000E0DAE7DEF818A0079B0C9922B2D0475F
:10C08000D8F800E0D1E7DEF818A00C991346404636
:10C0900022B2D047D8F800E0C7E700BF79B9000066
:10C0A000F43C01000B99109DCDF800900531DEF8AD
:10C0B000204009B2424608232846A047D5F800E0B0
:10C0C0003CE7109C20469847D4F800E06BE700BF9F
:10C0D000F0B5C36985B004462BB30A2968D00D2991
:10C0E0004AD01A7A914247D3587A884244D35D683D
:10C0F0008A1A05EBC205AA78002A50D0E8780028F1
:10C100004DD0207E00283AD095F905E0B4F90E0014
:10C11000A67DB4F90A70724406FB0202BA4262DCE0
:10C12000B4F9102030E00A2956D00D2924D0027E1F
:10C13000002A4BD0B0F90E00A57DB4F90A600622A2
:10C1400012FB0502B2423EDD228AE38102EBC50208
:10C1500012B218462282A78A668A02950B468DE89B
:10C16000C00001462046FFF719FEA37DE28903EBDC
:10C17000430302EB4303E381012005B0F0BDA67D3C
:10C18000B4F90E00B4F91020B4F814E0678A0296EE
:10C190000B468DE8804001462046FFF7FFFD2979D8
:10C1A000E389A27D012001FB0233E38105B0F0BDEC
:10C1B0000022C2819A7A817D038A01FB02330382C5
:10C1C000012005B0F0BDB4F91020C4E7857DB4F9B5
:10C1D0001020B0F90E00BEE7028A817DC38102EB18
:10C1E000C1030382C8E70020E0819B7A228A03FB17
:10C1F000062212B22282C7E7C1810282704700BFC5
:10C20000002908BF01218175704700BF81824182EA
:10C21000704700BFC07D7047B0F90A00704700BF8B
:10C22000B0F90C00704700BFF0B5C47DBDF81450E4
:10C23000022C75D0032C6ED0012C32D0002A79DB71
:10C24000B0F90840944265DD002978DBB0F906605A
:10C250005818B042C4BF731A1BB2002B5ADD002A13
:10C260001046B8BFD01D012440F3CF0002F00702F2
:10C27000704E01EBC01104FA02F2A5423144D2B271
:10C2800000F0A480C0F09580022D43D1013B11FA4B
:10C2900083F04B1E13F8011F514083421970F9D1EE
:10C2A000F0BDC488013CA21A12B2002A7BDBB0F9AF
:10C2B000064094422EDD00293DDBB0F90860581895
:10C2C000B042C4BF731A1BB2002B23DDC9B2C80829
:10C2D000584C02EBC01211F00701DBB204EB020074
:10C2E00039D0C1F10801C9B2534E8B42765C2AD2D3
:10C2F000C3EB010EFF2747FA0EF7012D06EA0706EA
:10C3000074D06ED3022D40F09480A75C7E40A6547A
:10C310008B421DD2F0BD0489E41A611A09B2C4E748
:10C320000689C488013EB21AE41A12B2611A002AC0
:10C3300009B285DAF0BD0B441BB20021BDE70B4406
:10C340001BB2002182E7012D50D04AD3022DDCD050
:10C350005B1ADBB28030072B18D9022D4ED0A3F127
:10C360000806C6F3C406B11C00EBC111012D0CBFB9
:10C37000FF24002400F1800202F8804C80328A42BF
:10C38000FAD1013600EBC61003F00703002BC1D031
:10C390002A4A012DD35C2DD006D3022DBAD10278C2
:10C3A00053400370F0BDF0BD027822EA030303702E
:10C3B000F0BD013BD24311FA83F0D2B24B1E13F809
:10C3C000011F114083421970F9D1F0BD013B11FAF0
:10C3D00083F04B1E13F8011F114383421970F9D1EA
:10C3E000F0BDA75C27EA0606A65491E7A75C3E438A
:10C3F000A6548DE7027813430370F0BDA3F108053E
:10C40000C5F3C405AC1C00EBC41400F1800212F8A3
:10C41000801CC94302F8801C8032A242F7D101354A
:10C4200013F0070300EBC5103FF474AF034AD35C6D
:10C43000B5E7F0BD208FFF1F188FFF1F108FFF1F64
:10C44000F0B5C47DBDF81450022C76D0032C6FD00B
:10C45000012C37D000297ADBB0F906408C4230DD60
:10C46000002A79DBB0F908609818B042C4BFB31A4B
:10C470001BB2002B25DDD2B2D008754C01EBC011E8
:10C4800012F00702DBB204EB010071D0C2F1080226
:10C49000D2B2704E9342B65C62D2C3EB020EFF275B
:10C4A00047FA0EF7012D06EA070600F0AC80C0F04F
:10C4B000A580022D40F0CA80675C7E40665493429E
:10C4C00053D2F0BDC488E41AA21A12B2002977DB55
:10C4D000B0F908408C42F4DD002A39DBB0F906607F
:10C4E0009818B042C4BFB31A1BB2002BE9DD002973
:10C4F0000846B8BFC81D012440F3CF0001F0070172
:10C50000534E02EBC01004FA01F1A54206EB000203
:10C51000C9B268D05AD3022DD3D1013B12FA83F0AD
:10C52000531E13F8012F4A4083421A70F9D1F0BD0F
:10C530000489013C611A09B2C8E7C6880489013E32
:10C54000711AE41A09B2A21A002912B284DAF0BDF3
:10C5500013441BB20022C1E713441BB2002281E73F
:10C56000012D50D04AD3022DA6D09B1ADBB28030C9
:10C57000072B18D9022D4ED0A3F10806C6F3C40626
:10C58000B11C00EBC111012D0CBFFF24002400F1F0
:10C59000800202F8804C80328A42FAD1013600EBE8
:10C5A000C61003F00703002B8BD02B4A012DD35C60
:10C5B0002DD006D3022D84D1027853400370F0BDF4
:10C5C000F0BD027822EA03030370F0BD013BC943CA
:10C5D00012FA83F0C9B2531E13F8012F0A408342A6
:10C5E0001A70F9D1F0BD013B12FA83F0531E13F813
:10C5F000012F0A4383421A70F9D1F0BD675C27EA24
:10C60000060666545BE7675C3E43665457E702786C
:10C6100013430370F0BDA3F10805C5F3C405AC1CBA
:10C6200000EBC41400F1800111F8802CD24301F812
:10C63000802C8031A142F7D1013513F0070300EBC4
:10C64000C5103FF43EAF044AD35CB5E7F0BD00BF70
:10C65000208FFF1F188FFF1F108FFF1FF8B50D1EB3
:10C6600006DB14461F460646FFF7D6FD854200DB73
:10C67000F8BD002CFCDB3046FFF7D2FD8442F7DA30
:10C680003046FFF7C7FD02284BD0032843D00128CE
:10C6900004D1F388013B1B1B2C461DB2012F03D094
:10C6A00026D3022F12D0F8BD002C2346B8BFE31DBD
:10C6B00043F3CF0305EBC3151E4804F00704435DA5
:10C6C000012101FA04F41C434455F8BD002C234613
:10C6D000B8BFE31D43F3CF0305EBC315154804F0C2
:10C6E0000704435D012101FA04F45C404455F8BDA0
:10C6F000002C2346B8BFE31D43F3CF0305EBC3155E
:10C700000C4804F00704435D012101FA04F423EA14
:10C7100004044455F8BD3389013B5B1B25461CB21C
:10C72000BCE7F18832890139013A4D1B141B2DB247
:10C7300024B2B3E7208FFF1F38B5402204460D46D0
:10C740008021FFF767FAFF23064A84F8255084F812
:10C75000223084F8263084F8243084F82330226094
:10C76000204638BDFC4101004FF4806200210148A1
:10C7700004F0FCBE208FFF1FF8B590F92230013382
:10C7800004460F4642D0012190F8260001F032FA0B
:10C79000002194F8240001F02DFA002194F82600DD
:10C7A00001F028FA94F8273083B1254B1A684FF02E
:10C7B0000043D3625763D36A002BFCDA936B94F87F
:10C7C00026000121BDE8F84001F014BA08268025B2
:10C7D000002194F8230001F00DFA17EA05034FF049
:10C7E000010194F8220008BF194601F003FA012163
:10C7F00094F82300CD4001F0FDF9013EE8D194F812
:10C8000026000121BDE8F84001F0F4B90D4C90F884
:10C81000203001255B002046002184F83B3084F85D
:10C820005E5084F85D50FEF715FA39462046FEF753
:10C8300011FA29462046BDE8F840FEF7CBBB00BF01
:10C84000D88EFF1F008EFF1FF8B50D4690F92210FD
:10C8500080F820200131044680F821501F4600F066
:10C86000AD80012190F8240001F0D8F9012194F85D
:10C87000260001F0D3F994F82730002B00F0D38084
:10C88000804E3046FEF704FFF37A002B40F0DB8049
:10C8900033687D4AD968914206D07C4E7C487D49F8
:10C8A0001E60DA6018611960E7B194F9250000286C
:10C8B00018DBC0B2012101F0B1F9012194F8250083
:10C8C00001F098F9012001F0D1F9002194F8250038
:10C8D00001F090F90A2001F0C9F9012194F825002E
:10C8E00001F088F9AE212046FFF746FFD52120460A
:10C8F000FFF742FF80212046FFF73EFFA821204698
:10C90000FFF73AFF3F212046FFF736FFD3212046AD
:10C91000FFF732FF00212046FFF72EFF402120467F
:10C92000FFF72AFF8D212046FFF726FF012D4DD06E
:10C9300014212046FFF720FF20212046FFF71CFF8F
:10C9400000212046FFF718FFA1212046FFF714FF22
:10C95000C8212046FFF710FFDA212046FFF70CFF21
:10C9600012212046FFF708FF81212046FFF704FF30
:10C97000CF212046FFF700FFD9212046FFF7FCFE1C
:10C98000F1212046FFF7F8FE2046DB21FFF7F4FEF9
:10C9900020464021FFF7F0FE2046A421FFF7ECFEE1
:10C9A0002046A621FFF7E8FE20462E21FFF7E4FEF1
:10C9B0002046AF21BDE8F840FFF7DEBE3648FEF75F
:10C9C0005DF936493448FEF7A3F96DE7204610219A
:10C9D000FFF7D2FE20462021FFF7CEFE20460021A1
:10C9E000FFF7CAFE2046A121FFF7C6FE2046C82158
:10C9F000FFF7C2FE2046DA21FFF7BEFE20461221D5
:10CA0000FFF7BAFE20468121FFF7B6FE20469F21A0
:10CA1000FFF7B2FE2046D921FFF7AEFE22212046C5
:10CA2000FFF7AAFEB0E7012194F8220001F0F6F822
:10CA3000012194F8230001F0F1F894F82730002B3D
:10CA40003FF432AF1CE772B6F37AD8071A4606D520
:10CA50001349F26808680240B2610A601A469907F1
:10CA600006D5104933690868F27A0340F3610B6018
:10CA7000530705D50C4A736911680B403362136084
:10CA800062B605E7D88EFF1F0000013801403F0065
:10CA90000000017800003F80008EFF1F801A060012
:10CAA00080E100E084E100E088E100E02DE9F84F5A
:10CAB00021210546FFF760FE28460021FFF75CFEB6
:10CAC00028467F21FFF758FE28462221FFF754FE13
:10CAD00028460021FFF750FE28460721FFF74CFEAD
:10CAE00095F92230013349D0012195F82600DFF86D
:10CAF000E480DFF8E4B001F07DF8012195F824002E
:10CB000001F078F8002195F8260001F073F808F597
:10CB100080694FF0004A95F8273018F8017F0BBB69
:10CB200008268024002195F8230001F063F817EA15
:10CB300004034FF0010195F8220008BF194601F0E7
:10CB400059F8012195F82300CC4001F053F8013E3B
:10CB5000E8D1C845DFD195F826000121BDE8F84F9E
:10CB600001F048B8DBF80020C2F82CA05763D36A64
:10CB7000002BFCDAC845936BCDD1ECE7DFF8508091
:10CB8000124F00244FF0010995F82030104888F822
:10CB90005E905B00402188F83B3088F85D90FEF79E
:10CBA00059F804F11006B6B2395D09480134A4B24F
:10CBB000FEF750F8B442F7D101210548FEF70AFA12
:10CBC000B4F5806FE0D1BDE8F88F00BF208FFF1F64
:10CBD000008EFF1F1F8FFF1FD88EFF1F844641EA64
:10CBE000000313F003036DD1403A41D351F8043BE5
:10CBF00040F8043B51F8043B40F8043B51F8043B37
:10CC000040F8043B51F8043B40F8043B51F8043B26
:10CC100040F8043B51F8043B40F8043B51F8043B16
:10CC200040F8043B51F8043B40F8043B51F8043B06
:10CC300040F8043B51F8043B40F8043B51F8043BF6
:10CC400040F8043B51F8043B40F8043B51F8043BE6
:10CC500040F8043B51F8043B40F8043B51F8043BD6
:10CC600040F8043B51F8043B40F8043B403ABDD245
:10CC7000303211D351F8043B40F8043B51F8043BE7
:10CC800040F8043B51F8043B40F8043B51F8043BA6
:10CC900040F8043B103AEDD20C3205D351F8043B76
:10CCA00040F8043B043AF9D2043208D0D2071CBF42
:10CCB00011F8013B00F8013B01D30B88038060466B
:10CCC000704700BF082A13D38B078DD010F00303E1
:10CCD0008AD0C3F10403D21ADB071CBF11F8013B51
:10CCE00000F8013B80D331F8023B20F8023B7BE7A0
:10CCF000043AD9D3013A11F8013B00F8013BF9D2CB
:10CD00000B7803704B7843708B7883706046704764
:10CD1000374A384913681B06FCD40B6813F08003AC
:10CD2000F8D172B634490A78002A5FD0334A3448C1
:10CD3000F0B4344C176806682568D4680C303E445B
:10CD4000143200681268304F35442C4420440244A9
:10CD5000C2F34E022D4E2E482E4D2F4C42F400426F
:10CD60003A60376806682D682C4A24680C303E44C7
:10CD7000006812682A4F35442C4420440244C2F310
:10CD80004E02284E2848294D294C42F400423A6070
:10CD9000376806682D68274A24680C303E440068CE
:10CDA0001268254F35442C4420440244C2F34E02FD
:10CDB000224E2348234D244C42F400423A60376807
:10CDC00006682D68214A24680C303E4400681268C9
:10CDD00035442C4420440244C2F34E021C4842F421
:10CDE000004202600B7062B6F0BC704762B67047DA
:10CDF00024B0034024B00B40369FFF1F38B00340DF
:10CE00003CB0034040B003402CB0034058B0034056
:10CE10005CB0034060B0034064B003406CB00340BA
:10CE200030B0034038B00B403CB00B4040B00B403A
:10CE300044B00B404CB00B402CB00B4058B00B40F2
:10CE40005CB00B4060B00B4064B00B406CB00B406A
:10CE500030B00B4030B42948294A2A4B2A4D60246F
:10CE6000E121047011701B78284C082B30D00A2B5C
:10CE70002748284937D00C2B0CBF35223D221223DE
:10CE80002A60236002600B60234B24491B78244AEC
:10CE9000BBB101230B601360224B23491B78234A4B
:10CEA000012B26D9042B0FD9082B1ED9102B94BF88
:10CEB000862387230B6013601D4B01221A7030BC40
:10CEC00070470B601360E7E784230B601360F3E7A0
:10CED00000F58E200F490830012213232A602360B9
:10CEE00002600B60D0E73922F7E785230B601360FF
:10CEF000E2E780230B601360DEE700BF00400740DD
:10CF0000014007402093FF1F08B003400CB00340CE
:10CF100008B00B400CB00B40399FFF1F20B00340FE
:10CF200020B00B402193FF1F24B0034024B00B40DE
:10CF3000369FFF1F0C2830B417D91023984228BF02
:10CF400018461C46104A114D1178181A8C42287048
:10CF500018D00F4913700B7823B10E490E4A0023E5
:10CF60000B60136030BCFFF775BF0A2802D90C2391
:10CF70001C46E7E7082802D90A231C46E2E70823F3
:10CF80001C46DFE730BC70472093FF1F359FFF1F13
:10CF9000369FFF1F24B0034024B00B4028282FD811
:10CFA000334B2DE9F0411E5CFF2E2BD0314B1B780B
:10CFB000002B2AD132062CD472B62F4D2F4C2F467F
:10CFC000012326602B7062B672B623681B060CD450
:10CFD0003B781BB9F4E72B78002BF1D062B602F056
:10CFE0007DFB72B623681806F5D5254B1B68002219
:10CFF0002A7062B6234A107843FA00F0BDE8F08147
:10D00000002070470020BDE8F081FFF781FE320666
:10D01000D2D572B61C4DDFF87C801C4C06F0400760
:10D02000FFB206F03F06D8F80030DFB123F010035E
:10D03000C8F8003001232660134A2B7062B672B61E
:10D04000236819060CD413781BB9ECE72B78002B56
:10D05000E9D062B602F042FB72B623681B06F5D532
:10D060000B4BC3E743F01003C8F80030E2E700BF02
:10D070004C420100369FFF1F389FFF1F00B0034046
:10D0800010B00340359FFF1F379FFF1F00B00B40BC
:10D0900010B00B400CB00B400A4A0B49136843F424
:10D0A000805313600B7843B9084BC0221A70084BA9
:10D0B00080F30C0000B218807047044B80221A7075
:10D0C000F5E700BF2C800440399FFF1F21C00C40B2
:10D0D00000C00C40F0B51B4B1B4E596818689A688D
:10D0E000DB6885B06C460FC4337899071DD5174AA5
:10D0F000174C1378174913F0700318BF1370164AB2
:10D10000164B8027177000263320032226706D46A9
:10D1100008701A7072B6043C45F001052046A84715
:10D1200062B6237813F0700309D10D4B064901E074
:10D13000013B02D00A78D207FAD505B0F0BD2370C2
:10D1400005B0F0BD7842010001000240000002403D
:10D15000040002400B000240070002400A000240A7
:10D16000410D0300B0F5006F0AD210B5094B1B78D2
:10D17000DB07044606D504F1A0500078C0B210BD0C
:10D1800000207047FFF7A6FF04F1A0500078C0B25E
:10D1900010BD00BF01000240B0F5006F17D238B5D6
:10D1A0000F4B1B78DA070D46044611D504F1A05049
:10D1B0000378AB420AD00B4A137813F0700318BF00
:10D1C0001370074A05701378DB07FCD538BD70472C
:10D1D000FFF780FF04F1A0500378AB42EBD1F5E7F5
:10D1E000010002400000024008B5104C08E023682E
:10D1F00059050DD423681A050FD42368DB0411D414
:10D2000023685803F3D501F023F823685905F1D5B5
:10D2100002F0C2FA23681A05EFD502F053FB236827
:10D22000DB04EDD500F0A8FEEAE700BF348004403F
:10D2300008B5FFF7D9FF00BF014B10221A807047D5
:10D2400000200540704700BF094908B50B6830B1A0
:10D250006A461844A2F58052904202D208601846ED
:10D2600008BD03F031FE0C2303604FF0FF3008BD12
:10D270002493FF1FFEE700BFEFF3138070B9EFF3B5
:10D2800010836BB9EFF305825AB94FF48070EFF356
:10D2900011832BB1984228BF184670474FF0FF30DA
:10D2A00070470F2A01D81846F1E7014BD05CEEE732
:10D2B000F0E300E0F0B44D1E2E46002400E00134FF
:10D2C000B0FBF2F302FB1300092800F130078ABF1C
:10D2D0003730F8B2C0B206F8010F1846002BEED175
:10D2E0000A1953704CB1107815F8016F287001338A
:10D2F000E01A834202F80169F5DB0846F0BC70478A
:10D300002DE9F04F0D4685B085EAE5790146824664
:10D3100017461C46A9EBE57903F03AFD002840F0DA
:10D320002F812AF000484046C74903F031FD00280C
:10D3300047D14046C44903F00DFD0646002840D1C0
:10D340000021504603F0FCFC002814BF04200320F9
:10D3500048451DDB002DC0F274815046002103F0CA
:10D36000EFFC254648BB49214E22462321706270BE
:10D37000A3700334002E00F07681A019202304F856
:10D38000013BA042FBD10023037005B0BDE8F08F44
:10D39000002DC0EB0906E0DA002E00F05281A5193D
:10D3A000202304F8013BAC42FBD15046002103F09E
:10D3B000C7FC002800F0228100262D232B706C1C56
:10D3C000D1E702AB01AA3946504603F06DFDBB46DA
:10D3D0008046DDF80490002F57D0C9F10003BB420E
:10D3E00000F39480404604F02BFB0646B145B8BFDD
:10D3F0000136B9F1000F40F098800136DDF808E001
:10D40000BEF1000F53D00136A81B002804EB060123
:10D4100053DC23462D221A700133B9F1000F63D17A
:10D4200037B11A46302002F8020B2E2058701346EE
:10D430008B4220D25F1C98F800201A708F4208F1AE
:10D44000010819D0019A4FF02E0E0BE083F801E08D
:10D4500002338B4203F101070DD218F8010B18704B
:10D460008F4209D0013A0192002AEFD03B468B420D
:10D4700003F10107F1D31946002DC0F2A980002362
:10D4800020460B7005B0BDE8F08FB9F1000FA4D1B4
:10D4900090F800806D496E4A012301939946B8F1D6
:10D4A000340F8CBF884690464FF0FF3397E7A81B98
:10D4B000002804EB060140F3D880014422460138DD
:10D4C0004FF0200C02F801CBC2F1010303442344C6
:10D4D000002BF7DC20EAE07301332344BEF1000F98
:10D4E00098D1B9F1000F9BD0A2DA002FA0D01A4634
:10D4F000302002F8020B2E275F70C9EB020302F8FE
:10D50000010B9342FBD10022019291E7C7F1000980
:10D510000126B1453046B8BF0136B9F1000FDFF83A
:10D520003081CDF804903FF468AFBFF667AF002FAD
:10D530003FF464AF09EB0703984207F102067FF658
:10D540005DAF002F07DD5046424903F05BFABBF1A7
:10D55000010B8246F7D102AB03AA5946504603F0AD
:10D56000A3FCDDF80490039A7B1CC9EB02029A42EB
:10D5700008BF09F10109804608BFCDF804903DE7D6
:10D580000021504603F0DCFB002814BF04200320D8
:10D5900048453BDA002DC0EB09063BDB4FF07E53DC
:10D5A0005046002163F31E0003F0CAFB2546002805
:10D5B00041D14E2341222370A37062700334002EA8
:10D5C00051D0A019202304F8013B8442FBD1DAE6B4
:10D5D000A8194342002B6FEA00007FF750AF0A46BC
:10D5E000202502F8015BC2F1010303440B44002B28
:10D5F000F7DC20EAE0730133194440E749214E2269
:10D60000462329706A70AB70E81CBCE6002D16DB5F
:10D610000026C3E79EB1A519202304F8013BAC42C4
:10D62000FBD14FF07E535046002163F31E0003F000
:10D6300087FB88B100262D232B706C1CB9E725468B
:10D64000EFE72546B1E600BFFFFF7F7F8C42010078
:10D6500088420100000020414E2341222B70AB7014
:10D660006A70E81C8FE620468DE62346D5E600BFAB
:10D67000704700BF10B40F4B53F8302092F880422F
:10D680002CB1012369B182F8803010BC704703EBE4
:10D69000C0035B681A6841B922F002021A6010BC2C
:10D6A000704782F8003110BC704742F003021A60E4
:10D6B00010BC7047904201001C4A02EBC0030129D4
:10D6C0005B6811D004291BD052F83000002280F88A
:10D6D000802229B1022920D0032922D01A60704764
:10D6E0004FF480721A60704752F830004FF4A27203
:10D6F00080F880121A601A6822F020021A607047BF
:10D7000052F830104FF4A272012081F880021A60A2
:10D710001A6842F020021A60704740F203121A6041
:10D7200070474FF481721A60704700BF9042010049
:10D73000212817D8F8B5042A13D8DFE802F0494C9D
:10D740004F1446002C4872B6236823F4702343F02C
:10D750008072C4F384011643236040F82150266090
:10D7600062B6F8BD70474FF41026244B03EBC0039C
:10D770000D465C68216811F4E06134D0204B214AE9
:10D780002149C3F89C2104F140422048C3F8A41168
:10D79000A2F592211E4FC3F8A0017C291D48C3F8B1
:10D7A000A871C3F8AC01CDD9A2F594237C2B18D96C
:10D7B000A2F596237C2B19D9A2F598237C2B17D997
:10D7C000A2F59A227C2A15D9F8BD4FF43026CCE771
:10D7D0004FF40026C9E74FF44026C6E74FF4202651
:10D7E000C3E70D48AFE7FFF767FFC7E70B48AAE7B6
:10D7F0000B48A8E70B48A6E72893FF1F90420100BB
:10D800000082FF1FF188FF1F9988FF1FC588FF1F37
:10D810006D88FF1F4188FF1F6093FF1FB093FF1F9C
:10D82000E093FF1F0094FF1F1A4B03EBC00010B4DE
:10D83000426802F14043A3F592217C2905D9A3F562
:10D8400094217C2913D8144900E0144972B6136856
:10D85000134C23F08773C2F3840023F4803343F026
:10D860008073136041F8204062B610BC7047A3F586
:10D8700096217C2909D9A3F598217C2907D9A3F5FC
:10D880009A237C2BF1D80749E0E70749DEE70749EF
:10D89000DCE700BF904201006093FF1F2893FF1F49
:10D8A00071D600000094FF1FB093FF1FE093FF1F8D
:10D8B00030B4054B054D064C002210211A602A6039
:10D8C0002060196030BC704714D0034004D003407E
:10D8D00000D00340282838B52ED0002904464FDD5B
:10D8E0005F4B1B78012505FA03F28A4202D82128F2
:10D8F00037D938BD0338C2B2012A3AD9202C4AD0D0
:10D90000192C48D0574A126802FB011222FA03F37D
:10D910001D2800F29B80DFE800F0928B847D9999AE
:10D92000766F99999999999999999968615A5399A2
:10D930004C99999999999945494B1B780B2B08D982
:10D940000C2B1CBF0C3B19410846BDE83840FFF7C3
:10D95000A3BBC3F10C0399400846BDE83840FFF76C
:10D960009BBB2946FFF786FE2946BDE83840FFF7F6
:10D97000A3BE3D4A126802FB011222FA03F3C7E775
:10D980002128B6D80021FFF775FE20460121BDE809
:10D990003840FFF791BE354A126802FB011222FAA5
:10D9A00003F3B5E73249334A0B604FF45173136008
:10D9B00038BD3149314A0B604FF45173136038BDA3
:10D9C0002F49304A0B6040F24443136038BD2E4962
:10D9D0002E4A0B6040F24443136038BD2C492D4A57
:10D9E0000B6040F24443136038BD2B492B4A0B6057
:10D9F00040F24443136038BD29492A4A0B6040F283
:10DA00004443136038BD2849284A0B6040F2444320
:10DA1000136038BD2649274A0B6040F24443136027
:10DA200038BD2549254A0B6040F24443136038BD98
:10DA30002349244A0B604FF45173136038BD2249C7
:10DA4000224A0B604FF45173136038BD212C3FF60E
:10DA500050AF7F29D4BF00210121204693E700BFAA
:10DA60000894FF1F088003400890034008800B4083
:10DA700010800B4048A0044018800B404CA004408C
:10DA80001880034008B004401080034004B00440F4
:10DA90004080034018C004403880034014C0044054
:10DAA0002880034010B00440208003400CB00440A4
:10DAB0003080034010C00440488003401CC0044034
:10DAC000189003403490044010900340309004407C
:10DAD00038B1102828BF1020044AC3B21078137040
:10DAE0007047024A01231078137070470894FF1F93
:10DAF0002DE9F8430E4680463249334D304603F057
:10DB00001FF947F6122300281ABF1D464FF00209DD
:10DB10004FF00109002425FA04F002F01BFF4FF03A
:10DB20005E51074602F06EFF0146304603F01CF9D5
:10DB300030B90134072CEED1E80902F00BFF07469B
:10DB40003146384603F012F84FF07C5102F050FE97
:10DB500003F05AF94FF6FF729042A8F1030328BF71
:10DB60001046012B29D9B8F1170F17D8174B23FAF4
:10DB700008F303F0010383F0010223B9B8F1190F90
:10DB80000FD0BDE8F883124B124D13491A6044EAD6
:10DB9000C9042A6008601C60BDE8F883B8F1200F52
:10DBA000ECD10E4B0E4D0F49002244EAC9041A6015
:10DBB0002A6008601C60BDE8F8830B4B0B4D0C49D4
:10DBC000F2E700BF001BB740006CDC026006F0000B
:10DBD00000800340048003400880034000800B4025
:10DBE00004800B4008800B400090034004900340E9
:10DBF00008900340212801D8FFF73CBD704700BFC3
:10DC0000212806D8044B53F8303093F80002C0B2F4
:10DC100070470020704700BF90420100212801D8C2
:10DC2000FFF74ABD704700BF72B60C490C4B0D4A56
:10DC30001B680868126862B6520102D5322B88BF91
:10DC400001300949C3F5BB334FF47A72FF33A1FBAE
:10DC5000031302FB00F000EB931070473C9FFF1F83
:10DC600018E000E004ED00E0ABAAAAAA2DE9F84311
:10DC7000054672B6204F214B214A1B683C6812684A
:10DC800062B6520102D5322B88BF013495B3C3F579
:10DC9000BB331C4EDFF86490DFF86480FF334FF431
:10DCA0007A72A6FB031302FB04F404EB931472B61E
:10DCB000D9F800103A68D8F800E062B6C1F5BB3375
:10DCC000FF33A6FB03031EF0806FC4EB93134FF4E6
:10DCD0007A7002D0322988BF013200FB0233B3F5DB
:10DCE0007A7F04D3013D05D004F57A74DFE701F0B3
:10DCF000F5FCDCE7BDE8F8833C9FFF1F18E000E07F
:10DD000004ED00E0ABAAAAAAF8B52D4B2D49DFF827
:10DD1000D0E0DFF8D0C02C4E2C4D2D4C2D4A2E4F8C
:10DD20004FF4000018604FF0807018604FF00070E2
:10DD300018604FF0806018604FF00060186000209D
:10DD4000086028234BF6FF71CCF80010CEF80030A5
:10DD5000336013602B6023603B60B36293620922DF
:10DD600045F8242CC4F8D80F05F57F65C7F8D41FF3
:10DD700007F5FF2707F5FA67C6F8F83F2B6006F5A9
:10DD8000FF26C4F8D42F05F5FD2504F5FF243860DF
:10DD900006F2F4761148316005F5FF6504F5FD647F
:10DDA0002B6023600260FFF755F81920FFF75EFF34
:10DDB00000F05AFE40F21310BDE8F840FFF756BFDE
:10DDC00008E100E004800340148003402480034005
:10DDD0002C8003401C8003403480034000800B40B3
:10DDE0000C800340088003402DE9F84F214B1B684D
:10DDF00007460BB101221A70DFF888901E4D99F882
:10DE00000040DFF884801D4E0134272C8ABF4FF07C
:10DE1000000A5FFA84FA5446AB462B78A34216D127
:10DE2000FFF72AFA40281FDC33791B06F5D59BF84B
:10DE300000300133272B86BF00221346DAB218F8D0
:10DE40000330DBB2F3712A702B78A342E8D00C497F
:10DE50000A4BFFB208F804700120AC22087089F860
:10DE600000A0DA70BDE8F88FFF28D6DD01F036FC9F
:10DE7000D3E700BFB49FFF1FB19FFF1F00C0064044
:10DE8000B09FFF1FB89FFF1F489FFF1F1C4BDFF86D
:10DE900094C01A681B49F0B542F480521A4D1A60BA
:10DEA000DFF884E0194F1A4E1A4C00238CF800302A
:10DEB0004FF451722B701F2840F213358EF800304A
:10DEC0003B70337025600A6012D819460124124A4B
:10DED000124D11701248547000212C274026937265
:10DEE0004FF4003491701174D7702E700460F0BD3F
:10DEF000C0F34431C0F3471400F01F03E7E700BF4D
:10DF0000348004400CC00440459FFF1FB19FFF1F99
:10DF1000B09FFF1F08C0044000C0064031E400E08D
:10DF200004E100E0449FFF1FB89FFF1F034B1B68E5
:10DF3000DB0401D5FFF758BF704700BF34800440B1
:10DF400010B5044C237823B101F0C8FB2378002BD3
:10DF5000FAD110BDB09FFF1F054A064B10781B7801
:10DF6000C0B2DBB2984238BF4030C01A704700BF21
:10DF7000449FFF1F459FFF1F30B42B4B1A79940617
:10DF80001FD52A48DA790378294901333F2B0978CC
:10DF9000C8BF00238B42D2B203D0264CD9B2E25480
:10DFA0000170254A116861B1244A1278D2B29342B5
:10DFB00036BFC2F140029B1A9B18272BC4BF012316
:10DFC0000B70194AD378DBB2180611D45A060DD556
:10DFD000154B1B795B0609D5194B1A491B680022A2
:10DFE0000A7003B11A70104B2C22DA7030BC7047E3
:10DFF00011790906EAD5144910480C780178C9B29C
:10E000008C420DD04A1C272A84BF00210A460F4D9E
:10E01000054C98BFD1B2AA5CD2B2E2710170D5E7CB
:10E020006C21D170D2E700BF00C00640449FFF1FA3
:10E03000459FFF1F709FFF1F409FFF1FB19FFF1F46
:10E04000B49FFF1FB09FFF1FB89FFF1F489FFF1F78
:10E0500021282FD8184B195CFF292BD0174B184AB1
:10E06000DFF870C003EBC000F0B54368DFF868E08C
:10E07000144F154D154E00241C60DEF800300120B1
:10E0800043F020038840CEF8003014604FF4A073B2
:10E0900038602E60C2F800C0013BFDD113689B05BB
:10E0A000FCD42023013BFDD1094B09B233F8110008
:10E0B00080B2F0BD00207047A043010090420100F3
:10E0C0000050044008500440045004400000020383
:10E0D0000051044080014A0038800440431E032B55
:10E0E00014D872B60A4951F8230068B170B4094CCB
:10E0F000058834F81320466841F82360521B24F841
:10E10000132062B670BC704762B67047002070473B
:10E1100014A0FF1F7CA2FF1F013803280BD872B682
:10E12000074B53F8203043B100205B680130002BCF
:10E13000FBD162B67047002070471846F9E700BF70
:10E1400068A0FF1FF0B472B61A491B4E012311F8E4
:10E15000014B194F9A00240742F0010505D556F8E6
:10E16000324064B156F83520BAB10133052BEED1F7
:10E1700062B6124B00221A70F0BC00F0F1BC0F4CDA
:10E180000F4D217847F8325007EB431308304A1EF1
:10E190005860227062B6F0BC70470849094B0A7893
:10E1A00047F8353007EBC5030830013A58600A706C
:10E1B00062B6F0E7EC4301000080FF1F91A0FF1F53
:10E1C00088004000C8004000431E032B1DD81B4A96
:10E1D000400140F0100030B4104472B6184CE25CBC
:10E1E000032A1BD8DFE802F00212151703220D885C
:10E1F000E25410F0080F14BFC823882343EA0543F4
:10E2000008310360416062B630BC704708300222BA
:10E21000EDE70522EBE708300422E8E7094A52F867
:10E22000230038B1084A52F82300416042F8231015
:10E2300062B6E9E742F82310034AF7E70080FF1FC0
:10E24000A0A0FF1F68A0FF1F78A0FF1F00BE70479F
:10E250002DE9F04FDFF814A3DFF814B387B044E0E2
:10E26000AC4F4FEA930807EBC809013ED9F80420E8
:10E2700003F00803F6B2A2F1080003F0FF04002B3C
:10E2800040F0FE8057F838301B0C99B222F8081C79
:10E29000002B00F0EC80A04B22F8064C42F8044C16
:10E2A00053F82620002A00F0CD819C4D55F82630E9
:10E2B00058609B4C45F8260034F81630194424F871
:10E2C000161000F02DFC002800F0C081954A964BF6
:10E2D00019F0080F00F1080018BF1346C9F8040030
:10E2E00047F8383008238AF800309AF80040E4B242
:10E2F00061071CD58D4B1B78B3B18D490A7802F0AC
:10E30000FF0322B1013BDBB20B7003B900BE8949A8
:10E310000A7802F0FF032AB1013BDBB20B70002B3D
:10E3200000F0668100F0B6FC04238AF8003004F0A7
:10E33000080303F0FF02002B00F0C6809BF80030BA
:10E34000DBB21E098CD19A08724F57F8321007EBD6
:10E35000C200C1F38301013940680C2900F28380B7
:10E36000DFE801F07878818181818181428181813A
:10E3700007000168704D714B40680193694B47F885
:10E3800032306F4E686040F2816288B26B4B296018
:10E390000024012190421C603C61BC61317000F29C
:10E3A000E980B0F5D06F80F00F82B0F5817F00F08A
:10E3B000DA8100F26B81802800F00182822840F02F
:10E3C000D881A8885F4B00F07F00042800F2D2813A
:10E3D0005D4A80000344147054701878840740F13B
:10E3E00002831170022174E1544B01931A6832B315
:10E3F000564B534E564819883478057840298E4636
:10E4000045F0020828BF4FF0400E002C84F00104B4
:10E410003470CEEB01010CBF8824C82407EBC8067A
:10E4200089B285F0010544EA0E447260198047F80C
:10E43000384072440570002966D0019B1A603E4B3B
:10E440001A88B2F5A06F0ED100219A785970414B0D
:10E450001A7008E03849404C0D68A54200F09980D8
:10E46000304947F832103D4A012313703AE72D4AEC
:10E470002D4B19F0080F18BF134647F8383031E715
:10E4800000F06EFB364A374952F82630002B00F078
:10E49000E48058688C5D42F8260003F10802C9F850
:10E4A0000420032C05D8DFE804F02C0229260222E0
:10E4B0008A551A8819F0080F0CBF8823C82343EA2D
:10E4C000024347F838300DE7E00700F19480210659
:10E4D00000F1D280A20706D5234A244913780220EE
:10E4E000DBB213700870E30602D5204B10221A70BD
:10E4F00007B0BDE8F08F04228A55DAE705228A5575
:10E50000D7E703228A55D4E7BEF1400F18BF002297
:10E5100093E700BF0080FF1F14A0FF1FC09FFF1FD5
:10E520007CA2FF1FC8004000880040009CA0FF1F85
:10E5300025A0FF1F14A1FF1F88A0FF1FBC9FFF1F66
:10E5400024A0FF1FC020074094A0FF1FD09FFF1FE3
:10E5500090A0FF1F98200740210900039420074046
:10E5600068A0FF1FA0A0FF1F882007408020074051
:10E5700090200740B0F5106F00F03E8140F2A2807D
:10E5800040F62112904240F01C82A44A01231370ED
:10E5900069E74C68A2498C427FF462AF0178A929EF
:10E5A0007FF45EAF417845297FF45AAF8178C22964
:10E5B0007FF456AFC1786B297FF452AF99489A4ED9
:10E5C0000178347881F00105002C41F002010570DA
:10E5D0000CBF8820C82084F0010447F8310007EB05
:10E5E000C10192483470002505244D60047037E75E
:10E5F00000F0E0FE96E68E4B88488A491A614FF09B
:10E60000020E80F800E08B4F0A708B491960996008
:10E610008A4E8B4D8B4C9A610D213970FF213170E0
:10E62000DFF848E229702270874D884A8EF8001082
:10E630009F27012406F8047C5D600470DA6007B04F
:10E64000BDE8F08F43F82600814D32E6814A47F855
:10E65000380013780133137044E68B5D032B00F20E
:10E66000A78001A252F823F0E5E20000E5E20000F5
:10E67000BFE60000B9E600006E49714B80220D2014
:10E6800008701A70A2077FF52EAF25E740F202321C
:10E69000904240F08E81AA8802F07F02042A68D856
:10E6A0006D88002D65D16348029192001044027874
:10E6B00042F00202027048E101238B5512E600236A
:10E6C0008B550FE6B0F5086F53D16348634A007865
:10E6D0001070ED888D4280F09B815248047844F0A0
:10E6E000020C07EBCC01402DAE464FF0010328BFD2
:10E6F0004FF0400E4A6002EB0E09CEEB05014FEAE7
:10E700000E4802930025C82242EA080384F0010261
:10E7100047F83C3035700270DFF814C1424BDFF827
:10E72000048151BBBEF1400F7FF42FAF42F00202D3
:10E7300007EBC203DFF8F8E0C3F8049095BB0D04C3
:10E7400045F088059DF8083033704029047009EBC6
:10E7500001034EF832507FF418AF0021404A01986F
:10E760001180036011E7AA8802F07F02042A40F2B8
:10E770002D81304B0F221A7007E74029D6D942F07D
:10E7800002020CEBC200C0F804907DB135489DF840
:10E7900008501D70403988F8004009F140034CF8DA
:10E7A0003200DBE70D0445F0C805CBE72248EEE771
:10E7B00019F0080F0CBF022303238B5592E5274A5B
:10E7C00002211470547084E727494A68002AD0D087
:10E7D0006C88B5F804E003E00C314A68002AC8D020
:10E7E0000B88A342F8D14B887345F5D1240A032C3A
:10E7F0000CBF117809896CE7174A0D4CA978117084
:10E8000004F1800502E00834AC4231D0236A1A06D4
:10E81000F9D5606A083800F0A3F9F4E794200740BE
:10E820000100040090A0FF1F24A0FF1F25A0FF1FD0
:10E830000080FF1FC020074088004000882007405C
:10E840008020074098200740D49FFF1F28A0FF1F6B
:10E85000C09FFF1F91A0FF1F9CA0FF1F94A0FF1F40
:10E86000D09FFF1FC8004000F04301008C200740EC
:10E870006F49704B704A02917049714D714C059609
:10E8800003954FF00009884616461D4604942868F3
:10E8900028B1446800F064F92046002CF9D1002327
:10E8A0002B60039B30681A46002342F8293028B1B8
:10E8B000446800F055F92046002CF9D1002232605E
:10E8C000029A98F800301146002241F8042B049A6D
:10E8D0000291023B4FF0000122F81910032B07D8D8
:10E8E000DFE803F0470247024FF0010388F80030E9
:10E8F00009F10109B9F1040F05F1040506F1040657
:10E9000008F10108C3D1504B059EDFF85491DFF8A0
:10E91000548100211970012518F8013B09F8043BC6
:10E920001B072BD4AC0044F0020244F00304002384
:10E9300047F8323047F83430444B994505F101052A
:10E94000EAD13378029383F0010500218946884695
:10E950008E460A463E48047844F0020C07EBCC038E
:10E960000393029B002B039B5A600CBF8822C82292
:10E97000CAE64FF0000388F80030B9E700F0D0F89D
:10E98000AC0007EB451300F10802002837D05A60AD
:10E99000304B47F8343000F0C3F844F0010307EB84
:10E9A000C30200F1080100B351602B4A47F833203D
:10E9B000B9E7B0F5A06F7FF4DCAE01230025029328
:10E9C000C3E740F621229042F7D0D2E66D88002DB1
:10E9D0007FF4CFAE2148029192001044027822F0D9
:10E9E00002020270B1E7022173E6174B44F0010204
:10E9F0001B7847F83200144A0133137093E7124B27
:10EA0000114A1B78AC00013347F834001370C2E799
:10EA100040298E464FF0010328BF4FF0400ECEEB49
:10EA200001014FEA0E4802EB0E090025029391E71F
:10EA300078A0FF1F14A0FF1F68A0FF1FA0A0FF1F4A
:10EA4000C09FFF1F7CA2FF1F91A0FF1FD420074083
:10EA500090A0FF1F88004000C8004000C020074071
:10EA6000C4200740EC4301002DE9F843204C00F09E
:10EA7000AFFF002204F1880023461A605A60083371
:10EA800083424FF00001F8D11A4A1B4F13681B4D07
:10EA90001B481C4EDFF87880DFF878C0DFF87890EC
:10EAA000DFF878E043F480231360C4F307233B705E
:10EAB000C4F307432B70240EFF2302F528320470A1
:10EAC000114D88F8003011488CF80030D432337082
:10EAD000012389F8003070268EF800104FF400747E
:10EAE000102107F8183C2E7004601170BDE8F883FF
:10EAF0000080FF1F348004409C200740B020074066
:10EB0000B42007401020074049E400E008E100E09D
:10EB100080200740882007409420074000210740BC
:10EB200072B60D480268B2FA82F30F2B10DC4FF078
:10EB30000041D94022EA0102026062B6074803EBB5
:10EB4000C303DB00C2180021C1501046516070475A
:10EB500062B60020704700BF0C94FF1FBC83FF1FEC
:10EB60000D4B0E4AC31AA2FB03231B090F2B0CD813
:10EB70000B4A127852B972B60A484FF00041026847
:10EB800021FA03F31A43026062B67047064A12780C
:10EB9000002AF0D0FFF7D6BABC83FF1F398EE338C6
:10EBA00091A0FF1F0C94FF1F9CA0FF1F38B50E4BB8
:10EBB0000E4C1B68218805468BB1B1F5917F05D2BB
:10EBC0000B4A4B1C55549BB2238038BD0022084889
:10EBD00098470021064A55540123238038BDB1F5DA
:10EBE000917FEDD338BD00BFC8A0FF1F86A2FF1FD5
:10EBF0008CA2FF1F2DE9F843224E234F31680123D9
:10EC000080463B70C1B1214D4B8801EB830001333D
:10EC100000220F2BC0F808802A7004D84B800023F4
:10EC20003B70BDE8F88340230B800320FFF7CCFA4C
:10EC3000FFF776FF3060F2E7DFF8549099F8003084
:10EC4000002BEED0114D45F6215408E0013C12D0C6
:10EC50002B7883B900F042FD99F800307BB1032096
:10EC6000FFF75AFA0528F1D8FFF75AFF014630603E
:10EC70000028EBD0C8E701232B70BDE8F883BDE87E
:10EC8000F88300BFE4A0FF1FB8A0FF1FE8A0FF1F8C
:10EC90009CA0FF1F094B1B787BB910B5084C21685D
:10ECA00009B14B8803B910BD9B000B800320FFF70F
:10ECB0008BFAFFF735FF206010BD7047B8A0FF1F2B
:10ECC000E4A0FF1F2DE9F041AD4E33680746002B4D
:10ECD00000F092801D885A88910803EB810104326C
:10ECE000AA428C6842D25A8004F00F064FEA1428D8
:10ECF000A449A6F1080208F00F00C4F30313062A82
:10ED000000F101050B701AD9B31E012B5FFA88F0D0
:10ED10004ED9052E48D0042E00F0A481731F022B7B
:10ED20007FD90F2E0ED1F72842D8F02802D0964B6B
:10ED30001B883BB1FFF73AFF0020BDE8F08127B107
:10ED4000BD4202D00020BDE8F081082EC4F3033399
:10ED500000F08780092E11D00A2E40F094800A2BF3
:10ED6000F0D18A4B8A4A1B68A02181E01846FFF740
:10ED7000F7FE0420FFF7B2F93060B5E7092BE1D1C7
:10ED8000270E00F07B81834B814A1B689021C4F3DE
:10ED900007461170EDB2FCB2002B00F09D802246B8
:10EDA00031462846984797E0F02843D9F72841D0C4
:10EDB000F1380E28C6D801A353F820F073EF0000F5
:10EDC00057EF000045EF000045ED000045ED000065
:10EDD00037EF000045ED000017F0000045ED0000A2
:10EDE000E1EF0000FBEF00001FEF000045ED000029
:10EDF00007EF0000EBEE0000674B1B78002BA1D063
:10EE00000420FFF76BF90346306000289AD005888C
:10EE1000002D7FF460AFFFF7A3FE35602846BDE804
:10EE2000F081FFF7C3FEC4F30740FFF7BFFE072ED4
:10EE300002D1200EFFF7BAFE534B584A19885848A2
:10EE40001468584D524A017000270E0AF0201F80A6
:10EE50002E7010700CB301225348A0470120BDE86A
:10EE6000F081082B7FF46EAF504B494A1B6880211C
:10EE7000C4F307461170EDB2240E6BB32846224648
:10EE80003146984728E00B2E11D10B2B7FF45AAF57
:10EE9000474B3F4A1B68B021EAE7464B1B68002BF3
:10EEA00000F0FB80404898470120BDE8F0810C2E1F
:10EEB00040F000810C2B7FF445AF3F4B344A1B6878
:10EEC000C0211170EDB2C4F30746002B00F0C880DA
:10EED00028463146240E98473849314A314B0D7047
:10EEE00016701C700120BDE8F081354B1B68002BAB
:10EEF00000F0D6809847C4F30746254BEDB2240EA8
:10EF000083F80080E8E72F4B1B68002BF2D12E4BD3
:10EF10001B68A3B1FE209847C4F30746EDE72B4BCF
:10EF20001B68002BE6D1284B1B6843B1FC20984797
:10EF3000C4F30746E1E7264B1B68002BDAD1C4F384
:10EF40000746DAE7234B1B68C4F30746002BD4D0EF
:10EF500030469847D1E7204B1A68002AEFD0260C9C
:10EF6000630C06F07F0003F47E531843F6B290471B
:10EF7000C3E71A4B1B68C4F30746002BE8D1BCE774
:10EF8000F0A0FF1F8AA2FF1F86A2FF1FCCA0FF1FB9
:10EF900084A2FF1F00A1FF1F9CA0FF1FC8A0FF1F8E
:10EFA00088A2FF1F89A2FF1F8CA2FF1FF8A0FF1FCE
:10EFB000FCA0FF1FE0A0FF1FBCA0FF1F8BA2FF1F34
:10EFC000A8A0FF1FACA0FF1FB0A0FF1FECA0FF1F59
:10EFD000DCA0FF1FF4A0FF1FC4A0FF1FD8A0FF1FCD
:10EFE0003F4B1B68002B85D13E4B1B68002BA6D0E6
:10EFF000FA209847C4F307467FE73B4B1B68002B7A
:10F000007FF478AF374B1B68002B98D0FB209847D4
:10F01000C4F3074671E7354B1B68002B7FF46AAFDA
:10F02000304B1B68002B8AD0F8209847C4F3074662
:10F0300063E70E2B7FF486AE2D4A2E4B1268E0213B
:10F040001970002A47D0260C610C06F07F0301F4EA
:10F050007E511943EDB2A1F5005128469047F6B212
:10F06000240E39E7FFF7A2FDC4F30740FFF79EFD2A
:10F07000200EFFF79BFD0020BDE8F0811E4B1D4ACE
:10F080001B6880211170EDB2C4F3074683B131468D
:10F0900028463A4698473C461EE70120BDE8F081E5
:10F0A000104B1B68002B3FF44AAFFF20984746E700
:10F0B0001C4611E70D2EBCD10D2B7FF443AE0F4B38
:10F0C0000C4A1B68D0211170EDB2C4F30746002B27
:10F0D0007FF4FEAEC4E7C4F30746EDB2240EFBE6B0
:10F0E000D4A0FF1FB0A0FF1FB4A0FF1FA4A0FF1F4C
:10F0F000C0A0FF1F84A2FF1FF8A0FF1FD0A0FF1F0A
:10F1000070B5124E33788BB1114D286840B14388E9
:10F11000C218147A6CB9FFF723FD33782C602BB139
:10F120000220FEF7DBFF28600028F0D14FF0FF300F
:10F1300070BD02880133934202D24380204670BDE5
:10F14000FFF70EFD002320462B6070BD9CA0FF1F23
:10F1500010A1FF1F70B50D4E33788BB10C4D286890
:10F1600040B1438803441C7A6CB9FFF7F9FC33784B
:10F170002C602BB10220FEF7B1FF28600028F0D1EF
:10F180004FF0FF3070BD204670BD00BF9CA0FF1F38
:10F1900010A1FF1F38B5164D2868E0B101884488DA
:10F1A000A14213DD03191B7A83B104F10803C218CD
:10F1B0000C1B002302E012F8011F21B10133A3420E
:10F1C000F9D1204638BD1C46204638BDFFF7C8FCA3
:10F1D0000020286038BD074B1B780BB9002038BDD4
:10F1E0000220FEF77BFF28600028D7D1F6E700BF9A
:10F1F00010A1FF1F9CA0FF1F2DE9F04F3D4D0122E4
:10F2000083B02A7071B3DFF8F8A0DFF8F880DFF878
:10F21000E89083460E46DAF80000002835D0364BD9
:10F2200001934488019BC4F14001B14228BF31469B
:10F2300067180022BFB21A70761A478000F10802E0
:10F2400049B1013C224459441BF8014B02F8014FDB
:10F250005945F9D147883F2F09D8284B05221A7004
:10F26000002ED8D10020287003B0BDE8F08F4022D6
:10F27000224B02800146002401201C70FEF7A4FFEF
:10F28000CAF80040002EC6D1ECE798F800204AB337
:10F29000194B019344F2D95401270BE0013C17D0DC
:10F2A00099F80020A2B92A7000F018FA2F7098F887
:10F2B0000020BAB10120FEF72FFF0528EED82F70ED
:10F2C000FFF72EFCCAF800000028AAD1013CE7D1C4
:10F2D0000199012200234FF0FF300A702B7003B018
:10F2E000BDE8F08F00234FF0FF302B7003B0BDE876
:10F2F000F08F00BF04A1FF1F0CA1FF1F14A1FF1F6F
:10F3000008A1FF1F9CA0FF1F00B583B002AB012125
:10F3100003F8010D1846FFF76FFF03B05DF804FB1B
:10F3200038B50E4D0E4C2B68012020702BB158883B
:10F3300000232370C0F1400038BD0A4B1B7813B97D
:10F340000020207038BDFEF7E7FE0528F8D8FFF74B
:10F35000E7FB034628600028E9D1F1E708A1FF1F79
:10F3600004A1FF1F9CA0FF1F0F4B1B78DBB110B542
:10F370000E4C2168B1B14B88A3B10D4800223F2B40
:10F38000027007DC07330B4401F1470003F8012F3B
:10F390008342FBD140230B800120FEF715FF0023A1
:10F3A000236010BD10BD70479CA0FF1F08A1FF1F68
:10F3B00014A1FF1F0D4B1B78BBB910B50C4C216875
:10F3C00003F0FF024B883F2B07DC07330B4401F1AE
:10F3D000470003F8012F8342FBD140230B8001201B
:10F3E000FEF7F2FE0023236010BD704704A1FF1F4B
:10F3F00008A1FF1F10B4EFF3108272B6437F33B938
:10F40000017F012907D003290FD00123437702B9D7
:10F4100062B610BC7047124C2168A1B1114943611A
:10F420000B68836108605861EFE70F4C216881B178
:10F430000E4943610B688361086058610C4B4FF0C3
:10F4400080511960E1E7074B4161816120601860DC
:10F45000DBE7064B4161816120601860EEE700BF89
:10F4600028A1FF1F24A1FF1F18A1FF1F1CA1FF1F20
:10F4700004ED00E070B5EFF3108272B60C4C20681A
:10F4800080B10C4E00254369236073B19D6102B9C0
:10F4900062B6457783689847EFF3108272B62068AA
:10F4A0000028F0D102B962B670BD3360EFE700BF4B
:10F4B00018A1FF1F1CA1FF1FFFF7DCBF184A30B4C3
:10F4C0001468002C27D0036821688B420ED2CB1A17
:10F4D00000218460C1602360E06010600223037536
:10F4E00030BC704711688B42144608D3A2685B1A7F
:10F4F0000360002AF6D18260C460A060EEE7D268A3
:10F50000C2608460E060C568CB1A0222A8602360F4
:10F51000027530BC70478460C4601060DEE700BFD5
:10F5200020A1FF1FF8B5224E34682CB32368002BAE
:10F530003AD1204F1D4604E03468ECB12368002B1B
:10F5400032D1A36803B1DD6020693360036825759B
:10F550001B68BB4221D1037F4560022BC46020D0D1
:10F56000FFF748FF6368002BE6D023602046FFF7D3
:10F57000A5FF3468002CE1D1EFF3108372B60E4A78
:10F5800000211068116003B962B628B18468FFF7E2
:10F5900095FF20460028F9D1F8BD22460021984762
:10F5A000E0E783689847DDE7013B2360E4E700BFBD
:10F5B00020A1FF1F45B5000030A1FF1F024A1368BC
:10F5C00001331360FFF7AEBF3C9FFF1FF8B572B168
:10F5D00006460F4614460025336817F8011B1B68C2
:10F5E00030469847013C0544F6D12846F8BD1546FB
:10F5F000FBE700BF00B5064A036812885B6883B06A
:10F6000001A9ADF804200222984703B05DF804FB7D
:10F61000C4430100F0B507468BB0002A33D0012A5D
:10F6200008BF0A2251B3212400E0F4B2B1FBF2F585
:10F6300002FB1511C8B2092900F1300198BFC8B208
:10F640000AA988BF3730214488BFC0B201F8240C12
:10F65000661E2946002DE8D133B1013CE4B20AAB65
:10F6600023442D2203F8242C3B6801AA11195B685E
:10F670003846C4F1220298470BB0F0BD30228DF815
:10F6800025202124E8E70368C9B21B6898470BB01E
:10F69000F0BD00BF0029BABF49422D2300230A2232
:10F6A000FFF7B8BF08B5F2F7A5FCF9F7CDFF00F0FA
:10F6B00015F8FAE7FFF74EBDFFF722BDFFF76ABD69
:10F6C000FFF752BEFFF72CBE08461146FFF794BD68
:10F6D0000846FFF719BE00BF704700BF38B5224C7F
:10F6E000237803B138BD01232370FFF753FD70BBAE
:10F6F00000F042F840BB00F0D5F810BBFEF72CFC40
:10F70000E0B900232370EFF30583002BEAD1EFF378
:10F71000108172B6154B1868E0B1154C2278CAB941
:10F7200045691D6001232370C5B1AA6101B962B6A4
:10F7300000254577836898472570D3E700F08EF958
:10F74000DFE700F089F9D9E700F084F9D3E7FFF7A4
:10F75000C3FFCDE70029C5D162B638BD054B1D609A
:10F760000029E5D1E3E700BF34A1FF1F28A1FF1F57
:10F770002CA1FF1F24A1FF1F054A064B10781B7800
:10F78000C0B2DBB2984238BF4030C01A704700BFE9
:10F790003CA1FF1F3DA1FF1FF0B4384B1A7912F0B6
:10F7A000300F2CD072B6997D01F0FF0200293DD0B8
:10F7B00062B6334F334938780D78334E1C46C0B2A9
:10F7C000EDB2431C402BE17928BF0023AB4202F18C
:10F7D000FF32C9B21CBFF154184612F0FF02F0D13B
:10F7E0002A4B1B68C2B23A704BB1A84236BFC5F172
:10F7F0004005401B40192728C4BF01221A701F4929
:10F80000CA78D2B2150616D452060DD51B4B1B79F9
:10F810005B0609D51E4B1F491B6800220A7003B105
:10F820001A70164B3C22DA70F0BC70474022D9792E
:10F830005A7462B6E3E70B791C06E5D5164B174EF2
:10F840001C783378E4B2DBB29C420ED0144D01E058
:10F85000A3420AD00133402B28BF00230879E85C7B
:10F86000C0B2C871087D0728F2D9DBB203493370F2
:10F870000B79180644BF7C23CB70C5E700A0064077
:10F880003CA1FF1F3DA1FF1F80A1FF1F38A1FF1F4B
:10F89000C4A1FF1FC0A1FF1FC8A1FF1FC1A1FF1F5F
:10F8A00040A1FF1F054A064B10781B78C0B2DBB29F
:10F8B000984238BF4030C01A704700BF3CA2FF1FBB
:10F8C000D1A1FF1FF0B4384B1A7912F0300F2CD0B1
:10F8D00072B6997D01F0FF0200293DD062B6334F28
:10F8E000334938780D78334E1C46C0B2EDB2431C14
:10F8F000402BE17928BF0023AB4202F1FF32C9B2AD
:10F900001CBFF154184612F0FF02F0D12A4B1B68BD
:10F91000C2B23A704BB1A84236BFC5F14005401B98
:10F9200040192728C4BF01221A701F49CA78D2B2D1
:10F93000150616D452060DD51B4B1B795B0609D54F
:10F940001E4B1F491B6800220A7003B11A70164B28
:10F950003C22DA70F0BC70474022D9795A7462B602
:10F96000E3E70B791C06E5D5164B174E1C78337868
:10F97000E4B2DBB29C420ED0144D01E0A3420AD0A7
:10F980000133282B28BF00230879E85CC0B2C87176
:10F99000087D0728F2D9DBB2034933700B791806CA
:10F9A00044BF7C23CB70C5E700B006403CA2FF1FDC
:10F9B000D1A1FF1FFCA1FF1FCCA1FF1F40A2FF1F71
:10F9C000D0A1FF1F44A2FF1F3DA2FF1FD4A1FF1F14
:10F9D00070B584B072B6194B194D1A487022412681
:10F9E0000F2480211A702E701A4604701970137833
:10F9F0001B06FCD5144B186862B6144B144C984285
:10FA000098BF00EB800001A998BF40000A22FDF7D3
:10FA100051FC01A92046002311F8012B01333AB112
:10FA20000A2B20F8022FF7D11623237004B070BDE3
:10FA30005B00DBB2237004B070BD00BF0000024069
:10FA40000700024006000240080002407F9698002E
:10FA5000E894FF1F704700BF704700BF704700BFAA
:10FA60002DE9F043DFF8EC808BB006460F4600F03E
:10FA700073F898F90030013304460D4637D030460C
:10FA8000394600F0DFF9002831D02BA3D3E9002359
:10FA90003046394600F026FE814668BB28A3D3E9EC
:10FAA00000233046394600F0FFFD00B398F90030DE
:10FAB000254ACDF82090042400200021022BCDE916
:10FAC0000467CDE9026700940192CDE906012CD0CC
:10FAD000684600F0BDF940B3089B1BB101F0F4F992
:10FAE000089B0360DDE906010BB0BDE8F08320460A
:10FAF00029460BB0BDE8F083134A98F90030019213
:10FB000003210022CDE90467CDE902670091089244
:10FB10002BB90E4B4FF06042CDE90623D8E70C49D4
:10FB20000020022BCDE90601D2D101F0CDF922232C
:10FB30000360D1E7AFF30080EF39FAFE422E864032
:10FB400051302DD5104987C05C440100FFFFEF47BD
:10FB50000000F07FFE94FF1F2DE9F04FB04F21F021
:10FB60000042BA4283B00C464FEAD17605460DD921
:10FB7000AC4FBA4225D9C1F31303034340F0EF80E1
:10FB80000EB10020014603B0BDE8F08FA64B9A42AB
:10FB900000F2CC80A54B9A4200F2DE808AA3D3E922
:10FBA000002300F05DF90022A14B00F09BFD00282E
:10FBB00000F005812846214600229D4B00F050F9B7
:10FBC000E1E783A3D3E9002300F08CFD002840F097
:10FBD000CB802846214680A3D3E9002300F064FDB2
:10FBE0000028CED1934B284603EBC60821467CA3C0
:10FBF000D3E9002300F0E6FAD8E9002300F030F959
:10FC000000F07AFD804600F077FA77A3D3E900236D
:10FC100006460F4600F0D6FA02460B462846214615
:10FC200000F01CF972A3D3E90023CDE900013046AE
:10FC3000394600F0C7FA82468B4652465B46DDE9FC
:10FC4000000100F00BF905460C462A4623462846DB
:10FC5000214600F0B7FA68A3D3E9002306460F4611
:10FC600000F0B0FA66A3D3E9002300F0F7F83246BB
:10FC70003B4600F0A7FA64A3D3E9002300F0F0F8B4
:10FC800032463B4600F09EFA61A3D3E9002300F020
:10FC9000E5F832463B4600F095FA5FA3D3E900232E
:10FCA00000F0DEF832463B4600F08CFA02460B4686
:10FCB0002846214600F0D2F806460F46284621463F
:10FCC00032463B46B8F1000F56D000F07BFA324680
:10FCD00004460D463B4600204FF0804100F0BEF840
:10FCE00002460B462046294600F096FB02460B468C
:10FCF0005046594600F0B2F8DDE9002300F0AEF8B6
:10FD00000B4602464A49002000F0A8F86FF47F73C2
:10FD100098454FDA08F57A7801EB085100224FF048
:10FD2000B87300F04FFA03B0BDE8F08F424B9A422F
:10FD30003FF658AF414BF4002344D3E9002300F0D1
:10FD40008DF83F4BC6F101081C44CDE90001D4E910
:10FD500000ABC6EB080870E74FF0000875E70246F5
:10FD60000B4600F07DF80EE717A3D3E900231046F9
:10FD7000194600F027FA06E700F024FA0022804630
:10FD800089464FF080433046394600F067F8024616
:10FD90000B464046494600F03FFB2A46234600F00A
:10FDA0005DF802460B460020214900F057F803B0E9
:10FDB000BDE8F08F01EB085103B0BDE8F08F80463D
:10FDC00043E700BFAFF300809C7500883CE4377EBA
:10FDD000EF39FAFE422E864051302DD5104987C0AA
:10FDE000FE822B654715F73F0000E0FE422EE63FFE
:10FDF000763C7935EF39EA3DD0A4BE726937663E6C
:10FE0000F16BD2C541BDBB3E2CDE25AF6A56113F1A
:10FE100093BDBE166CC1663F3E5555555555C53F01
:10FE2000412E8640FFFFEF7F422ED63FFFFF2F3E41
:10FE30000000F03F60440100B1A2F03F80440100A7
:10FE40007044010041F0004101F58010C00F70477F
:10FE50000020704781F0004102E000BF83F00043C2
:10FE600030B54FEA41044FEA430594EA050F08BF55
:10FE700090EA020F1FBF54EA000C55EA020C7FEA19
:10FE8000645C7FEA655C00F0E2804FEA5454D4EB96
:10FE90005555B8BF6D420CDD2C4480EA020281EA60
:10FEA000030382EA000083EA010180EA020281EA98
:10FEB0000303362D88BF30BD11F0004F4FEA0131EA
:10FEC0004FF4801C4CEA113102D0404261EB4101F9
:10FED00013F0004F4FEA03334CEA133302D052427F
:10FEE00063EB430394EA050F00F0A780A4F101043B
:10FEF000D5F1200E0DDB02FA0EFC22FA05F2801875
:10FF000041F1000103FA0EF2801843FA05F359415A
:10FF10000EE0A5F120050EF1200E012A03FA0EFCD9
:10FF200028BF4CF0020C43FA05F3C01851EBE37103
:10FF300001F0004507D54FF0000EDCF1000C7EEB20
:10FF400000006EEB0101B1F5801F1BD3B1F5001F5E
:10FF50000CD349085FEA30004FEA3C0C04F101047D
:10FF60004FEA445212F5800F80F09A80BCF1004FA6
:10FF700008BF5FEA500C50F1000041EB045141EA28
:10FF8000050130BD5FEA4C0C404141EB010111F429
:10FF9000801FA4F10104E9D191F0000F04BF0146D4
:10FFA0000020B1FA81F308BF2033A3F10B03B3F1B2
:10FFB00020020CDA0C3208DD02F1140CC2F10C0242
:10FFC00001FA0CF021FA02F10CE002F11402D8BFA0
:10FFD000C2F1200C01FA02F120FA0CFCDCBF41EA6C
:10FFE0000C019040E41AA2BF01EB0451294330BD3B
:10FFF0006FEA04041F3C1CDA0C340EDC04F1140418
:020000021000EC
:10000000C4F1200220FA04F001FA02F340EA0300EE
:1000100021FA04F345EA030130BDC4F10C04C4F134
:10002000200220FA02F001FA04F340EA0300294614
:1000300030BD21FA04F0294630BD94F0000F83F45E
:10004000801306BF81F480110134013D4EE77FEA41
:10005000645C18BF7FEA655C29D094EA050F08BF8D
:1000600090EA020F05D054EA000C04BF194610466E
:1000700030BD91EA030F1EBF0021002030BD5FEAB2
:10008000545C05D14000494128BF41F0004130BDDA
:1000900014F580043CBF01F5801130BD01F000452E
:1000A00045F0FE4141F470014FF0000030BD7FEAA1
:1000B000645C1ABF194610467FEA655C1CBF0B469C
:1000C000024650EA013406BF52EA033591EA030FB3
:1000D00041F4002130BD00BF90F0000F04BF0021AB
:1000E000704730B54FF4806404F132044FF00005DE
:1000F0004FF0000150E700BF90F0000F04BF002157
:10010000704730B54FF4806404F1320410F00045BC
:1001100048BF40424FF000013EE700BF42004FEAB7
:10012000E2014FEA31014FEA02701FBF12F07F4334
:1001300093F07F4F81F06051704792F0000F14BF31
:1001400093F07F4F704730B54FF4607401F0004575
:1001500021F0004120E700BF50EA010208BF7047CC
:1001600030B54FF000050AE050EA010208BF7047C1
:1001700030B511F0004502D5404261EB41014FF42A
:10018000806404F132045FEA915C3FF4DCAE4FF02E
:1001900003025FEADC0C18BF03325FEADC0C18BF15
:1001A000033202EBDC02C2F1200300FA03FC20FA66
:1001B00002F001FA03FE40EA0E0021FA02F11444B3
:1001C000C1E600BF70B54FF0FF0C4CF4E06C1CEAC8
:1001D00011541DBF1CEA135594EA0C0F95EA0C0F3D
:1001E00000F0DEF82C4481EA030621EA4C5123EAB0
:1001F0004C5350EA013518BF52EA033541F48011DF
:1002000043F4801338D0A0FB02CE4FF00005E1FB91
:1002100002E506F00042E0FB03E54FF00006E1FBDB
:1002200003569CF0000F18BF4EF0010EA4F1FF041E
:10023000B6F5007F64F5407404D25FEA4E0E6D415E
:1002400046EB060642EAC62141EA55514FEAC5206F
:1002500040EA5E504FEACE2EB4F1FD0C88BFBCF5EB
:10026000E06F1ED8BEF1004F08BF5FEA500E50F19C
:10027000000041EB045170BD06F0004646EA010162
:1002800040EA020081EA0301B4EB5C04C2BFD4EB94
:100290000C0541EA045170BD41F480114FF0000E8D
:1002A000013C00F3AB8014F1360FDEBF002001F0FB
:1002B000004170BDC4F10004203C35DA0C341BDC75
:1002C00004F11404C4F1200500FA05F320FA04F047
:1002D00001FA05F240EA020001F0004221F000417B
:1002E00010EBD37021FA04F642EB06015EEA430EEE
:1002F00008BF20EAD37070BDC4F10C04C4F120051E
:1003000000FA04F320FA05F001FA04F240EA0200D0
:1003100001F0004110EBD37041F100015EEA430EA1
:1003200008BF20EAD37070BDC4F1200500FA05F2C1
:100330004EEA020E20FA04F301FA05F243EA020340
:1003400021FA04F001F0004121FA04F220EA02004F
:1003500000EBD3705EEA430E08BF20EAD37070BD95
:1003600094F0000F0FD101F00046400041EB010175
:1003700011F4801F08BF013CF7D041EA060195F057
:10038000000F18BF704703F00046520043EB030311
:1003900013F4801F08BF013DF7D043EA06037047FE
:1003A00094EA0C0F0CEA135518BF95EA0C0F0CD009
:1003B00050EA410618BF52EA4306D1D181EA03014F
:1003C00001F000414FF0000070BD50EA410606BF49
:1003D0001046194652EA430619D094EA0C0F02D18E
:1003E00050EA013613D195EA0C0F05D152EA0336D3
:1003F0001CBF104619460AD181EA030101F00041F1
:1004000041F0FE4141F470014FF0000070BD41F039
:10041000FE4141F4780170BD70B54FF0FF0C4CF413
:10042000E06C1CEA11541DBF1CEA135594EA0C0F32
:1004300095EA0C0F00F0A7F8A4EB050481EA030E7F
:1004400052EA03354FEA013100F088804FEA033366
:100450004FF0805545EA131343EA12634FEA022234
:1004600045EA111545EA10654FEA00260EF00041F5
:100470009D4208BF964244F1FD0404F5407402D247
:100480005B084FEA3202B61A65EB03055B084FEAD8
:1004900032024FF480104FF4002CB6EB020E75EBD5
:1004A000030E22BFB61A754640EA0C005B084FEAFD
:1004B0003202B6EB020E75EB030E22BFB61A75467A
:1004C00040EA5C005B084FEA3202B6EB020E75EBC5
:1004D000030E22BFB61A754640EA9C005B084FEA3D
:1004E0003202B6EB020E75EB030E22BFB61A75464A
:1004F00040EADC0055EA060E18D04FEA051545EA39
:1005000016754FEA06164FEAC30343EA52734FEAE1
:10051000C2025FEA1C1CC0D111F4801F0BD141EA5A
:1005200000014FF000004FF0004CB6E711F4801FBF
:1005300004BF01430020B4F1FD0C88BFBCF5E06F9F
:100540003FF6AFAEB5EB030C04BFB6EB020C5FEAAF
:10055000500C50F1000041EB045170BD0EF0004E04
:100560004EEA113114EB5C04C2BFD4EB0C0541EA36
:10057000045170BD41F480114FF0000E013C90E633
:1005800045EA060E8DE60CEA135594EA0C0F08BFF7
:1005900095EA0C0F3FF43BAF94EA0C0F0AD150EAF6
:1005A00001347FF434AF95EA0C0F7FF425AF104689
:1005B00019462CE795EA0C0F06D152EA03353FF4B1
:1005C000FDAE1046194622E750EA410618BF52EA2E
:1005D00043067FF4C5AE50EA41047FF40DAF52EA02
:1005E00043057FF4EBAE12E74FF0FF3C06E000BF9F
:1005F0004FF0010C02E000BF4FF0010C4DF804CDAC
:100600004FEA410C7FEA6C5C4FEA430C18BF7FEA6B
:100610006C5C1BD001B050EA410C0CBF52EA430C99
:1006200091EA030F02BF90EA020F0020704710F119
:10063000000F91EA030F58BF994208BF90422CBFA8
:10064000D8176FEAE37040F0010070474FEA410CA1
:100650007FEA6C5C02D150EA013C07D14FEA430CBF
:100660007FEA6C5CD6D152EA033CD3D05DF8040B30
:10067000704700BF8446104662468C461946634662
:1006800000E000BF01B5FFF7B7FF002848BF10F139
:10069000000F01BD4DF808EDFFF7F4FF0CBF01207E
:1006A00000205DF808FB00BF4DF808EDFFF7EAFFFA
:1006B00034BF012000205DF808FB00BF4DF808EDB5
:1006C000FFF7E0FF94BF012000205DF808FB00BFAA
:1006D0004DF808EDFFF7CEFF94BF012000205DF834
:1006E00008FB00BF4DF808EDFFF7C4FF34BF012041
:1006F00000205DF808FB00BF4FEA410212F500122E
:1007000015D211D56FF47873B3EB625212D94FEA58
:10071000C12343F0004343EA505311F0004F23FA42
:1007200002F018BF404270474FF00000704750EA97
:10073000013005D111F0004008BF6FF00040704754
:100740004FF00000704700BF4FEA4102B2F1E043B2
:1007500024BFB3F5001CDCF1FE5C0DD901F0004CA8
:100760004FEAC0024CEA5070B2F1004F40EB8300F8
:1007700008BF20F00100704711F0804F21D113F124
:100780003872BCBF01F00040704741F480114FEA5D
:100790005252C2F11802C2F1200C10FA0CF320FAE6
:1007A00002F018BF40F001004FEAC1234FEAD32303
:1007B00003FA0CFC40EA0C0023FA02F34FEA43036D
:1007C000CCE77FEA625307D150EA01331EBF4FF0F6
:1007D000FE4040F44000704701F0004040F0FE4011
:1007E00040F40000704700BF80F0004002E000BF0E
:1007F00081F0004142001FBF5FEA410392EA030F0C
:100800007FEA226C7FEA236C6AD04FEA1262D2EB55
:100810001363C1BFD218414048404140B8BF5B425A
:10082000192B88BF704710F0004F40F4000020F0F3
:100830007F4018BF404211F0004F41F4000121F009
:100840007F4118BF494292EA030F3FD0A2F1010253
:1008500041FA03FC10EB0C00C3F1200301FA03F191
:1008600000F0004302D5494260EB4000B0F5000FB4
:1008700013D3B0F1807F06D340084FEA310102F173
:100880000102FE2A51D2B1F1004F40EBC25008BF25
:1008900020F0010040EA03007047490040EB0000EF
:1008A00010F4000FA2F10102EDD1B0FA80FCACF11E
:1008B000080CB2EB0C0200FA0CF0AABF00EBC2501D
:1008C00052421843BCBFD0401843704792F0000F0B
:1008D00081F4000106BF80F400000132013BB5E75E
:1008E0004FEA41037FEA226C18BF7FEA236C21D0D4
:1008F00092EA030F04D092F0000F08BF0846704739
:1009000090EA010F1CBF0020704712F07F4F04D106
:10091000400028BF40F00040704712F100723CBF19
:1009200000F50000704700F0004343F0FE4040F443
:10093000000070477FEA226216BF08467FEA236301
:100940000146420206BF5FEA412390EA010F40F4EC
:10095000800070474FF0000304E000BF10F0004338
:1009600048BF40425FEA000C08BF704743F096431F
:1009700001464FF000001CE050EA010208BF70473A
:100980004FF000030AE000BF50EA010208BF7047C1
:1009900011F0004302D5404261EB41015FEA010CD6
:1009A00002BF84460146002043F0B64308BFA3F1CE
:1009B0008053A3F50003BCFA8CF2083AA3EBC253B0
:1009C00010DB01FA02FC634400FA02FCC2F12002CF
:1009D000BCF1004F20FA02F243EB020008BF20F006
:1009E0000100704702F1200201FA02FCC2F120026C
:1009F00050EA4C0021FA02F243EB020008BF20EA61
:100A0000DC7070474FF0FF0C1CEAD0521EBF1CEA8E
:100A1000D15392EA0C0F93EA0C0F6FD01A4480EA7C
:100A2000010C400218BF5FEA41211ED04FF0006365
:100A300043EA501043EA5111A0FB01310CF0004091
:100A4000B1F5000F3EBF490041EAD3715B0040EAB7
:100A5000010062F17F02FD2A1DD8B3F1004F40EB87
:100A6000C25008BF20F00100704790F0000F0CF05A
:100A7000004C08BF49024CEA502040EA51207F3A1E
:100A8000C2BFD2F1FF0340EAC250704740F40000F9
:100A90004FF00003013A5DDC12F1190FDCBF00F0EA
:100AA00000407047C2F10002410021FA02F1C2F198
:100AB000200200FA02FC5FEA310040F1000053EA34
:100AC0004C0308BF20EADC70704792F0000F00F082
:100AD000004C02BF400010F4000F013AF9D040EA88
:100AE0000C0093F0000F01F0004C02BF490011F41C
:100AF000000F013BF9D041EA0C018FE70CEAD1531A
:100B000092EA0C0F18BF93EA0C0F0AD030F0004C99
:100B100018BF31F0004CD8D180EA010000F000404D
:100B2000704790F0000F17BF90F0004F084691F00B
:100B3000000F91F0004F14D092EA0C0F01D1420245
:100B40000FD193EA0C0F03D14B0218BF084608D10E
:100B500080EA010000F0004040F0FE4040F4000058
:100B6000704740F0FE4040F4400070474FF0FF0CEB
:100B70001CEAD0521EBF1CEAD15392EA0C0F93EA32
:100B80000C0F69D0A2EB030280EA010C49024FEA84
:100B9000402037D04FF0805343EA111143EA10133D
:100BA0000CF000408B4238BF5B0042F17D024FF4F5
:100BB000000C8B4224BF5B1A40EA0C00B3EB510FD0
:100BC00024BFA3EB510340EA5C00B3EB910F24BFB9
:100BD000A3EB910340EA9C00B3EBD10F24BFA3EB3E
:100BE000D10340EADC001B0118BF5FEA1C1CE0D106
:100BF000FD2A3FF650AF8B4240EBC25008BF20F0B9
:100C0000010070470CF0004C4CEA50207F32C2BF0C
:100C1000D2F1FF0340EAC250704740F400004FF0A9
:100C20000003013A37E792F0000F00F0004C02BFDA
:100C3000400010F4000F013AF9D040EA0C0093F0A4
:100C4000000F01F0004C02BF490011F4000F013BFE
:100C5000F9D041EA0C0195E70CEAD15392EA0C0F66
:100C600008D142027FF47DAF93EA0C0F7FF470AF9E
:100C7000084676E793EA0C0F04D14B023FF44CAFE1
:100C800008466EE730F0004C18BF31F0004CCAD176
:100C900030F000427FF45CAF31F000437FF43CAFB2
:100CA0005FE700BF4FF0FF3C06E000BF4FF0010CD4
:100CB00002E000BF4FF0010C4DF804CD4FEA4002B6
:100CC0004FEA41037FEA226C18BF7FEA236C11D000
:100CD00001B052EA530C18BF90EA010F58BFB2EBB3
:100CE000030088BFC81738BF6FEAE17018BF40F033
:100CF000010070477FEA226C02D15FEA402C05D1E7
:100D00007FEA236CE4D15FEA412CE1D05DF8040B6B
:100D1000704700BF844608466146FFE70FB5FFF7FE
:100D2000C9FF002848BF10F1000F0FBD4DF808EDB6
:100D3000FFF7F4FF0CBF012000205DF808FB00BFA7
:100D40004DF808EDFFF7EAFF34BF012000205DF801
:100D500008FB00BF4DF808EDFFF7E0FF94BF01204E
:100D600000205DF808FB00BF4DF808EDFFF7D2FF4B
:100D700094BF012000205DF808FB00BF4DF808ED8E
:100D8000FFF7C8FF34BF012000205DF808FB00BF5B
:100D90004FEA40024FEA41037FEA226C02D15FEA48
:100DA000402C08D17FEA236C02D15FEA412C02D1AA
:100DB0004FF0000070474FF0010070474FEA4002CB
:100DC000B2F1FE4F0FD34FF09E03B3EB12620DD979
:100DD0004FEA002343F0004310F0004F23FA02F0E3
:100DE00018BF404270474FF00000704712F1610F8A
:100DF00001D1420205D110F0004008BF6FF0004061
:100E000070474FF00000704742000ED2B2F1FE4F23
:100E10000BD34FF09E03B3EB126209D44FEA0023C9
:100E200043F0004323FA02F070474FF00000704790
:100E300012F1610F01D1420202D14FF0FF30704731
:100E40004FF00000704700BF10B502FB01F100F049
:100E500071F80446D8B150F8042C22F00302043A89
:100E6000242A18D8132A14D900231B2A03604360AC
:100E700016D9242A8360C36011BF00F110020361F8
:100E8000436100F118020023136053609360204611
:100E900010BD0246F7E7002100F068FB204610BDB8
:100EA00000F10802EFE700BFF0B583B016461F4619
:100EB0000D460024FFF732F9009733462A46019485
:100EC00000F03CFE03B0F0BD014B1868704700BF56
:100ED0002899FF1F70B50F4E0F4D761BB61018BF27
:100EE000002405D0013455F8043B9847A642F9D1B7
:100EF0000A4E0B4D761B03F057FBB61018BF0024AB
:100F000006D0013455F8043B9847A642F9D170BD8C
:100F100070BD00BFB4450100B4450100C0450100EB
:100F2000B4450100024B0146186800F003B800BF49
:100F30002899FF1F2DE9F04F01F10B05162D83B005
:100F4000064640F29F8035F0070500F1BF80A942B8
:100F500000F2BC8000F058FBB5F5FC7FC0F09C822D
:100F60006B0A00F0BA80042B00F28381A80900F11B
:100F7000390E4FEA4E033830C44F07EB8303A3F119
:100F800008015C68A14207D1ACE0002A80F2AC8085
:100F9000E468A14200F0A680636823F003035A1BB3
:100FA0000F2AF2DDB9493C6901F1080E744500F0E1
:100FB000B381636823F003035A1B0F2A00F399815E
:100FC000002AC1F814E0C1F810E080F29E80B3F569
:100FD000007F80F06781DB0803F1010C01229B1088
:100FE00002FA03F34A6851F83C80C4F8088001EB28
:100FF000CC091A43A9F10803E3604A6041F83C4078
:10100000C8F80C40831001249C40944200F28A806E
:10101000144206D120F003006400144200F10400E1
:10102000FAD007EBC009CC468046DCF80C108C45A2
:1010300007D173E1002A80F28181C9688C4500F0F4
:101040006D814B6823F003035A1B0F2AF2DD0C4617
:10105000D1F80CC054F8088F4B1945F001054D60CC
:1010600042F00101C8F80CC03046CCF808807B6122
:101070003B61C3F80CE0C3F808E059609A5000F0F7
:10108000C5FA1FE0102921D800F0BEFA102506236A
:1010900002207E4F07EB8303A3F108025C689442B1
:1010A00000F045816368E168A56823F003032344E9
:1010B00030465A68E96042F001028D605A6000F0E3
:1010C000A5FA0834204603B0BDE8F08F00240C23B5
:1010D0002046336003B0BDE8F08F80234FF0400E10
:1010E0003F2049E770465DE72344E1685A68A568F8
:1010F00042F00102E96030468D605A6000F086FAE5
:101100000834204603B0BDE8F08F234430465A68C7
:1011100042F001025A6000F079FA0834204603B028
:10112000BDE8F08FBC68636823F00308A84504D3CA
:10113000C5EB08030F2B00F38C80554BDFF8609153
:101140001A68D9F8003001332A4404EB080A00F089
:10115000608102F580520F3222F47F6222F00F028A
:1011600011463046019200F043FCB0F1FF3F834648
:10117000019A00F05881824500F2FC80454B1968C5
:10118000DA451144196000F05381D9F80000DFF806
:1011900010E101301BBFCAEB0B0A5144CEF800B07E
:1011A00019601BF0070100F01781C1F10800C1F5BB
:1011B0008051834408315A44C2F30B02C2EB010947
:1011C00049463046019300F013FC431C019B00F09C
:1011D0003F81CBEB00024A4442F001021968C7F894
:1011E00008B04944BC42CBF804201960DFF8A49051
:1011F00016D0B8F10F0F40F2FD806268A8F10C0321
:1012000023F00703E01802F001024FF0050E1A4325
:101210000F2B6260C0F804E0C0F808E000F21C8107
:101220001D4BBC681A68914288BF19601B4B1A6835
:101230009142626888BF196022F003029542A2EBD6
:10124000050301D80F2B04DC304600F0DFF9002441
:1012500038E7621943F0010345F001056560304647
:10126000BA60536000F0D2F90834204603B0BDE8FC
:10127000F08F142B71D9542B00F2A480280B00F1AD
:101280006F0E4FEA4E036E3076E600BF2C99FF1FBB
:1012900050A2FF1F54A2FF1F4CA2FF1F48A2FF1F16
:1012A000389DFF1F5A0A042A5ED9142A00F2B3801F
:1012B00002F15C0149005B3207EB810C57F8211009
:1012C000DFF8DC81ACF1080C8C4500F088804A68BE
:1012D00022F00302934202D289688C45F7D1D1F8FB
:1012E0000CC07A68C4F80CC0A160CCF80840CC608F
:1012F00088E6631942F0010745F001056560304654
:101300004B610B61C3F80CE0C3F808E05F609A50D2
:10131000083400F07BF9D5E64A6873E608F1010865
:1013200018F0030F0CF1080C7FF47FAE30E0DC689E
:10133000A34208BF02303FF435AEB3E60B440C467F
:101340005A68C96854F8085F42F001025A60304692
:10135000E9608D6000F05AF9B4E603F15C0E03F128
:101360005B004FEA4E0307E69A0902F13901490092
:101370003832A1E7BC424A4B3FF400AF9C68626838
:1013800022F003025AE759F80839994540F0828063
:1013900010F0030F00F1FF30F5D17B6823EA04035E
:1013A0007B6064009C423FF6BDAE002C3FF4BAAEB9
:1013B0001C4240467FF435AE64001C4200F104003C
:1013C000FAD02EE6B3F5AA7F18D8E80B00F1780E14
:1013D0004FEA4E037730CFE54FF48051EBE6012121
:1013E000D8F80430921001FA02F21A43C8F8042027
:1013F000614677E70123CBF8043025E740F25452E9
:10140000934220D8A80C00F17D0E4FEA4E037C30A9
:10141000B2E51032A4E6542A26D81A0B02F16F0165
:1014200049006E3248E7BC68626822F0030205E7B3
:10143000CAF30B0000287FF4A8AE4244BB6842F018
:1014400001025A60ECE6FE234FF07F0E7E2093E50A
:1014500001224FF00009C1E604F10801304600F016
:1014600045FCD9F80010DBE6B2F5AA7F05D8DA0B07
:1014700002F17801490077321EE740F254518A4266
:1014800005D89A0C02F17D0149007C3214E7FE2157
:101490007E2211E77B6884E7E808431C5B00F8E5DF
:1014A0002C99FF1F8842F0B50DD98B1898420AD2AB
:1014B0008118002A51D09A1A13F8014D01F8014DF4
:1014C0009342F9D1F0BD0F2A48D941EA00039B07A6
:1014D00046D100F1100401F11003154653F8106CC9
:1014E00044F8106C53F80C6C44F80C6C53F8086C0E
:1014F00044F8086C103D53F8046C44F8046C0F2D4C
:1015000003F1100304F11004E8D8A2F1100323F052
:101510000F0302F00F0E1033BEF1030F1944034402
:1015200021D91E1F0D467446043C55F8047B46F82D
:10153000047F032CF8D8AEF1040424F0030404342F
:101540002344214402F0030262B1013B0A4411F832
:10155000014B03F8014F8A42F9D1F0BD0346F3E78E
:101560000346F2E7F0BD7246EEE700BF70B48407B1
:1015700046D0541E002A41D0CDB2034602E0621E7E
:10158000E4B3144603F8015B9A07F8D1032C2ED973
:10159000CDB245EA05250F2C45EA054519D903F1D9
:1015A00010022646103E0F2E42F8105C42F80C5CEA
:1015B00042F8085C42F8045C02F11002F2D8A4F18F
:1015C000100222F00F0204F00F041032032C134417
:1015D0000DD91E462246043A032A46F8045BFAD87F
:1015E000221F22F003020432134404F003042CB13E
:1015F000C9B21C4403F8011BA342FBD170BC704765
:1016000014460346C2E700BF704700BF704700BFE3
:101610002DE9F04F174683B0002900F0C1800E4637
:10162000814607F10B05FFF7EFFF56F804EC162D86
:101630002EF00304A6F1080840D810221546AF4248
:1016400041D8944275DAC94B996808EB0400884286
:10165000416800F0D98021F0010303445B68DB0797
:101660007DD51EF0010F35D039464846FFF762FCA4
:101670000746E0B156F8043C23F001034344A0F1CF
:1016800008029A4200F04481221F242A00F231818C
:10169000132A00F20481034632461168196051682A
:1016A000596092689A603146484600F01FFB4846F0
:1016B000FFF7ACFF384603B0BDE8F08F25F0070513
:1016C000002D2A46BBDA0C230020C9F8003003B0F5
:1016D000BDE8F08F56F8083CC3EB080ADAF804308E
:1016E00023F0030C04EB0C039342BDDB5746DAF8FE
:1016F0000C1057F8080F221F242AC160886000F2DE
:101700001781132A40F212813168CAF808107168F3
:10171000CAF80C101B2A00F22B8108360AF11002BD
:101720003168116071685160B16891603E461C4635
:10173000D046631B0F2B1DD8D8F8043003F00103EB
:1017400023434444C8F80430636843F001036360F2
:101750004846FFF75BFF304603B0BDE8F08F21F04D
:1017600003012144914221DBC36882680C46D360A7
:101770009A60DEE7D8F8042008EB050102F00102C8
:10178000154343F001020B44C8F804504A605A68FC
:1017900042F0010208315A60484600F0A7FAD7E744
:1017A000114603B0BDE8F04FFFF7C4BB1EF0010FB8
:1017B0007FF45AAF56F8083CC3EB080ADAF8043055
:1017C00023F0030C01EB0C0E96458BDBC36882689B
:1017D0005746D3609A6057F8081FDAF80C30CB6090
:1017E000221F242A996000F29980132A62D9336853
:1017F000CAF808307368CAF80C301B2A00F2A080BF
:1018000008360AF1100356E021F0030BA34405F15A
:101810001000834559DA1EF0010F7FF425AF56F80A
:10182000081CC1EB080ADAF8041021F0030CE344A9
:1018300058453FF757AF5746DAF80C1057F8080FDE
:10184000221F242AC160886000F2B480132A40F26B
:10185000A5803168CAF808107168CAF80C101B2AF4
:1018600000F2AF8008360AF1100231681160716829
:101870005160B16891600AEB0501C5EB0B0242F0C3
:10188000010299604A60DAF8043003F001031D4355
:101890004846CAF80450FFF7B9FE38465CE733689B
:1018A0000360736843601B2A27D800F1080306F120
:1018B0000802F2E63B4632681A6072685A60B26803
:1018C0009A603E467446D04633E708EB0501C5EB07
:1018D0000B0B4BF0010299604A6056F8043C03F090
:1018E00001031D43484646F8045CFFF78FFE30466F
:1018F00032E73146FFF7D6FDD5E6B3688360F3687B
:10190000C360242A28D000F1100306F11002C4E6B7
:1019100050F8043C23F003031C440AE731463846E0
:101920007446D046FFF7BEFD3E4602E73A46F7E66C
:10193000314638461C46D046FFF7B4FD3E46F8E631
:10194000B368CAF81030F368CAF81430242A1BD0E0
:1019500010360AF11803AEE7336903617369436116
:1019600006F1180200F1180397E600BF2C99FF1F3B
:10197000B168CAF81010F168CAF81410242A0FD000
:1019800010360AF11802CBE63369CAF818307369C9
:10199000CAF81C3018360AF120038CE73A4664E78F
:1019A0003269CAF818207269CAF81C2018360AF180
:1019B0002002B5E6314638460193FFF773FD019BDF
:1019C00059E7B168CAF81010F168CAF81410242A4F
:1019D00003D010360AF1180247E73269CAF8182016
:1019E0007269CAF81C2018360AF120023DE700BFD0
:1019F00038B5074C0023054608462360FBF724FC56
:101A0000431C00D038BD2368002BFBD02B6038BDB1
:101A1000B0A3FF1FFFFFFFFFFFFFFFFFFFFFFFFF61
:101A2000FFFFFFFFFFFFFFFFFFFFFFFFFFFFFFFFC6
:101A3000FFFFFFFFFFFFFFFFFFFFFFFFFFFFFFFFB6
:101A400090F800F06DE9024520F007016FF0000CFE
:101A500010F0070491F820F040F049804FF00004A6
:101A60006FF00700D1E9002391F840F000F1080081
:101A700082FA4CF2A4FA8CF283FA4CF3A2FA8CF3B9
:101A80004BBBD1E9022382FA4CF200F10800A4FA20
:101A90008CF283FA4CF3A2FA8CF3E3B9D1E9042374
:101AA00082FA4CF200F10800A4FA8CF283FA4CF3AB
:101AB000A2FA8CF37BB9D1E9062301F1200182FA65
:101AC0004CF200F10800A4FA8CF283FA4CF3A2FA6B
:101AD0008CF3002BC6D0002A04BF04301A4612BA79
:101AE000B2FA82F2FDE8024500EBD2007047D1E97C
:101AF000002304F00305C4F100004FEAC50514F00B
:101B0000040F91F840F00CFA05F562EA05021CBFDB
:101B100063EA050362464FF00004A9E7024B13B1E4
:101B2000024800F005B8704700000000291C0100C1
:101B3000002301461A46184600F0CEBC2DE9F047B6
:101B400088B0364C119DD4F8009006460F461446D6
:101B50009846002D43D00022314B30463946FEF7DF
:101B6000A3FD80BB0DF11C0E0321109B039300917C
:101B70003B46CDF80880019432464846CDF810E047
:101B800000F092FD079BD8F800109842C1F10001C7
:101B90002ED2491B2B4610F8012B03F8012B079A74
:101BA000824203EB0106F6D8B44224DDA21B1A449C
:101BB000302103F8011B9A42FBD100231370284601
:101BC00008B0BDE8F0870022164B30463946FEF7D4
:101BD00089FD0028C6D00DF11C0E0221C5E7D9F8F9
:101BE000502004F123039A4207DDD9F85450B2E79C
:101BF0000E462B46D8E71A46DFE704F1240A524680
:101C0000D9F854104846FFF703FD05460028D6D002
